:020000040800F2
:1000000000800020F53E0008393F0008D93C000878
:10001000393F0008393F0008393F00080000000060
:100020000000000000000000000000000196000831
:10003000393F00080000000091960008D59600089E
:10004000393F0008393F0008393F0008393F0008B0
:10005000393F0008393F0008D11B0008F11B000898
:10006000091C00080B1C00080D1C0008393F000883
:10007000393F0008393F0008393F0008393F000880
:10008000393F0008393F0008393F0008393F000870
:10009000393F0008393F0008393F0008251C000897
:1000A000393F0008393F0008393F0008393F000850
:1000B000393F0008393F0008393F0008393F000840
:1000C000393F0008393F0008393F0008393F000830
:1000D000393F0008395F000851630008393F0008C4
:1000E000811C0008E5580008393F0008393F000826
:1000F000393F000800000000000000000000000080
:1001000000000000000000005FF808F108B5034897
:1001100007F040F8BDE8084006F048B9C15F0108A3
:1001200006F044B970B515460022C0E90115027009
:10013000C0E90332C0E90522C0E907224262DDE9D5
:100140000412044600F11C0610F04EF838B9294696
:10015000074807F01FF82B21064803F041FDDDE9B1
:1001600004233146204610F02CF8204670BD00BF15
:10017000DF5F01080A60010810B50446C06910B1CC
:10018000012111F0BBFA206910B1012111F0B6FA7A
:10019000204610BD2DE9F04100259DF81860C0E90A
:1001A00001120570C0E90335C0E90555C0E90755DE
:1001B000456231460446174600F11C080FF068FE00
:1001C00038B93946074806F0E5FF2021064803F014
:1001D00007FD3246414620460FF048FE2046BDE866
:1001E000F08100BFDF5F01080A600108F8B5002553
:1001F000C0E901120570C0E90335C0E90555C0E941
:100200000755456206990446164600F11C070FF093
:100210002BFF38B93146074806F0BCFF20210648BD
:1002200003F0DEFC069A394620460FF007FF204611
:10023000F8BD00BFDF5F01080A6001082DE9F04149
:10024000884B9EB0D3E9001214331B6881EA020484
:100250005C400EAE0094844806F09CFF2146304678
:100260000CF0CAF8304601F047FD10F0F9FB012709
:1002700005464FF0080804AC7C4B7D4A3946009790
:100280002046FFF787FF2146284610F08FFC2046C6
:10029000FFF772FFCDE900681026764B04211A465D
:1002A0002046FFF73FFF2146284610F07FFC2046FE
:1002B000FFF762FF14AB00936F4B04211A46CDF891
:1002C00004802046FFF72EFF2146284610F06EFCE2
:1002D0002046FFF751FF10AB0093684B01961A467A
:1002E00004212046FFF71EFF2146284610F05EFC41
:1002F0002046FFF741FF16AB614A019600930421A7
:10030000604B2046FFF70EFF2146284610F04EFCBA
:100310002046FFF731FF1AAB5B4A01960093042198
:10032000584B2046FFF7FEFE2146284610F03EFCC3
:100330002046FFF721FF04210FAB544A019100939F
:100340002046504BFFF7EEFE2146284610F02EFCCB
:100350002046FFF711FF0B234D4A009302214D4B1E
:100360002046FFF743FF2146284610F01FFC204699
:10037000FFF702FF0E230026474A00930221474B56
:100380002046FFF733FF2146284610F00FFC204699
:10039000FFF7F2FE424B434A394600962046FFF7EC
:1003A000F9FE2146284610F001FC2046FFF7E4FE46
:1003B00003233D4F05933D4B3D4920468DF810608A
:1003C0000697CDE90736CDE90966CDE90B660D96AE
:1003D0000FF0F2FE38B93946364806F0DBFE202130
:1003E000354803F0FDFB324A0BA920460FF0B4FE5E
:1003F0002146284610F0DAFB2046FFF7BDFE002319
:100400002E4A009301212E4B2046FFF7C3FE2146C2
:10041000284610F0CBFB2046FFF7AEFE0121294B0A
:10042000294A00912046FFF7B5FE2146284610F0E4
:10043000BDFB2046FFF7A0FE2846244B244A254951
:1004400010F080FA244B0493244B0593244B06931D
:10045000244B009394E80700052310F05DFD1EB0C7
:10046000BDE8F0815000F81FE45D0108075E010857
:100470001A5E01081F5E0108265E01082D5E010854
:10048000345E0108165E01083C5E0108445E010806
:10049000735E01084B5E01089F5E0108765E0108ED
:1004A000A75E0108D05E0108D95E0108E55E01087B
:1004B0001E5F0108DF5F01080A600108575F01083D
:1004C0002D5F0108685F01088A5F010821010008AB
:1004D000975F0108BB5F0108A1520008295200087C
:1004E0000D0100080000080807B58DF8041001A9E7
:1004F0008DF805208DF8063002F09CFA03B05DF807
:1005000004FB00002DE9F04F85B0FFF797FEFA20BD
:100510000AF002FB10F0BEFA0FF0CAFE5E4806F0C9
:1005200039FE10F0B7FA5D4B5D4A5E4E1A605E4AC6
:1005300005465A605D4A5E4C9A605E4A1A615E4AA0
:10054000DA605E4A5A61336813F0010F04D102F099
:100550009BF90123206033605049206802F040F885
:1005600057492846266810F05AF95649024601A80C
:1005700002F018F801A9304602F0A2F8524B01A986
:100580000193524B82462068029302F097F9504B38
:10059000DFF8689101934F4B89F8000001A92068AA
:1005A000029302F08BF94C4B4C4E01934C4B307044
:1005B00001A92068029302F081F94A4B4A4F019346
:1005C0000023387001A92068029302F077F9DFF860
:1005D0003081464988F80000284610F0FDF8444D67
:1005E00099F80010F0B120682A7880F84410337828
:1005F000FFF77AFF31782A780B462068FFF774FFFF
:10060000206802F0CDFB3B4806F0C4FD01224FF408
:10061000FA71206802F098FB002009F0F7FF05B09E
:10062000BDE8F08F2068DFF8DCB080F8441003F0FC
:10063000C7F999F800109BF800302A782068FFF776
:1006400053FF33782A789BF800102068FFF74CFF9F
:100650003B782A7831782068FFF746FFDFF8A890CA
:10066000254A99F80030127839782068FFF73CFF66
:100670003B782A7899F800102068FFF735FF98F842
:1006800000302A7839782068FFF72EFF33785246F9
:1006900098F80010B1E700BFEC61010804040020E5
:1006A000155B0008B8030020491B0008555C0008D2
:1006B00000040020E55B0008B15B0008D958000881
:1006C000D95E01080962010815620108B90700082E
:1006D0001A620108150900081F6201081E040020A3
:1006E000450A00082662010820040020D05E0108A7
:1006F000170600202C620108160600201C040020AA
:100700001F04002080080020810800207FB5204BB6
:10071000684603931F4B02931F4B00931F4B01939B
:100720001F4B04931F4B059303F084FB18B9212141
:100730001D4803F055FAE02003F072FB1B4B1870C4
:1007400010B31B4806F026FDFF21E02003F0C4FB98
:100750002D21E02003F0BBFBFA2004F043FD3521FE
:10076000E02003F0B4FBFA2004F03CFD3921E02046
:1007700003F0ADFBFA2004F035FD3D21E02003F04D
:10078000A6FB07B05DF804FB0A4806F003FDF8E796
:10079000511D000899580008615800087D5800084C
:1007A000C5570008FD570008DC6001081D04002043
:1007B000276101084861010808B500F08DFA00F0D2
:1007C000A5FAFFF7A3FF00F05FFA014B187808BD08
:1007D0001706002008B50A4B1B7863B1094806F0DC
:1007E000D9FCFF21E02003F077FBBDE808403D2164
:1007F000E02003F06CBB0448BDE8084006F0CABC2A
:100800001D0400206D6101089A6101082DE9F04F77
:1008100085B01F46904606460D4610F03BF904464B
:100820003A46414601A810F0F1FE374B01A819786D
:1008300010F012FF354920460FF0CEFF814601F03F
:10084000ABFC01F049FD347882460CBB05F1010890
:100850002B78A3421CDD4046514600F0A5F94FEA33
:10086000C40B08F1080868B3B9F1000F06D00BF10A
:1008700002010622294401A810F0D4FE05EB44042D
:10088000B4F9021101A810F0F6FE33780133337089
:10089000B9F1000F14BF082302233478FF1A2B7814
:1008A000A34209D901A810F0E4FEB8420CD329787C
:1008B0001748091B06F06EFC01A810F0DAFE05B01F
:1008C000BDE8F08F0134C3E74FEAC40808F1010026
:1008D0005146284400F068F998B9B9F1000F06D0E4
:1008E00008F102010622294401A810F09BFE05EB45
:1008F0004403B3F9021101A810F0BDFE33780133AF
:1009000033700134E4B2CAE7680500208A5F010849
:10091000CB61010870B52B4BC0B21B788EB09842EA
:1009200003D100F0D9F900F0F1F905F0F3F8264B06
:10093000C3E9000100F0A8F901F02EFC044610F014
:10094000A9F822490FF048FF30B9204601F0C4FC55
:1009500001461F4811F0F8F900F02EF900F07CF97B
:10096000002000F037FE012203211A4804F05CFE4B
:10097000002000F04BFE02221648114604F054FEFF
:10098000FFF728FF00230124114D134E8DF803308B
:100990002B789DF80320934210D92146304606F06B
:1009A000F9FB322301AA29460DF10300FFF72EFFC0
:1009B000014601A806F054FC0134E9E7074B18781A
:1009C0000EB070BD1F04002008000020575F010812
:1009D00026040020000002404360010817060020A2
:1009E0001FB50A22144901A810F010FE002101A829
:1009F00010F032FE022101A810F02EFE002101A805
:100A000010F02AFE0D4B01A8B3F9001010F033FED0
:100A10000B4B01A8198810F03AFE01A810F027FE30
:100A2000044601A810F025FE21460246012002F0EE
:100A3000E9FE04B010BD00BFF30300202204002033
:100A4000240400202DE9F048254BC0B21B78254E28
:100A5000984204D1244806F09DFB00233370234FB5
:100A60003478D7E90001B1F1004F08BF0028204DCC
:100A70000BD0D5E90023121A63EB01039C46002139
:100A80001C48904271EB0C030DDA21461A4806F01F
:100A900081FBD5E90023C7E90023FFF7A1FF174B2E
:100AA0001878BDE8F088164D2B78A34212D9294654
:100AB0003223144A0B48FFF7A9FE07463278611C1F
:100AC0002B78114806F066FB3A460E49022002F0E8
:100AD00099FEE4E721460D4806F05CFB0C4BDFE78E
:100AE0001E040020F20300207360010800000020B3
:100AF00008000020085101008E6001081606002041
:100B000026040020C0030020A0600108BF60010887
:100B10001706002013B500F0DFFD01F03DFB0124B6
:100B200003689B689847124B4FF4967201931149E2
:100B300000230094104809F07BFC4FF0FF31204661
:100B400001F046F94FF4FA7004F04CFB4FF0FF311E
:100B5000002001F03DF9094806F01CFB084806F0AA
:100B600019FBC82004F03EFB09F03CFEFEE700BF85
:100B7000BC03002046620108050500084F62010819
:100B800062620108FF23044A1370044A1370044A86
:100B90001370044A137070471C04002020040020C6
:100BA0001E0400201F04002008B5082200F0C8F829
:100BB000B0FA80F0400908BD38B5064C25683DB94B
:100BC000042010F08FFD40F6E44305704380206060
:100BD000206838BD6C0500200378F7B504465BBB80
:100BE00004F0EEF9184900F085FB00F0D3FC85B263
:100BF000284600F02BFB144900F030FC00F014FAFA
:100C0000064660880F4600F021FB0F4900F026FCE5
:100C100000F00AFA3B46CDE9000132460B4806F0E7
:100C2000B9FA6388AB4209D9094806F0B3FA012042
:100C300000F080FF0123237003B0F0BD054803B02E
:100C4000BDE8F04006F0A6BA00007A44FF62010851
:100C5000356301084E630108037810B504463BB1C3
:100C6000044806F097FA002000F064FF0023237088
:100C700010BD00BF6663010808B5FFF79DFFBDE822
:100C80000840FFF7E9BF0000002310B50F4C2370A8
:100C9000FFF792FFFFF7A0FF012000F0B7FC0C4820
:100CA00010F096FF0A4810F0E1FF094810F060FFCD
:100CB00038B1074811F07AF801232370FFF7DCFF01
:100CC00010BD044806F066FAF8E700BF680500208A
:100CD00026040020D662010810B5FFF7CDFF04F00E
:100CE0006FF9074900F006FB00F054FC84B221467E
:100CF000044806F04FFA044B20461C8010BD00BF8C
:100D000000007A44BB6201082404002010B50020D2
:100D100000F07CFCFFF750FFFFF75EFF10F0F0FEE5
:100D20000446FFF7A9FF2146034806F033FA034BB8
:100D300020461C8010BD00BF9362010822040020E1
:100D400030B50024A24201D1002007E0035D013448
:100D50000D1915F8015CAB42F4D0581B30BD0000F2
:100D600081F0004102E000BF83F0004330B54FEA5C
:100D700041044FEA430594EA050F08BF90EA020FC9
:100D80001FBF54EA000C55EA020C7FEA645C7FEA5C
:100D9000655C00F0E2804FEA5454D4EB5555B8BF7F
:100DA0006D420CDD2C4480EA020281EA030382EAF0
:100DB000000083EA010180EA020281EA0303362D82
:100DC00088BF30BD11F0004F4FEA01314FF4801C55
:100DD0004CEA113102D0404261EB410113F0004F67
:100DE0004FEA03334CEA133302D0524263EB43031E
:100DF00094EA050F00F0A780A4F10104D5F1200EBC
:100E00000DDB02FA0EFC22FA05F2801841F1000116
:100E100003FA0EF2801843FA05F359410EE0A5F1EA
:100E200020050EF1200E012A03FA0EFC28BF4CF01B
:100E3000020C43FA05F3C01851EBE37101F00045D1
:100E400007D54FF0000EDCF1000C7EEB00006EEBDE
:100E50000101B1F5801F1BD3B1F5001F0CD3490868
:100E60005FEA30004FEA3C0C04F101044FEA4452BF
:100E700012F5800F80F09A80BCF1004F08BF5FEA46
:100E8000500C50F1000041EB045141EA050130BD26
:100E90005FEA4C0C404141EB010111F4801FA4F1C9
:100EA0000104E9D191F0000F04BF01460020B1FA1E
:100EB00081F308BF2033A3F10B03B3F120020CDA56
:100EC0000C3208DD02F1140CC2F10C0201FA0CF034
:100ED00021FA02F10CE002F11402D8BFC2F1200C99
:100EE00001FA02F120FA0CFCDCBF41EA0C0190404F
:100EF000E41AA2BF01EB0451294330BD6FEA040498
:100F00001F3C1CDA0C340EDC04F11404C4F1200282
:100F100020FA04F001FA02F340EA030021FA04F394
:100F200045EA030130BDC4F10C04C4F1200220FAEB
:100F300002F001FA04F340EA0300294630BD21FA29
:100F400004F0294630BD94F0000F83F4801306BFEF
:100F500081F480110134013D4EE77FEA645C18BFE3
:100F60007FEA655C29D094EA050F08BF90EA020F7A
:100F700005D054EA000C04BF1946104630BD91EA72
:100F8000030F1EBF0021002030BD5FEA545C05D175
:100F90004000494128BF41F0004130BD14F58004B4
:100FA0003CBF01F5801130BD01F0004545F0FE4128
:100FB00041F470014FF0000030BD7FEA645C1ABF5D
:100FC000194610467FEA655C1CBF0B46024650EA94
:100FD000013406BF52EA033591EA030F41F40021C0
:100FE00030BD00BF90F0000F04BF0021704730B546
:100FF0004FF4806404F132044FF000054FF000011B
:1010000050E700BF90F0000F04BF0021704730B5DB
:101010004FF4806404F1320410F0004548BF4042B0
:101020004FF000013EE700BF42004FEAE2014FEA05
:1010300031014FEA02701FBF12F07F4393F07F4FE0
:1010400081F06051704732F07F4208BF704793F0E3
:101050007F4F04BF41F40021704730B54FF46074F6
:1010600001F0004521F000411CE700BF50EA0102F9
:1010700008BF704730B54FF000050AE050EA0102A2
:1010800008BF704730B511F0004502D5404261EB12
:1010900041014FF4806404F132045FEA915C3FF453
:1010A000D8AE4FF003025FEADC0C18BF03325FEAF0
:1010B000DC0C18BF033202EBDC02C2F1200300FAA1
:1010C00003FC20FA02F001FA03FE40EA0E0021FAC6
:1010D00002F11444BDE600BF80F0004002E000BF12
:1010E00081F0004142001FBF5FEA410392EA030F13
:1010F0007FEA226C7FEA236C6AD04FEA1262D2EB5D
:101100001363C1BFD218414048404140B8BF5B4261
:10111000192B88BF704710F0004F40F4000020F0FA
:101120007F4018BF404211F0004F41F4000121F010
:101130007F4118BF494292EA030F3FD0A2F101025A
:1011400041FA03FC10EB0C00C3F1200301FA03F198
:1011500000F0004302D5494260EB4000B0F5000FBB
:1011600013D3B0F1807F06D340084FEA310102F17A
:101170000102FE2A51D2B1F1004F40EBC25008BF2C
:1011800020F0010040EA03007047490040EB0000F6
:1011900010F4000FA2F10102EDD1B0FA80FCACF125
:1011A000080CB2EB0C0200FA0CF0AABF00EBC25024
:1011B00052421843BCBFD0401843704792F0000F12
:1011C00081F4000106BF80F400000132013BB5E765
:1011D0004FEA41037FEA226C18BF7FEA236C21D0DB
:1011E00092EA030F04D092F0000F08BF0846704740
:1011F00090EA010F1CBF0020704712F07F4F04D10E
:10120000400028BF40F00040704712F100723CBF20
:1012100000F50000704700F0004343F0FE4040F44A
:10122000000070477FEA226216BF08467FEA236308
:101230000146420206BF5FEA412390EA010F40F4F3
:10124000800070474FF0000304E000BF10F000433F
:1012500048BF40425FEA000C08BF704743F0964326
:1012600001464FF000001CE050EA010208BF704741
:101270004FF000030AE000BF50EA010208BF7047C8
:1012800011F0004302D5404261EB41015FEA010CDD
:1012900002BF84460146002043F0B64308BFA3F1D5
:1012A0008053A3F50003BCFA8CF2083AA3EBC253B7
:1012B00010DB01FA02FC634400FA02FCC2F12002D6
:1012C000BCF1004F20FA02F243EB020008BF20F00D
:1012D0000100704702F1200201FA02FCC2F1200273
:1012E00050EA4C0021FA02F243EB020008BF20EA68
:1012F000DC7070474FF0FF0C1CEAD0521EBF1CEA96
:10130000D15392EA0C0F93EA0C0F6FD01A4480EA83
:10131000010C400218BF5FEA41211ED04FF000636C
:1013200043EA501043EA5111A0FB01310CF0004098
:10133000B1F5000F3EBF490041EAD3715B0040EABE
:10134000010062F17F02FD2A1DD8B3F1004F40EB8E
:10135000C25008BF20F00100704790F0000F0CF061
:10136000004C08BF49024CEA502040EA51207F3A25
:10137000C2BFD2F1FF0340EAC250704740F4000000
:101380004FF00003013A5DDC12F1190FDCBF00F0F1
:1013900000407047C2F10002410021FA02F1C2F19F
:1013A000200200FA02FC5FEA310040F1000053EA3B
:1013B0004C0308BF20EADC70704792F0000F00F089
:1013C000004C02BF400010F4000F013AF9D040EA8F
:1013D0000C0093F0000F01F0004C02BF490011F423
:1013E000000F013BF9D041EA0C018FE70CEAD15321
:1013F00092EA0C0F18BF93EA0C0F0AD030F0004CA1
:1014000018BF31F0004CD8D180EA010000F0004054
:10141000704790F0000F17BF90F0004F084691F012
:10142000000F91F0004F14D092EA0C0F01D142024C
:101430000FD193EA0C0F03D14B0218BF084608D115
:1014400080EA010000F0004040F0FE4040F400005F
:10145000704740F0FE4040F4400070474FF0FF0CF2
:101460001CEAD0521EBF1CEAD15392EA0C0F93EA39
:101470000C0F69D0A2EB030280EA010C49024FEA8B
:10148000402037D04FF0805343EA111143EA101344
:101490000CF000408B4238BF5B0042F17D024FF4FC
:1014A000000C8B4224BF5B1A40EA0C00B3EB510FD7
:1014B00024BFA3EB510340EA5C00B3EB910F24BFC0
:1014C000A3EB910340EA9C00B3EBD10F24BFA3EB45
:1014D000D10340EADC001B0118BF5FEA1C1CE0D10D
:1014E000FD2A3FF650AF8B4240EBC25008BF20F0C0
:1014F000010070470CF0004C4CEA50207F32C2BF14
:10150000D2F1FF0340EAC250704740F400004FF0B0
:101510000003013A37E792F0000F00F0004C02BFE1
:10152000400010F4000F013AF9D040EA0C0093F0AB
:10153000000F01F0004C02BF490011F4000F013B05
:10154000F9D041EA0C0195E70CEAD15392EA0C0F6D
:1015500008D142027FF47DAF93EA0C0F7FF470AFA5
:10156000084676E793EA0C0F04D14B023FF44CAFE8
:1015700008466EE730F0004C18BF31F0004CCAD17D
:1015800030F000427FF45CAF31F000437FF43CAFB9
:101590005FE700BF42000ED2B2F1FE4F0BD34FF017
:1015A0009E03B3EB126209D44FEA002343F00043D9
:1015B00023FA02F070474FF00000704712F1610FFC
:1015C00001D1420202D14FF0FF3070474FF00000CE
:1015D000704700BF002310B504461A460D21094884
:1015E00003F0E4FF34B92246BDE810400D21054860
:1015F00004F0AAB8012CF6D0BDE810400F21024833
:1016000002F0EEBA0008024081630108002310B521
:1016100004461A460C21094803F0C8FF34B9224693
:10162000BDE810400C21054804F08EB8012CF6D01E
:10163000BDE810401C21024802F0D2BA000002406E
:10164000816301080146014805F082BE7205002051
:101650000146014805F07CBE7A050020014601489C
:1016600005F082BE720500200146014805F07CBEEF
:101670007A05002038B505460024A54200DC38BDB7
:1016800003F0A4FD0134F8E7012108B5084600F095
:101690009FFBBDE80840032004F098BE10B5074C3E
:1016A0000B21204604F044F8002320461A460B2163
:1016B00003F07CFFBDE8104003F07ABD000002405B
:1016C00008B504F00DFDBDE80840022201481146AE
:1016D00003F0AABF000002402DE9F0410220AAB0A9
:1016E00003F0CAFC03F02CFD0AF00EFA02220021DE
:1016F000B84803F099FF0122B648114603F094FF61
:1017000001220221B34803F08FFF02220321B148D6
:1017100003F08AFF00220421AE4803F085FF022275
:101720000821AC4803F080FF01220921A94803F0F9
:101730007BFF01220A21A74803F076FF02220B213A
:10174000A44803F071FF0020FFF760FF00220F2183
:10175000A04803F069FF012200219F4803F064FFC5
:10176000002202219C4803F05FFF002203219A48D7
:1017700003F05AFF02220621974803F055FF00228A
:101780000821954803F050FF00220921924803F0F8
:101790004BFF01220C21904803F046FF02220D214D
:1017A0008D4803F041FF02220E218B4803F03CFFDD
:1017B00002220F21884803F037FF0020FFF70AFFBD
:1017C00003F0E8FC0023ADF8183001238DF81A303F
:1017D00006980AF0F5F803F0DDFC0AF043F904F08E
:1017E000A3F97E4802F0C6F94FF4E13004F06CFC36
:1017F0007B4B1A680AB97B4A1A607B4B1A680AB994
:10180000784A1A60794805F0C5FC794805F0C2FCB1
:101810007849794805F0BEFC00F09AFA30B977486B
:1018200005F0B8FCDA21764802F0DAF903F0C0FCE2
:1018300007A800F061FA18B9E021714802F0D0F968
:101840009DF823009DF81E3004909DF822009DF81D
:101850001D2003909DF821009DF81C1002909DF81A
:101860002000684D01909DF81F00674E009067486A
:1018700005F090FC664B674A1693674B1A951593D3
:101880002AAB43F8442D93E80300644C8DE8030031
:101890001796189415AB0FCB10F0C2F8002800F083
:1018A0002A815F4805F076FC00224A48114603F081
:1018B000BBFE0F2302220021464803F055FD10F025
:1018C00049F8584BCDE920451D93574B574C1B9376
:1018D000574B1C93574BCDE91E361FAB93E80700BF
:1018E0008DE807001BAB0FCB0FF0AAFF0122207081
:1018F0000F21384803F098FE2378002B00F0008178
:101900004D4805F047FC0FF073FF4C4C4C4B6561A4
:10191000E3604C4BDFF8708123614B4BA3604B4B72
:1019200063604B4B23604B4BA3614B4BE36104F172
:1019300010030FCB8DE80F0094E80F0010F0BCF9F6
:1019400010F0DEF80146454805F024FC0AF0AEFC34
:1019500022AC60B9424BCDE925552493414BCDF8DB
:1019600088802393009594E80F000AF0A5FC3E4B75
:10197000002723933D4B012622933D4B09A9249335
:101980003C4B204625933C4B01ACCDE926353B4BE7
:1019900028933B4B29930423CDE909378DF829601F
:1019A00006F0FAF906F0ECF911F0DCFC10223946E9
:1019B00011A810F0D1FE334BCDE90B55CDE90D83C5
:1019C00003238DF84960109310AD0FCD0FC42B6821
:1019D00023605BE00000024000040240891600081A
:1019E000B0090020A15F0008B4090020C863010805
:1019F000D9630108A0860100E9630108FF630108BB
:101A00001064010895710008C55700084964010871
:101A1000771D0008751600085D1D0008FD570008B9
:101A20007964010899580008615800087005002081
:101A30007D580008511D00088A640108B850002034
:101A4000E55100086D510008151E0008551E0008DC
:101A5000411E00082596000865960008D26401081A
:101A60008D720008B9720008E9B90008B1B8000821
:101A7000C1B7000859B700086DB70008691600081B
:101A8000511600085D160008155B0008224B0093F4
:101A90000BAB0FCB0AF0F8FC03F092FA1F49044697
:101AA000FFF728FC13F012FE01461D4805F072FBFB
:101AB0004FF08041204613F0E1FD50B3194F174E0F
:101AC000194C03F07DFA3946054613F0EBFDD8B901
:101AD00031462846FFF70EFC13F0F8FD014620467C
:101AE00005F058FB4FF0FF3000F078F94FF47A70B2
:101AF00003F078FBE5E7F7210C4802F071F8E0E627
:101B00000B4805F047FB00E74FF0FF31002000F0E5
:101B10005FF92AB0BDE8F0814516000800007A445C
:101B2000E564010800002040F26401081064010827
:101B3000B864010808B1FFF7B1BD02220B210148CA
:101B400003F072BD0000024010B50AF087FD0020CE
:101B5000FFF7F0FF1A4C09F085FF01220C2119480C
:101B600003F062FD04F0F8F800F048F900F04AF9DB
:101B700003F06AFE144805F00DFB04F0AFF903F022
:101B800009FB204601220D2103F04EFD01222046D3
:101B90000E2103F049FD0021084604F09BF800F0F7
:101BA000D7F800F037F94FF4E13004F08DFA074828
:101BB00005F0F0FA09F07CFEBDE8104004F0CAB868
:101BC0000000024000040240BA630108E2900108EC
:101BD000054B5A69D20705D501225A61034B1B6890
:101BE00003B11847704700BF00040140840500207E
:101BF000044B5A69920703D502225A6107F060BA72
:101C0000704700BF0004014070477047044B5A6999
:101C1000D20603D510225A6107F06CBC704700BF92
:101C20000004014010B5134C6369180603D58023E6
:101C3000636107F009FC6369990603D5202363619A
:101C400007F046FC6369DA0506D54FF480736361DB
:101C5000094B1B6803B1984763699B0508D54FF48E
:101C600000736361054B1B6813B1BDE81040184752
:101C700010BD00BF0004014094050020980500201D
:101C800010B5194C63695B0504D54FF4806363613B
:101C900007F0EAFA6369180504D54FF4006363613D
:101CA00007F09CFB6369D90406D54FF48053636148
:101CB0000E4B1B6803B1984763699A0406D54FF42D
:101CC000005363610A4B1B6803B1984763691B04A7
:101CD00008D54FF400436361064B1B6813B1BDE8A0
:101CE0001040184710BD00BF0004014088050020C7
:101CF0008C0500209005002073B5134E054603F0B7
:101D000061FD3478B4B9F82302A800F8013DA0229F
:101D1000012103F0B3FD20B903F070FD204602B0AD
:101D200070BDA0220821094803F0B6FD0028F3D0B9
:101D30000123337003F062FD044A012413682B6011
:101D400053686B60EAE700BFA40500209C050020F3
:101D5000014803F067BD00BFA086010007B58DF8FC
:101D600004108DF805200221024601A803F078FD39
:101D700003B05DF804FB37B50023054602A81446FE
:101D800000F8011D137001212A4603F077FD20B1F0
:101D90002A460121204603F07FFD03B030BD00003C
:101DA00038B50A4C05460121204603F0C1FC00234A
:101DB00020461A46012103F0F9FB85F00102204676
:101DC000BDE83840012103F0BFBC00BF0000024065
:101DD000CB0701D5FFF7E4BF7047000008B5C30784
:101DE00009D50121044803F0B8FC00B10120BDE889
:101DF0000840FFF7D5BF08BD000002400020FFF7F4
:101E0000CFBF000001220321014803F00DBC00BF39
:101E100000040240012310B5084C1A462046032155
:101E200003F0C4FB2046032103F082FC032220467A
:101E3000BDE81040114603F099BB00BF000402400A
:101E4000021C18BF01220321014803F07DBC00BF22
:101E5000000402400321014803F07FBC000402405B
:101E6000084611B1012900D07047FFF7B3BB0846FF
:101E700011B1012900D07047FFF7C8BB014B0360C7
:101E8000704700BF18650108FFF762BF03F09ABCF6
:101E900003F0B4BC10B50446084611461A4603F0D8
:101EA000DFFC08B90123237110BD10B504460846B4
:101EB00011461A4603F0E2FC08B90123237110BD54
:101EC00010B50446084611461A4603F0E5FC08B969
:101ED0000123237110BD03F01DBE084611461A46AA
:101EE0009DF8003003F0B6BE03F07CBE03F060BE88
:101EF000084603F0F1BC7047704700007FB500F161
:101F00000806054630460C4610F08CFAF8B92E4803
:101F100005F040F9A27C617C2C4805F03BF968682B
:101F2000002103681B6898476868002103685B68A4
:101F30009847022000F06CF8022000F087F86368F0
:101F4000012B0FD0022B1AD0DBB94E250BE06421F8
:101F5000304610F053FA0028DCD141211C4801F032
:101F60003FFED7E74525A368A3B1012B0ED1092673
:101F7000E368032B20D8DFE803F025230F1D4F254E
:101F8000F1E71721124801F02BFEDEE7232110486C
:101F900001F026FE0826EBE70F23A27C29460292D9
:101FA000627C20680192227C0092324604F0C6F8DE
:101FB00004B070BD0223F0E73321054801F010FEA4
:101FC0000123EAE70523E8E75C650108B565010838
:101FD0007565010810B50446FFF772FB04F10800AF
:101FE000BDE8104010F021BA084604F06FB9084669
:101FF00004F09CB910B50446044BC0E9003101213E
:10200000083010F01DFA204610BD00BFDC65010845
:10201000042817D8DFE800F00309100E120000238F
:1020200003211A46084803F0C1BA002203210648DA
:1020300003F0FABA0222F9E70122F7E70321024886
:1020400003F018BB704700BF00000240042817D8F7
:10205000DFE800F00309100E1200002302211A46E7
:10206000084803F0A3BA00220221064803F0DCBAB4
:102070000222F9E70122F7E70221024803F0FABA47
:10208000704700BF0000024010B50446024B0360D9
:1020900010F09EF9204610BDFC65010810B50446FD
:1020A000054B283040F8283C044B40F8083CFFF72B
:1020B000EBFF204610BD00BF1C690108DC6501086C
:1020C00010B50446FFF7E0FF204608210FF016FB8D
:1020D000204610BD10B50446FFF7E0FF20463C2126
:1020E0000FF00CFB204610BD38B50A4C0D462046BB
:1020F000012103F01DFB002320461A46012103F0B5
:1021000055FA85F001022046BDE83840012103F070
:102110001BBB00BF00000240084603F063B800008C
:1021200010B5074C0B21204603F002FB002320468C
:102130001A460B2103F03AFABDE8104003F038B814
:102140000000024070B5044610F0F2F82346002566
:102150000D4A04F11C0643F8112B3046C4F8115007
:102160005D60FFF78BFE314604F12000FFF742FF70
:10217000064B84F834502363054B0648A36305F0EF
:1021800009F8204670BD00BF1C69010828650108D8
:10219000486501080369010810B5084C2368DB078E
:1021A00009D40748FFF7CEFF0123064A0649044831
:1021B000236010F063F9024810BD00BFA80500209D
:1021C000C8050020A84F00209D20000808B50B215D
:1021D000054803F0C7FA28B1BDE808400B210248C2
:1021E00003F0D4BA08BD00BF0000024009B1FFF7F8
:1021F00097BF02220B21014803F016BA00000240EB
:1022000038B50546FFF7E2FF044628B1002128460D
:10221000FFF7ECFF02F0CCFF02F0D2FE05460CB156
:10222000FFF77EFF284638BDF8B50C460646224922
:10223000204613F041FA20B90021204613F01EFA7F
:1022400068B11E492046FFF755F813F03FFA0146E2
:102250001B4804F09FFF98211A4801F0C1FC30464A
:10226000FFF7B4FF054618B1174804F093FF1FE0CD
:102270003046FFF7C5FF114906462046FFF73AF8FA
:1022800013F024FA0D4907463046FFF733F813F0F0
:102290001DFA3A4601460D4804F07CFF31462046BF
:1022A00013F00AFA30B10A4804F074FFFFF738FF60
:1022B0002846F8BD0748D8E73333534000007A4436
:1022C0000466010833660108736601089266010816
:1022D000C6660108DF660108113070472DE9F0413C
:1022E000002600F11104D2B0C0F8116018496660F0
:1022F0000546FFF799FF3146074605F11C00FFF739
:10230000B6FD01A80FF064FC9DF80430012B17D135
:10231000DDF805300F48C5F81130DDF80930DFF879
:102320003C80636004F036FF05F1190614F8011BC8
:10233000404604F02FFFB442F8D1074804F02AFFCA
:1023400039462846FFF752FF52B0BDE8F08100BF82
:1023500000004040F7660108C66301081E670108D7
:1023600010B5044686B0354804F014FF20461C34EE
:10237000FFF7B4FF00212046FFF772FD0120FFF7B1
:1023800047FE00212046FFF772FD0120FFF75EFEA9
:102390002B4804F0FFFE4FF4FA7010F089F9044660
:1023A000002844D1274804F0F5FE274804F0F2FE47
:1023B000264804F0EFFE264804F0ECFE254804F021
:1023C000E9FE254804F0E6FE244804F0E3FE244834
:1023D00004F0E0FE234804F0DDFE234A23492448AC
:1023E00004F0D8FE2349244804F0D4FE234804F026
:1023F000D1FE234B234A1B6823490093234B1268C9
:102400001B68234811F04AF82149224804F0C2FE13
:1024100003A803F021FB03A804F01CFE01461E489C
:1024200004F0B8FE094804F0B5FE06B010BD1B4824
:1024300004F0B0FE204610F043F9B6E72367010828
:102440003567010863670108C5630108A1670108D2
:10245000D2670108E16701080368010827680108DD
:102460004B680108C66301086E68010874680108BA
:1024700092680108A2680108A9680108B468010807
:102480006400F81F5000F81FD46801085400F81FBA
:10249000AC050020E6680108F168010897670108AB
:1024A000436830B55568002B18BF6124D1E900316D
:1024B00008BF7024002D14BF6125702500681268C4
:1024C00085B0CDE90152009102462146024804F050
:1024D00061FE05B030BD00BF3469010810B5044687
:1024E000C06908B104F0D2FE206908B104F0CEFE44
:1024F000606808B104F0CAFE204610BD10B504465D
:10250000006807F0B5FE204610BD0000FE2307B5A9
:1025100002A901F8043D054B1868002300681A461B
:1025200007F028FC03B05DF804FB00BF1006002094
:10253000C121014801F054BB52690108D0B51F46C2
:102540007423C0E900310023044683600820164646
:102550000FF0C8F8C0E90067A0602046D0BD0000B9
:10256000036837B5632B05460C4601D0FFF7E0FF43
:102570000023A96802AA42F8043D0831204604F06D
:10258000F9FB019A3AB12146044804F003FE2E21DA
:10259000034801F025FB03B030BD00BF946901087A
:1025A000C1690108F8B5632300260446C0E900317B
:1025B0008660282017460FF095F84FF00043002260
:1025C0000546C0E9002331461A22083010F0C4F84D
:1025D0002046A5603946FFF7C3FF2046F8BD00003E
:1025E0000B6870B506460C461BB95321164801F01E
:1025F000F7FA63681BB95421134801F0F1FAA36894
:102600001BB95521104801F0EBFAE3681BB95621BC
:102610000D4801F0E5FA23691BB957210A4801F07A
:10262000DFFA63691BB95821074801F0D9FA0FCCCA
:1026300006F12C050FC5012394E8030085E803008B
:1026400086F8283070BD00BFC16901082DE9F84344
:10265000D0E90173884600254FF00C09DB1B0A4EB8
:102660009B105E43ECB2B4420BD209FB04724146AC
:10267000506810F033FF01350028F3D12046BDE843
:10268000F8834FF0FF30FAE7ABAAAAAA2DE9F04190
:10269000D0E9047588460026ED1BED10F4B2AC427B
:1026A0000AD2414657F8340010F018FF01360028CE
:1026B000F4D12046BDE8F0814FF0FF30FAE700008A
:1026C0002DE9F0410E4649680446FFF7BFFFC0B24E
:1026D000FF2807D071682B4804F05CFD72212A485E
:1026E00001F07EFAD4E90123284F9B1A9B107B430B
:1026F0007E2B03D97521244801F072FAD4E9011226
:102700000C25E068531A9B10121A7B4392107A43EF
:102710000133934205FB03F80ED84144A160D4E98C
:10272000013496E80700E31A04E9070017489B10F4
:1027300058430138BDE8F081404604F0BDFD054630
:1027400018B96921124801F04BFAD4E901C30027F6
:10275000A3EB0C039A100D4B5343002B09DD05EB43
:10276000070E0CEB070207CA013B8EE807000C3787
:10277000F3E7604604F08AFD65604544C4E902550C
:10278000CDE700BF736E0108C1690108ABAAAAAA10
:10279000936E01081FB56E23CDE90131002301A915
:1027A0000393FFF78DFF05B05DF804FB002170B5C2
:1027B00018220446C0E90011C0E90211C0E9041161
:1027C000C0E90611C0E9081180F828102C300FF07C
:1027D000C3FFFF2300204FF000411E4E84F8443019
:1027E0003268C4E9120112F00102C4E9140184F84C
:1027F000583084F859300DD10121174D08462A6010
:1028000007F0DEF901232860144A15492846336091
:102810000FF034FE134B1A680AB90F4A1A601249B6
:102820002046FFF7B7FF114B114918702046FFF7FC
:10283000B1FF104B104918702046FFF7ABFF0F4B4C
:102840000F4918702046FFF7A5FF0E4B1870204661
:1028500070BD00BF0C06002080060020A84F00209D
:10286000FD24000810060020896F010817060020CB
:10287000916F010815060020996F010814060020C9
:102880009E6F01081606002010B5084C2368DB0770
:1028900009D40748FFF78AFF0123064A064904487E
:1028A00023600FF0EBFD024810BD00BF08060020BA
:1028B00020060020A84F0020DD2400082DE9F0416B
:1028C0000E4609680446FFF7E1FEC0B2FF2807D0B4
:1028D00031682B4804F05EFC7D212A4801F080F924
:1028E000D4E904239B1AB3F57E7F03D380212548C6
:1028F00001F076F9D4E90452A169531BDB100133CE
:10290000521AB3EBE20F4FEAC30711D83D44656199
:10291000D4E904239B1ADB1003F10051013902EBC7
:10292000C10296E8030082E80300581EBDE8F0816A
:10293000384604F0C1FC054618B96921124801F077
:102940004FF9D4E904E34FF0000CA3EB0E03DA10C7
:10295000A2EB0C03002B0BDD4FEACC0305EB0308C5
:10296000734493E803000CF1010C88E80300EFE7DF
:10297000704604F08BFC25613D44A561C7E700BFAC
:10298000CB6E0108C1690108936E010838B5D0E922
:1029900001239B1A074A9B105343CDB29D42044624
:1029A00003D39C21044801F01BF90C20636800FB51
:1029B000053038BDABAAAAAAC16901080F4A38B5CB
:1029C0001368054613F00103CCB205D10C490D483C
:1029D000C1E9000301231360FF2C0DD0D5E90423C6
:1029E0009B1AB4EBE30F03D3A821074801F0F8F8D2
:1029F000286900EBC40038BD0148FCE7040600204C
:102A000018060020416A0108C169010810B5D0E923
:102A10000730C9B2D2B2834209D01C788C4204D1AB
:102A20005C78944201D1987810BD0333F3E74FF0FE
:102A3000FF30F9E72DE9F0410A780D46D0E904139B
:102A40005B1AB2EBE30F044603D389214A4801F035
:102A5000C7F8D4E901239B1A484A9B10534369786D
:102A6000994203D38A21444801F0BAF8D4E9041307
:102A7000AA785B1AB2EBE30F03D38B213E4801F037
:102A8000AFF86A7829782046FFF7C0FFC3B2FF2B62
:102A900006462CD03A4804F07DFB29782046FFF703
:102AA0008DFF697807462046FFF770FF3146804664
:102AB0002046FFF783FF414602463846FFF7F0FC09
:102AC00029782046FFF77AFF697806462046FFF707
:102AD0005DFFA97807462046FFF770FF394602469A
:102AE0003046FFF7DDFC9221234801F079F8D4E964
:102AF0000723224F9B1A7B437E2B03D995211E4827
:102B000001F06EF8D4E90762616A931B7B43521AA5
:102B100057430133BB4203EB43080AD846442662BD
:102B20002A88236A23F8032CAA7803F8012CBDE82D
:102B3000F081404604F0C0FB064618B969211148EF
:102B400001F04EF8D4E90702131A0C4A5A43002345
:102B5000002A0ADDC118B1F800C0F71826F803C032
:102B60008978013AB9700333F2E704F08FFBE6612C
:102B700046446662D3E700BFC1690108ABAAAAAAAE
:102B8000266A0108936E010813B5FF24084A02ABB8
:102B9000106803F8044D0A460068194607F08EF9DC
:102BA000012814BF20469DF8040002B010BD00BFEC
:102BB00010060020F8B51F460B680C46632B16461E
:102BC0004FF000004FF000410DD0742B2DD1A368C1
:102BD000D3E900458D4208BF844201D0A4187D414D
:102BE00020462946F8BDA468D4E900238B4208BFDB
:102BF000824206D00E4804F0CDFACB210D4800F0F9
:102C0000EFFF3B4604F10800324604F073F9002858
:102C100071F1000304460D46E2DA074804F0BAFAFF
:102C2000D021044800F0DCFFDAE704460D46D7E780
:102C3000476B0108C1690108796B01082DE9F0476C
:102C40000F460646FFF7BAFE00244368DFF860909F
:102C5000002B026814BF612170211348FFB204F0F9
:102C600099FAD6E90758454516D02B78BB4211D1C1
:102C700069783046FFF78AFE016869290AD1D0E9F0
:102C8000012A484604F086FADAF8003003B1984782
:102C90000134E4B20335E6E72146044804F07AFA49
:102CA0002046BDE8F08700BF9F6B0108E86B010874
:102CB000C66B01082DE9F34788460746FFF77EFEFD
:102CC000002543680268002B14BF612170211B4856
:102CD00004F060FAFC693E6ADFF86890033403365A
:102CE0005FFA88F8A64220D0234633F8032D9B785C
:102CF000ADF804208DF8063014F8033C984512D145
:102D00009DF805103846FFF741FE016869290AD190
:102D1000D0E9012A484604F03DFADAF8043003B15C
:102D200098470135EDB20334DCE72946044804F046
:102D300031FA284602B0BDE8F08700BF066C0108F2
:102D4000536C01082F6C010890F8283073B50446C5
:102D50000D46164623B940F209110D4800F040FF18
:102D60000C49CDE9006423462A460B4807F060FB76
:102D7000012801460AD0094804F00CFA40F20F116C
:102D8000034802B0BDE8704000F02ABF02B070BD39
:102D9000C1690108416E0108153300084C6E010835
:102DA0002DE9F74F04462C4804F0F4F90027DFF82A
:102DB000BC80D4E90431C91AFEB2C910B1423BD972
:102DC0004FF00C0A03EBC60252682448002A08BFE1
:102DD000702153F8362018BF612104F0DBF994F814
:102DE0004430DFF88CB0B3420CBF40461C4804F0BE
:102DF000D1F9D4E90759A9451CD02B78B34217D192
:102E00006B7820690AFB03F395F802C0616800EB58
:102E1000CC0ECA18C958DEF804305268002B50F89E
:102E20003C30584600930CBF7023612304F0B2F984
:102E30000335E0E70137BCE7D4E907239B1AA26812
:102E400064680848121B921043434243064803B08B
:102E5000BDE8F04F04F09EB9EB6E0108FA6E010870
:102E6000C6630108ABAAAAAA356F01080A6F010858
:102E7000166F010800232DE9F047C0E904330E4620
:102E80001946D6E907574FF000430446C0E902133C
:102E9000C0E90013FF208846994620745FFA82FA41
:102EA000BD4220D02B7853451BD169783046FFF7BF
:102EB0006DFDDDE9082301463046FFF77BFE4945FD
:102EC00008BF40450DD0D4E900234B4508BF42451B
:102ED00003D0904271EB030303DA6B78C4E900017D
:102EE00023740335DCE72046BDE8F087F8B50D46CE
:102EF0000D4B896806464B434FF47A71B3FBF1F1F1
:102F0000FFF742FEF36A0446C7B29847C6E91401C8
:102F100004F0CAF80146054804F03CF9FF2F0CBF45
:102F2000287C2046F8BD00BF40420F00036A01081C
:102F30007FB504460D46036C16489847A36B984727
:102F4000D5E9002301A804F047F89DF805209DF875
:102F500006109DF807009DF80430666BB047E36BE0
:102F60009847236B9847A36B9847E36A9847C4E94F
:102F7000140104F099F80146074804F00BF9002108
:102F80002046FFF701FEC0B2FE2808BF287C04B02F
:102F900070BD00BF0D250008696F0108D1E900234D
:102FA000B3F1004F08BF002A2DE9F04B05460C464F
:102FB00016D03A4E3A4FDFF81081D4E90223012AA5
:102FC00073F1000110DA134302D0364804F0E2F83E
:102FD000354804F0DFF894F810904846BDE8F08BCF
:102FE000BDE8F04BFFF7A4BF052A73F100031ADA1E
:102FF000384604F0CFF821462846FFF777FF5FFAFE
:1030000080F9B9F1FF0F16D1284804F0C3F84FF446
:10301000D471274800F0E4FD264B274A40F2A9115D
:1030200023480FF031FA304604F0B4F82146284620
:10303000FFF77EFFE3E7237C4B452BD1D5E914BC9A
:10304000D4E9002393457CEB030114DA404604F0F5
:10305000A1F8D5E91423D4E90001801A61EB03013A
:103060008C468346C4E902BC04F02AF801461348A2
:1030700004F090F8A1E7BBEB02006CEB030102281F
:1030800071F10003A9DB04F01BF801460C4804F0C1
:1030900081F8A2E70B4804F07DF89EE7936D0108E4
:1030A000756D0108386D01085D6D0108AD6D010891
:1030B000C1690108D36D0108CB6F0108F86D0108E3
:1030C0000B6E01082A6E0108D96D0108F0B504469F
:1030D00089B00D46FFF772FCE36A074698472A4617
:1030E000C4E91201CDE90001214602A8FFF7C2FEA2
:1030F00029462046FFF7A2FD9DF818300646FF2B13
:103100000ED168B97B682948002B14BF612170215A
:103110003A6804F03FF840F22911254800F060FDBC
:10312000D4E9120103F0C0FF0146224804F032F84E
:103130003146214804F02EF89DF81810FF2913D1CC
:103140001E4804F027F800224FF00043CDE9042385
:1031500002A92046FFF722FF064629462046FFF730
:10316000A9FD304609B0F0BD2046FFF70FFCD0E9BD
:103170000067DDE9020103F097FF3A460346314656
:103180000F4804F007F8D4E91223DDE90201801AA0
:1031900061EB03010F460646CDE9046703F090FF9B
:1031A0000146084803F0F6FFD2E700BF7F6A010836
:1031B000C1690108B26A0108D16A0108EC6A010814
:1031C000056B0108296B010870B504460D46FFF731
:1031D000F5FB436833B194F8591094F85800BDE8F2
:1031E0007040184729462046BDE87040FFF76EBF83
:1031F0002DE9F74F04463C4803F0CCFF3B4803F071
:10320000C9FF3B4803F0C6FF384803F0C3FF94F8FA
:103210004430FF2B04D14FF4AF71364800F0E0FC8E
:1032200094F844102046FFF7C9FB43680268002B5E
:1032300014BF61217021304803F0ACFFDFF8B4B057
:1032400094F8445029462046FFF7B8FB29468046AB
:103250002046FFF7B9FFC3B2FF2B06460ED1274821
:1032600003F098FF4FF4B471224800F0B9FC244BEE
:10327000244A40F269111F480FF006F90146204622
:10328000FFF784FB3246814629462046FFF7BEFB06
:10329000C7B2FF2F824610D11B4803F07BFF514677
:1032A0002046FFF78BFB494602464046FFF7F8F8F9
:1032B00040F27111584600F093FC51462046FFF74A
:1032C0007DFB0190114803F065FF114803F062FF98
:1032D000019A49464046FFF7E3F884F8585084F8CD
:1032E00059603D46AEE700BFC6630108736C010834
:1032F000926C0108C1690108B16C0108CF6C01082A
:10330000D36D0108A66F0108F26C0108126D010867
:10331000286D010808B5FFF7B7FAFFF769FF00004D
:103320002DE9F8431F461646FFF730FBB7F1004F73
:1033300008BF002ED0E9005884681AD0742D01D03F
:10334000FFF7F6F8D4E9000103F0BAFE39468146EA
:10335000304603F0B5FE4A46034641460A4803F0AC
:1033600019FF742D01D0FFF7E3F8C4E90067BDE849
:10337000F883742D01D0FFF7DBF8D4E9000103F0E6
:103380009FFE024B0246E8E74F6A0108736A010894
:10339000FF23044A1370044A1370044A1370044A4A
:1033A0001370704717060020150600201406002031
:1033B000160600201FB5184BC0B21B7883420AD1F5
:1033C000164BC9B21B685B78994222D1144B18780E
:1033D00005B05DF804FB09F097F90023ADF80C3057
:1033E000104B5A7812B101228DF80C201B7813B1C2
:1033F00001238DF80D300C4B0C481A780C4B1978C2
:10340000002300930068039B09F0CCFA08B1094B34
:10341000DDE7094BDBE700BF700700201007002045
:1034200017060020740800207C0800207008002087
:103430007808002014060020150600202DE9FF4121
:1034400023490446FFF7A6F9224B2349187020466A
:10345000FFF7A0F9DFF8A4800A2288F80000002313
:103460001E4901A8FFF76AF801A92046FFF728F9CD
:103470001B4B1C4F01931C4B387001A92046029333
:10348000FFF71CFA194B1A4D01930023287001A96C
:1034900020460293FFF712FA0646034698F80020EA
:1034A00029782046FDF720F82B783A7831462046D7
:1034B000FDF71AF829780F4A0B4612782046FDF7D7
:1034C00013F801220C4B1A7004B0BDE8F08100BF64
:1034D000767101087E0800207F710108887101085B
:1034E0008F7101088C0600203D390008A271010887
:1034F0007007002016060020880800207D080020A4
:10350000354B2DE9F7431A68344D12F0010F01BF16
:10351000FF222A7001221A602B780446FF2B57D114
:103520002F4B1B780BB9FFF789FF2E4B6946009391
:103530002D4B20460193FFF7C1F92C4B28700093C7
:103540002B4B694620460193FFF7B8F90027294E17
:10355000294B30706946204600930197FFF7AEF97A
:10356000264B814669462046CDE90037FFF7A6F98C
:103570000746234A3378127829782046FCF7B4FFAF
:10358000204A2B78127831782046FCF7ADFF1E4A8E
:10359000DFF880804B46127831782046FCF7A4FF94
:1035A000337898F8002049462046FCF79DFF174ADB
:1035B0003B46127831782046FCF796FF337898F82E
:1035C000002039462046FCF78FFF2A78104B1A70EE
:1035D000287803B0BDE8F083840600208908002025
:1035E00088080020B8710108413A0008C17101083B
:1035F000E53600087F080020CA710108D77101086C
:103600007E080020170600207D08002015060020F7
:10361000800800208C060020244B2DE9F3411B7804
:1036200005460E460BB9FFF709FF214B69462846B0
:1036300001930096FFF742F9044630460FF060FF11
:10364000804605300EF058F8074631460FF050FF1F
:10365000184907EB08000FF04BFF39462846FFF7E3
:1036600099F80646144F154A3B78127821462846A9
:10367000FCF73AFF2346324639782846FCF734FFF8
:1036800008200EF02FF800230D4A436013680470E1
:1036900046702BB91060204602B0BDE8F081134699
:1036A0005A68002AFBD15860F5E700BF880800205F
:1036B000B5330008D49E01087007002014060020CE
:1036C0008806002070B50D460446FFF7DDF8044972
:1036D00022462B46BDE870400978FFF721BE00BFA7
:1036E0008C06002073B5384C266876B904200DF09E
:1036F000F9FF3246054606600421012006F060FA13
:1037000028603248256009F01FF8314B314D1968A7
:1037100031480131196003F03DFD08F0F5FF2B78C9
:103720001BB901232B7009F025F8002302A941F8E9
:10373000043D2368294A186806F0C0FB012806D01A
:10374000274803F027FDDE21264800F049FA019EB4
:10375000731C17D1244803F01DFD002350213C2089
:103760002B7003F05FFE0446C51702462B461F4828
:1037700003F010FD20462946FFF7A4FF1C4B1878E4
:1037800002B070BD4EB131461A4803F003FD0198F6
:103790000021FFF797FF184BF1E7184803F0FAFCF8
:1037A00008F05CFF23686BB1304608F0CDFF256858
:1037B00035B1286806F05CFD042128460DF09EFF17
:1037C000002323600E4BDAE708070020F5390008D4
:1037D00084080020820800201A700108A0860100D9
:1037E0002D7001084770010893700108A47001084A
:1037F00015060020BB7001087D080020D07001086C
:1038000017060020044B1870044B1A600022044B6A
:103810001960044B1A8070477C080020780800204B
:1038200070080020740800202DE9F04342F2107067
:1038300085B008F08FFF4FF000090446DFF8F880EC
:10384000354FFF22002140460EF086FF334D78228F
:10385000002138460EF080FF314885F8009003F0D3
:1038600099FC002C54D02146782238460EF050FFA7
:10387000C7F87090216F89B12A4E582230460EF059
:1038800047FF3E67236FC6F84890996C31B11A7FA5
:1038900022B140460EF03CFFC6F8488001232B7051
:1038A0002578022D30D160680021FFF70BFF236FD0
:1038B000F3B1D3E9142313431AD01B4B1E6806F04F
:1038C000D9FF01461948B047236FD3E9140103F02B
:1038D000EBFB236F01461A6D154803F05BFC236F69
:1038E00001A8D3E9142303F077FB01A802F0A4F8A0
:1038F000104803F04FFC204609F0B8FB032D08D117
:10390000284605B0BDE8F083032DD0D10020CBE7D9
:10391000012508F0A3FEF3E7900600200C07002025
:10392000E07001081807002088000020FE700108E0
:103930000B7101083C7101087107002008B5194B93
:10394000C9B21B78994209D1174B184A1B68C0B2FB
:1039500013601BB1197881420DD1136008F0B2FEDB
:1039600008B108F0D1FEFFF75FFF032811D8DFE8A8
:1039700000F007040E0B5B68EBE70D4803F00AFC50
:103980000A4B1B68587808BD0A4B1878FBE70A4BAE
:10399000FBE70A4840F2B51100F022F94FF0FF3082
:1039A000F1E700BF14060020880600201007002061
:1039B0005C710108160600207D0800204770010890
:1039C00010B50446FFF79CFD03492046FFF724FE8F
:1039D000024B187010BD00BFAF71010881080020B4
:1039E00008B5002300681A4606F0C4F9431E584281
:1039F000584108BD07B50B78012B0ED004D3022B1C
:103A00000FD003B05DF804FB002302A941F8043D88
:103A1000054B1868FFF7E4FFF3E702A94FF0FF3307
:103A2000F4E70431F4E700BF0807002010B50446AE
:103A3000006810B101210DF061FE204610BD0000AC
:103A400030B5304BC0B21B788BB0834201D12E4BC6
:103A500040E00DF01FF82D4904460CF0BDFE054670
:103A600000283AD02A4A214601A80CF0BEFE294A75
:103A7000214604A80CF0B9FE274A214607A80CF0FD
:103A8000B4FE079A0499019809F08CF807A8FFF78B
:103A9000CDFF04A8FFF7CAFF01A8FFF7C7FF1F4922
:103AA00020460CF0B3FE40B20AF082FC09F012F896
:103AB0001B4920460CF0AAFEC0B20AF047FC08F0F1
:103AC000FFFF184920460CF087FE09F053F8002D3F
:103AD000BDD0154B18780BB030BD214601A8134A54
:103AE0000CF083FE214604A8114A0CF07EFE21460C
:103AF00007A8104A0CF079FE049A0799019809F07A
:103B00003FF8C3E77F080020170600201A5E01086F
:103B1000265E01081F5E01082D5E01089F5E0108F8
:103B2000735E0108238D01087E080020445E0108B1
:103B30003C5E0108345E0108FF23074A1370074A00
:103B40001370074A1370074A1370074A1370074A25
:103B50001370074A13707047700700207F08002019
:103B60007E0800207D0800208C06002080080020B0
:103B700081080020014B1860704700BF1409002025
:103B800073B5124C064623780D46114A1BB91378BB
:103B90000BB172B6FEE70123002113700D486422B9
:103BA0000EF0DAFD2B4600960B4A642109480FF00F
:103BB00041FC0A4B1B6803B198470125054E30466E
:103BC00003F02CFB72B62570F9E700BFF408002063
:103BD0008A0800208C080020F871010814090020D0
:103BE00073B5134C064623780D46124A1BB9137859
:103BF0000BB172B6FEE70123002113700E48642258
:103C00000EF0AAFD2B4600960C4A64210A480FF0DC
:103C100011FC0B4B1B6803B19847074803F0FEFAF1
:103C2000084803F0FBFA72B601232370FEE700BFD9
:103C3000F50800208B0800208C0800202072010865
:103C4000140900202F7201080368DFF888C080B5CE
:103C5000CCF80030164F4368164E3B608368164D13
:103C60003360C36815492B600369154A0B604369CB
:103C7000144C13608369C0692360134B1860DCF82F
:103C80000000386830682868096810481268002108
:103C9000226864221B680EF05FFD23680C4A6421D1
:103CA0000A480FF0C7FB094803F0B8FAFEE700BF67
:103CB000040900200C090020100900200809002038
:103CC000F0080020F8080020FC0800208C080020E4
:103CD000E571010800090020074B1B6803B19847F4
:103CE0001EF0040F0CBFEFF30880EFF30980816929
:103CF000004A1047493C0008140900202DE9FF4103
:103D00009846244B07461B780C468DF807201BB9B4
:103D10002D212148FFF764FF204B1B7823B9002495
:103D2000204604B0BDE8F0811D4E1E4D33782BB106
:103D3000EB6898470028F2D0002333702B6998472E
:103D40000028ECD0BCB16B683A4601210DF10700A8
:103D50009847044610B90123337009E0AB683A462E
:103D6000012103A8984704460028F4D09DF80C4090
:103D70006B699847D4E79DF807308DF80D808DF872
:103D80000C303A462B68022103A898470028EFD14F
:103D9000E1E700BF190900204B7201083409002037
:103DA000180900201C0900200323F7B58DF8033003
:103DB000164B07461B781BB95E211548FFF710FF0D
:103DC000144D2B6998470446C0B16B683A460121EF
:103DD0000DF103009847104E044620B96B699847CF
:103DE000012333700AE0AB683A46012101A89847E5
:103DF000012704466B6920B998473770204603B005
:103E0000F0BD9847054B1F700023EAE71909002011
:103E10004B7201081C0900201809002034090020F9
:103E2000034B1B780BB1FFF7BFBF1846704700BFAD
:103E300034090020F8B50023194A1A4E1370C768D8
:103E4000194A337013700FB90020F8BD8368002B36
:103E5000FAD00368002BF7D04368002BF4D0036935
:103E6000002BF1D04369002BEED004460F4D0FCC50
:103E70000FC594E8030085E80300B8470028E3D0A5
:103E80000124E0203470FFF78FFFE220FFF78CFF62
:103E9000E420FFF789FFE620FFF786FF2046D4E7FE
:103EA0003409002019090020180900201C090020ED
:103EB00008B5032200230121FFF720FFC043C0B251
:103EC00008BDCB430322DBB20021FFF717BF0B462F
:103ED00001220021FFF712BF38B505460C46FFF757
:103EE000E7FF40EA0401C9B22846BDE83840FFF7C1
:103EF000E8BF0000002103E00A4B5B584350043147
:103F000009480A4B42189A42F6D3094A02E00023B4
:103F100042F8043B074B9A42F9D300F00FF8FCF744
:103F2000F9FD7047ECAE010800000020B803002046
:103F3000B8030020DC500020FEE70000314B82B0C7
:103F40001A6842F480721A6099682F4A0A409A608F
:103F50001A6822F0885222F001121A601A6822F4BC
:103F600080221A609A6822F47D029A600022DA6048
:103F700001921B6813F4007318BF01230193019B86
:103F8000012B37D14FF48051204B1A68A3F5806381
:103F900022F00102C3F80024D3F8002422F0020228
:103FA000C3F80024D3F8002422F00402C3F800244C
:103FB0005A6A42F080525A62154A11605168C90625
:103FC000FCD49A689A609A689A609A689A605A686B
:103FD00022F460425A605A6842F440425A609A6839
:103FE00022F003029A609A689A60064A936813F076
:103FF0000C0FFBD14FF00062064B9A60064ADA6064
:1040000002B07047003802400CC0FF88003C0240FC
:104010000070004000ED00E00003FA0530B5012417
:1040200003780A4D03F01F029440C278590952B137
:10403000074A2B44D26842781201D2B283F8002397
:1040400045F8214030BD2031FAE700BF00E100E033
:1040500000ED00E008B5084B98420BD101214FF468
:10406000007000F047FBBDE8084000214FF40070ED
:1040700000F040BB08BD00BF0024014043680A793E
:1040800023F0407323F4807343EA02230A6810B5D7
:1040900013434360D1E9032313438A6884681343BD
:1040A000084A224013434A7943EA420383600A7D67
:1040B000036B013A23F0F873D2B243EA025303636D
:1040C00010BD00BFFDF7FFC000234FF0407203603A
:1040D000037143718360C0E90323012303757047B3
:1040E000836819B143F001038360704723F0010333
:1040F000FAE70000044B5A6818B142F400025A6013
:10410000704722F40002FAE7002701401D2970B52C
:104110001BD90725A1F11E06C46D06EB4606B54066
:1041200024EA050403FA06F62643C665062A38D8AB
:104130001F24013A036C02EB8202944023EA040339
:1041400001FA02F21A43026470BD13290DD9072641
:10415000A1F11405C46805EB4505AE4024EA060448
:1041600003FA05F52543C560E0E709290DD90726BF
:10417000A1F10A04056904EB4404A64025EA0605FA
:1041800003FA04F42C430461D0E70726446901EBE9
:104190004105AE4024EA060403FA05F626434661CB
:1041A000C4E70C2A0CD81F24073AC36B02EB820227
:1041B000944023EA040301FA02F21A43C263C3E7FC
:1041C000122A0CD81F240D3A836B02EB8202944012
:1041D00023EA040301FA02F21A438263B4E7182ABD
:1041E0000CD81F24133A436B02EB8202944023EA5B
:1041F000040301FA02F21A434263A5E71F24193AA5
:10420000036B02EB8202944023EA040391401943BA
:10421000016399E7836843F0804383607047806D52
:1042200080B270470368194214BF01200020704714
:10423000C943016070470000044B1A6818B142F08E
:1042400002021A60704722F00202FAE7003C0240C4
:10425000044B1A6818B142F004021A60704722F049
:104260000402FAE7003C0240044B1A6818B142F01D
:1042700008021A60704722F00802FAE7003C024088
:10428000044B5A68D20741BF034ADA60034ADA6036
:10429000704700BF003C0240EFCDAB89050403022C
:1042A000024A536843F0010353607047003C0240E8
:1042B000014B9861704700BF003C0240084B9A696F
:1042C000D10709D49A69D20508D49B6913F4F05F29
:1042D00014BF03200420704701207047022070475C
:1042E000003C0240042313B504468DF80730FFF765
:1042F000E5FF8DF807009DF80730012B0AD11CB9A6
:1043000005238DF8073007E0FFF7D8FF013C8DF853
:104310000700F0E7002CF3D09DF8070002B010BDB5
:1043200010B504464FF40040FFF7DCFF042804BF3B
:104330000023236010BD000038B504464FF4004050
:104340000D46FFF7CFFF04280BD1064A4FF400407B
:10435000536823F4807353602560BDE83840FFF74D
:10436000C1BF38BD003C024038B504464FF40040A0
:104370000D46FFF7B7FF04281BD135B125704FF468
:104380000040BDE83840FFF7ADBFFF2324F0030530
:1043900004F003042968E40003FA04F421EA0404A5
:1043A0002846FFF7BDFF21462846BDE83840FFF705
:1043B000C3BF38BD2DE9F0430022012703250E6855
:1043C00007FA02F333EA060431D14FEA420C05FA48
:1043D0000CF4E44391F804E0D0F800900EFA0CF8E5
:1043E00004EA09090EF1FF3E48EA0908BEF1010F8F
:1043F000C0F8008011D8D0F808E004EA0E0E4C791D
:1044000004FA0CF444EA0E048460848824EA030469
:104410008B7993409BB223438380C36805FA0CF4E5
:1044200023EA0404CB7903FA0CF32343C36001327B
:10443000102AC5D1BDE8F08310B50F2401F00703A1
:10444000C90800EB8100016A9B009C4021EA04013D
:104450000162016A9A400A43026210BD7FB50446B8
:10446000868868460D4600F0D7F8029A2B4926F058
:104470003F06B2FBF1F13604360C88B20643A68043
:104480002388274E23F001031B041B0C23802B6879
:10449000B3421ED85B00B2FBF3F39BB2042B38BFD0
:1044A0000423013080B22084A3832388AA8843F0A8
:1044B000010323802388698923F481630A4323F05D
:1044C0000203134323802A89AB891343238104B059
:1044D00070BD4BF6FF70EE8886421BBF1920434328
:1044E00003EB4303B2FBF3F30BBFB2FBF3F39BB25B
:1044F0009BB243F48043C3F30B020AB943F00103B8
:104500004FF496724A434FF47A7192FBF1F2013202
:1045100092B243F400432284C6E700BF40420F003A
:10452000A086010041F28832044BC0E90023002339
:1045300083604FF480438381704700BF0000FFBF5A
:10454000038819B143F001030380704723F001038E
:104550001B041B0CF8E7038819B143F48073038034
:10456000704723F480731B041B0CF8E7038819B110
:1045700043F400730380704723F400731B041B0C87
:10458000F8E7038819B143F480630380704723F48C
:1045900080631B041B0CF8E722B141F0010189B2D2
:1045A0000182704701F0FE01F9E701827047008A3D
:1045B000C0B270470388B1F5006F1BBF23F40063DE
:1045C0001B0443F400631B0C03807047838A008B39
:1045D00043EA004321F07F401840431A58425841B3
:1045E0007047002382B0009301930B0F019000935A
:1045F000009B21F07F4153B1019B14330193019B38
:104600001B680B4214BF0120002002B07047019BC1
:10461000090C1833F2E70000204B10B59A6802F03D
:104620000C020C2A30D8DFE802F02F2F2F2F072F93
:104630002F2F072F2F2F2000194B184A0360936844
:104640001849C3F30313CC5C0368E34043609468E8
:10465000C4F302240C5D23FA04F484609268C2F36C
:10466000C2228A5CD340C36010BD99680E4CC1F36E
:1046700083419A68615C9B68094BC2F381524B434A
:104680000132B3FBF2F3D8E74FF400425B68C3F3A7
:104690004233013302FA03F3CFE700BF0038024090
:1046A0000024F4001400002024000020044BDA69E8
:1046B00011B11043D861704722EA0000FAE700BF49
:1046C00000380240044B1A6A11B110431862704757
:1046D00022EA0000FAE700BF00380240044B5A6AA1
:1046E00011B110435862704722EA0000FAE700BF98
:1046F00000380240044B5A6911B1104358617047A9
:1047000022EA0000FAE700BF0038024030B50D464B
:104710000446028AEB8892B222F440521A438989F5
:1047200002828389288923F4B052AB8822F00C02DC
:104730000343688985B003431343A381A38A684672
:104740009BB223F440730B43A382FFF765FFDDE9BF
:104750000231154A944218BF19461923A2894B43C6
:10476000296810044CBF49008900B3FBF1F16425AE
:10477000B1FBF5F3A2891801120405FB13130BD545
:10478000DA003232B2FBF5F202F0070242EA00032D
:104790009BB2238105B030BD1B013233B3FBF5F36F
:1047A00003F00F030343F3E700380140838919B195
:1047B00043F400538381704723F400531B041B0C04
:1047C000F8E7C1F30801818070478088C0F30800D2
:1047D000704701F01F0310B5C1F342140121012CF1
:1047E00001FA03F105D10C3003683AB119430160B5
:1047F00010BD022C0CBF10301430F5E723EA010184
:10480000F5E70388194214BF0120002070470123F7
:10481000C1F3421210B5012A01F01F0403FA04F398
:104820000DD182891340028892B26BB10123090A2B
:1048300003FA01F10A4214BF1846002010BD022AF3
:104840000CBF028A828AEDE71846F7E70B0A0121BE
:104850009940C94389B20180704700002DE9F341B6
:104860001E46002304460D46019317461AB901203F
:1048700002B0BDE8F08140F6FF7301934FF40031C0
:104880002046FFF7AEFE002846D101212046FFF763
:1048900062FE40F6FF73DFF8E48001934146204654
:1048A000FFF794FE00283ED0314600222046FFF755
:1048B00073FE40F6FF732D4E019331462046FFF7FD
:1048C00085FE002835D0297820466E1CFFF76DFE46
:1048D0003D4440F6FF77DFF89880AE42019733D130
:1048E000234D29462046FFF77CFE002838D020467D
:1048F0000121FFF73BFE40F6FF731E4D1E4C019356
:1049000029462046FFF76DFE0028B0D0019B5A1EB5
:104910000192002BF4D104E0019B5A1E0192002B5E
:10492000ACD10020A4E7019B5A1E0192002BB5D107
:10493000F7E7019B5A1E0192002BBED1F1E7019BC4
:104940005A1E0192002BECD041462046FFF749FE4B
:104950000028F4D016F8011B2046FFF726FEBCE71E
:10496000019B5A1E0192002BBBD1DAE7820007009F
:10497000040000101000001000540040010003006B
:104980002DE9F3411E46002304460D4601931746C8
:104990001AB9012002B0BDE8F08140F6FF7301931F
:1049A0004FF400312046FFF71CFE002837D10121CB
:1049B0002046FFF7D0FD40F6FF73DFF8E08001935B
:1049C00041462046FFF702FE002842D03146002231
:1049D0002046FFF7E1FD40F6FF732C4E0193314670
:1049E0002046FFF7F3FD002839D0297820466E1CB9
:1049F000FFF7DBFD3D4440F6FF77DFF89480AE42E1
:104A0000019737D1224D29462046FFF7EAFD0028BD
:104A1000BFD1019B5A1E0192002BF4D104E0019BEF
:104A20005A1E0192002BBBD120460121FFF79EFDAB
:104A300040F6FF73174D184C019329462046FFF7A7
:104A4000D0FD20B1019B5A1E0192002BF5D1002010
:104A5000A0E7019B5A1E0192002BB1D1E4E7019B14
:104A60005A1E0192002BBAD1DEE7019B5A1E019219
:104A7000002BD9D041462046FFF7B3FD0028F4D0E3
:104A800016F8011B2046FFF790FDB8E782000700EB
:104A9000040000101000001000540040010003004A
:104AA0002DE9F3411F46002304460D4601931646A7
:104AB0001AB9012002B0BDE8F0814FF40031FFF7D0
:104AC00090FD08B90020F5E701212046FFF759FDC8
:104AD0004FF2FF712046FFF76DFD01212046FFF7E1
:104AE0003AFD40F6FF73DFF8B88101934146204656
:104AF000FFF76CFD00283AD0394601222046FFF727
:104B00004BFD40F6FF73614F019339462046FFF796
:104B100068FD002831D0012E3BD100212046FFF74F
:104B200030FD04F07FFD31462046238BFFF71EFD4C
:104B300004F098FD40F6FF73554E01933146204630
:104B4000FFF74FFDF8B12046FFF731FD287040F622
:104B5000FF73504D019329462046FFF742FD002880
:104B6000A7D0019B5A1E0192002BF4D1AAE7019B0A
:104B70005A1E0192002BB9D1A4E7019B5A1E019243
:104B8000002BC2D19EE7019B5A1E0192002BD5D16A
:104B900098E7022E29D14FF400612046FFF70AFD65
:104BA00004F040FD00212046238BFFF7EAFC04F0CF
:104BB00059FD40F6FF73384E019331462046FFF70A
:104BC00010FD60B104F02EFD01212046FFF7CEFC60
:104BD000238A2B70238A6B7004F044FDB7E7019B96
:104BE0005A1E0192002BE8D16CE740F6FF77033E96
:104BF000238BDFF8A4802E44B54201972DD1264E99
:104C000031462046FFF7EDFC98B300212046FFF720
:104C1000B8FC04F007FD2046FFF7C9FC012128700D
:104C20002046FFF7A3FC04F01DFD2046FFF7BFFC64
:104C300040F6FF73194E6870019331462046FFF726
:104C4000C5FCE0B12046FFF7B2FCA8707FE7019BEE
:104C50005A1E0192002B3FF435AF41462046FFF724
:104C6000C0FC0028F3D02046FFF7A1FC05F8010B9B
:104C7000C2E7019B5A1E0192002BC1D122E7019B82
:104C80005A1E0192002BD8D11CE700BF0200001071
:104C9000400000101000001004000010400003004D
:104CA0000100030038B5204B08219A691F4842F4DF
:104CB00000129A619A6922F400129A615A6A22F4E7
:104CC00000125A6200F034FD012308211A461748E9
:104CD00000F06CFC09211548012200F0A5FC092117
:104CE000124800F03AFDD8B1012038BD082128460D
:104CF00000F01EFD00F06AFA0821284600F01EFDB3
:104D000000F064FA013CF1D10921084800F025FDCA
:104D100020B94FF4A1710648FEF762FF2046E4E790
:104D20003324024DEEE700BF003802400004024089
:104D30005F7201082DE9FF41444B054698420E463B
:104D400017467CD103F5F2335A6A082142F4001267
:104D50005A629A693E4842F400129A619A6922F4B2
:104D600000129A6100F0E4FC012308211A46384839
:104D700000F01CFC09213648012200F055FC0921F5
:104D8000334800F0EAFC002855D0012308211A46D8
:104D90002F4800F00BFC042208212D4800F082FC73
:104DA000012309211A462A4800F000FC04220921A7
:104DB000274800F077FC274B9A6942F400129A6169
:104DC0009A6922F400129A616846FFF7ABFB224B06
:104DD000694601934FF48063ADF80A304FF4804385
:104DE0002846ADF80C30ADF808700096FFF736FB9A
:104DF00028460121FFF7A4FB012019E008214046C5
:104E000000F096FC00F0E2F90821404600F096FC24
:104E100000F0DCF9013CF1D109210D4800F09DFCC6
:104E20000028B2D10D484FF4B571FEF7D9FE2046E7
:104E300004B0BDE8F0813324DFF81480EAE740F2E3
:104E400079110648FEF7CCFEBEE700BF00540040D3
:104E500000040240003802400000FFBF5F720108FA
:104E600008B50020FFF746F900210748FFF738F999
:104E700000214FF40070FFF725FC044A136823F06B
:104E80000103136008BD00BF002401400038024048
:104E900038B50122072301460F48FFF737F90221F1
:104EA0000D48FFF7C5F90C48FFF7B4F900240B4D86
:104EB00002210948FFF7B6F920B1BDE8384006489D
:104EC000FFF7ADB90134B4F5805FF1DB4C21284622
:104ED000FEF786FEECE700BF00240140A672010841
:104EE000F0B5064689B03248FFF7B4F8314B1A687E
:104EF0000192019A910747D501214FF40070FFF705
:104F0000E1FB0120FFF7F6F82B4A536843F4003326
:104F10005360A2F5374253681B07FCD501250024D6
:104F200002A8FFF7D1F802A921488DF81C508DF88E
:104F30000D4006948DF80C40FFF7A0F82A46062392
:104F400031461B48FFF7E2F829461948FFF7C8F831
:104F500002211748FFF76CF91548FFF75BF9144D6C
:104F6000164F02212846FFF75DF9B8B10825002445
:104F70003046FFF78DFF013D0444F9D1FFF770FF84
:104F8000C4F3CF0009B0F0BD1A6842F001021A6004
:104F9000019A9207B0D41A680192F9E70134B4F586
:104FA000805FDEDB38213846FEF71AFED9E700BF06
:104FB000002401400038024000270140A672010889
:104FC00008B51120FFF78CFFFCF73CF901460848B3
:104FD000FCF744FAFCF728F803A3D3E900230FF009
:104FE000F5FF10F0ADFA08BD2FDD24068195F33FE3
:104FF00000F07F450F4A536A43F0805353620E4BD3
:105000001A465968C906FCD41B68022823F4C05309
:1050100006D143F4C05313605368DB06FCD47047D9
:10502000012802D143F48053F5E70028F3D143F47B
:105030000063F0E7003802400070004010B50C4BF0
:105040005A68D206FCD41C6814F4C05F0BD114F467
:1050500080500AD114F4006404D106482A21FEF7D6
:10506000BFFD204610BD0220FCE70120FAE700BF8B
:1050700000700040B072010838B505460120FFF706
:10508000E7F8022D01BF144A136843F001031360CF
:10509000124B1A6842F480721A601A689205FCD5A5
:1050A0005A6822F4604242F440425A6000229A60F8
:1050B0000A4B9C6814F00C04FBD14FF480721A6008
:1050C000074B084A28461A60FFF794FF2046BDE8C0
:1050D0003840FFF7B1B800BF003C02400038024042
:1050E00010000020D0FE3F000C4B5A6B900513D4EB
:1050F0005A6A42F080525A62094A116841F480713A
:105100001160596B41F480715963596B8905FCD565
:10511000136823F480731360704700BF00380240A7
:1051200000700040054B5A6B910706D45A6B42F051
:1051300001025A635A6B9207FCD57047003802404F
:10514000094B5A6A42F020025A629A6942F02002E0
:105150009A619A6922F020029A610022A3F509332C
:105160001A801A855A6270470038024015210238A9
:10517000002248430121064B1A85D86299825A625F
:105180001A8219801A8AD207FCD500221A80704729
:1051900000140040002349F6FE7282B00193019B87
:1051A000934201DD02B07047019B01330193F6E7A2
:1051B000002340F6FE7282B00193019B934201DD11
:1051C00002B07047019B01330193F6E7002382B0E0
:1051D0000193019BB3F5CC7F01DD02B07047019BC9
:1051E0000133F5E7D0B1012801D1FFF7EFBF0C4B38
:1051F00000211A684FF47A73B2FBF3F2094B013ABB
:1052000092B21A8501220138D8629A8259621982B3
:105210001A801A8AD207FCD500221A80704700BF74
:10522000100000200014004000F1774303F57803DC
:10523000B3F5804F2DE9F04106460C4617462DD2B6
:1052400002F1F73303F608030344B3F5804F25D288
:10525000FFF7F4FE804610B10020FFF7CBFEFFF70A
:105260000FF801252744361BA7420AD1FFF718F88B
:10527000B8F1000F02D04046FFF7BCFE2846BDE85B
:10528000F08141F60270FFF713F8301914F8011B92
:10529000FFF76AF8042818BF0025E5E70025EDE7C9
:1052A00010B50C4600F1774101F57801B1F5804F5A
:1052B0000DD202F1F73303F608030344B3F5804F30
:1052C00005D2014620460DF023FA012010BD002032
:1052D000FCE7000008B5114B984215D003F5806338
:1052E000984213D003F58063984211D003F5806390
:1052F00098420FD003F5006398420DD0084B094A3D
:10530000142109480DF0C0F8002008BD0120FCE779
:105310000220FAE70320F8E70520F6E70000024044
:1053200003730108BD7201081C7301080F2808B53A
:1053300005D9094B094A3B2109480DF0A5F801237D
:1053400003FA00F0C043074A5168014051601368F6
:105350001840106008BD00BF29730108C77201081A
:105360001C730108000401400F292DE9F84F824603
:105370000D4693461F4605D95A4B5B4A55215B485B
:105380000DF082F84FF0010909FA05F900F0B8F8BC
:105390006FEA0903564E032D7268564C02EA030267
:1053A0007260326803EA0203534A3360136A43F0BF
:1053B000010313622ED80F22A3684FEA850802FA70
:1053C00008F223EA0203A3605046FFF783FFA368B5
:1053D00000FA08F01843A0601BF0020F18BFB36872
:1053E000464A1CBF43EA0903B3601BF0040F1EBF0B
:1053F000F36843EA0903F360336843EA090333605F
:105400003B01DBB2002D45D182F806334023136007
:10541000BDE8F88F072D13D80F22A5F10408E36823
:105420004FEA880802FA08F223EA0203E3605046D2
:10543000FFF750FFE36800FA08F01843E060CBE79D
:105440000B2D13D80F22A5F1080823694FEA88080D
:1054500002FA08F223EA020323615046FFF73AFFFB
:10546000236900FA08F018432061B5E70F22A5F17F
:105470000C0863694FEA880802FA08F223EA02037B
:1054800063615046FFF726FF636900FA08F018438E
:105490006061A1E7012D03D182F807338023B6E7CD
:1054A000022D04D182F808334FF48073AFE7032D47
:1054B00004D182F809334FF40073A8E7042D04D116
:1054C00082F80A334FF48063A1E7092D04D882F8EB
:1054D00017334FF400039AE782F828334FF48073B0
:1054E000536095E735730108E27201081C730108E7
:1054F00000040140000001400038024000E100E0EB
:10550000144B984205D1144AD36943F00103D36187
:105510007047124B984204D10F4AD36943F00203FB
:10552000F5E70F4B984204D10B4AD36943F00403CB
:10553000EDE70C4B984204D1074AD36943F00803C6
:10554000E5E7094B9842E3D1034AD36943F02003CE
:10555000DDE700BF000002400038024000040240C6
:1055600000080240000C02400014024003234900DE
:1055700010B584688B4024EA030484600124022A65
:1055800004FA01F407D0032A0DD0012A07D1836859
:105590002343836003E083688A401A438260836800
:1055A0001C43846010BD82681343F2E70F29F8B5ED
:1055B00004460F4615461E4603D940211948FEF7FA
:1055C0000FFB2046FFF79CFF03237A009340DB4349
:1055D0002168194021600121D4F800C001FA02F0CD
:1055E0004CEA000CB940C4F800C009B266B1A68804
:1055F000314389B2A180E168012D03EA0103E36030
:1056000006D0022D08D0F8BDA68826EA0101F1E7F0
:10561000E3680343E360F6E7E36805FA02F21A433E
:10562000E260F0E7857301080F2970B505460C4666
:10563000164603D960210E48FEF7D2FA2846FFF736
:105640005FFF032361008B40DB43EA68012E02EA1F
:105650000302EA6005D0022E03D02A6813402B60B3
:1056600070BDEA6806FA01F11143E960F5E700BF91
:10567000857301080F2910B505D9074B074A762114
:1056800007480CF001FFFFF73BFF4B0003210268C6
:1056900099401143016010BD29730108417301084D
:1056A000857301080F2938B50446154605D97C21B4
:1056B0001B4B1C4A1C480CF0E7FE0F2A03D91B4B5E
:1056C000184A7D21F6E7FFF71BFF07294FF00F036C
:1056D00018D8006A8A00934020EA03032362236AF1
:1056E00005FA02F21A4322620322236849008A4023
:1056F00023EA020323600223226803FA01F1114323
:10570000216038BDA1F10802406A9200934020EA6E
:1057100003036362636A95401D436562E4E700BF6B
:105720002973010854730108857301087273010815
:10573000012303FA01F189B201837047012303FABF
:1057400001F189B241837047012303FA01F189B263
:105750000AB10183704741837047008A084100F015
:10576000010070470F2938B505460C4603D9A92119
:105770000548FEF735FA28686400E04000F00300B1
:10578000431E5842584138BD85730108808A08413C
:10579000C04300F00100704710B5084C23681BB9E6
:1057A000012004F0D5FA206023682BB9BDE8104031
:1057B00036210348FEF714BA10BD00BF3809002097
:1057C0009073010810B50B4C22681AB93C210A48A5
:1057D000FEF706FA206842F2107104F001FC01287D
:1057E0000CBF0124002403D040210348FEF7F8F940
:1057F000204610BD380900209073010810B5074CF1
:1058000022681AB94D210648FEF7EAF900232068FC
:105810001A46BDE81040194604F0F6B938090020D0
:105820009073010810B50446FFF7B6FFFFF7CAFFF3
:10583000214610220348FFF77DFA0446FFF7DEFFFA
:10584000204610BD0054004010B5FFF7A5FFFFF73C
:10585000B9FFFFF727FA0446FFF7D0FF204610BD37
:1058600008B513460A4601460348FEF7F7FF003025
:1058700018BF012008BD00BF0054004008B5134602
:105880000A4601460348FFF77BF8003018BF0120A5
:1058900008BD00BF0054004008B513460A46014643
:1058A0000348FFF7FDF8003018BF012008BD00BF16
:1058B000005400400A23B0FBF3F203FB120040EA5D
:1058C0000210C0B270470000CA22024B5A62532233
:1058D0005A62704700280040014B1860704700BFB3
:1058E0003C0900204FF400320F4B10B50F4C5A61A9
:1058F000E368DB0503D430210D48FEF771F9FFF7AB
:10590000E3FF4FF40072A36823F48853A360094BAC
:10591000C3F88420FF236362074B1B6813B1BDE803
:105920001040184710BD00BF00040140002800408F
:10593000D673010800E100E03C0900202DE9F04F9A
:105940009846374B85B01B78824691469DF8387053
:105950009DF83C602BB9334B334A8C2133480CF013
:1059600093FD431E1E2B59D80C2957D8A2F5FA6374
:10597000632B53D8B8F1170F50D83B2F4ED83B2E7E
:105980004CD802F13000C0B2FFF794FF83460846BE
:10599000FFF790FF04465046FFF78CFF40F4005598
:1059A0004046FFF787FF45EA0B4545EA04250446D4
:1059B0003846FFF77FFF000240EA04443046FFF715
:1059C00079FF20431A4CFFF77FFFE36843F0800321
:1059D000E360E3685B06FCD565602060E36823F064
:1059E0008003E360124BDA689206FCD5FF2204A81C
:1059F0005A6200F80C6D8DF807A08DF80810ADF80C
:105A000009908DF806808DF8057001F00AFB094BAE
:105A1000C3E90001012005B0BDE8F08F0020FAE7DE
:105A200040090020D09E01081C740108D6730108AB
:105A3000002800404809002037B50578C4788378ED
:105A4000B0F8052001790195407800902046FFF7D5
:105A500075FF03B030BD000038B52B4B04461B78F2
:105A60001BB9E4212948FEF7BBF8294AD36823F083
:105A70002003D360D3689B06FCD513685268C2F339
:105A80000741080900EB800001F00F0101EB400124
:105A9000C9B201F5FA61A4F80510C2F30721C1F3F8
:105AA00000108500284401F00F0101EB4001D2B243
:105AB0002171C2F3011101EB810102F00F0202EB2F
:105AC0004102E270C3F30742C2F3011101EB81010D
:105AD00002F00F0202EB4102A270C3F30722C2F3ED
:105AE000021101EB810102F00F0202EB4102DBB275
:105AF0006270C3F3021202EB820203F00F0303EBA6
:105B00004203237038BD00BF40090020D67301084E
:105B1000002800401FB501A8FFF79EFF01A801F073
:105B200080FA05B05DF804FB08B5FFF7DDFA1B4A03
:105B3000136843F480731360FFF7C6FE184A536B73
:105B400023F4403343F482035363164BDA6842F084
:105B50008002DA60DA685106FCD5FF221A611A6900
:105B600042F4FE021A619A6822F040029A609A6832
:105B700022F44C529A60DA6822F08002DA60094B13
:105B8000DA689206FCD5FF225A620122064B1A708F
:105B9000FFF7C0FF054BC3E9000108BD00700040DE
:105BA0000038024000280040400900204809002039
:105BB00008B5094B1B7823B940F21F110748FEF7BF
:105BC0000FF8FFF781FE064B9A6822F480729A6004
:105BD000FF225A6208BD00BF40090020D6730108A9
:105BE0000028004008B5144B1B7833B9134B144AF6
:105BF00040F2271113480CF047FCFFF765FE124BEB
:105C0000DA6822F48072DA60104A916841F4003157
:105C10009160116841F400311160F0210C4A82F862
:105C200029134FF4007151609A6842F488529A60C7
:105C3000FF225A6208BD00BF40090020D09E010823
:105C400028740108D67301080028004000040140B0
:105C500000E100E0F8B51E46194B17461B7833B932
:105C6000184B194A4FF4A37118480CF00DFC184C4E
:105C7000FFF72AFEA56825F48075A560E56825F480
:105C80008075E560FFF716FE05460846FFF712FE31
:105C9000000440EA05613846FFF70CFE0546304631
:105CA000FFF708FE084340EA0520E368DB07FCD560
:105CB000FF23E0616362BDE8F840FFF793BF00BFD8
:105CC00040090020D09E01083D740108D6730108E8
:105CD0000028004038B50D46044603F0A3FC194ADD
:105CE000136823F00103136003F0BCFC25B1164ACE
:105CF000536843F00603536072B6BFF34F8FBFF390
:105D00006F8F124A0120136823F0030343F40073DA
:105D100043F001031360FEF7A7FA0D4B1A6942F036
:105D200004021A6130BF1A69022022F004021A61CB
:105D3000FFF7A2F9034A136843F00103136004B1AB
:105D400062B638BD10E000E0002004E000700040C2
:105D500000ED00E062B6704700220E4B10B51A70DD
:105D60000D4A0E4C1388204623F040031B041B0CE5
:105D700013800D210222FFF757FC204602220E213C
:105D8000FFF752FC2046BDE8104002220F21FFF72A
:105D90004BBC00BF50090020003800400004024006
:105DA000284A38B5136A054643F480531362052226
:105DB00025480C461146FFF775FC052206212248AE
:105DC000FFF770FC052207211F48FFF76BFCC5B1E8
:105DD000022205211C48FFF7C9FB022206211A48AE
:105DE000FFF7C4FB022207211748FFF7BFFB012C76
:105DF00021D144F451740122144B1C80144B1A70AD
:105E000038BD2A4605211048FFF7B0FB2A46062177
:105E10000D48FFF7ABFB2A4607210B48FFF7A6FB0F
:105E2000012C05D0022C03D0032C14BF0024032422
:105E300044F45974DFE7022CDBD0032C0CBF03249D
:105E40000024D6E700380240000002400030014044
:105E50005109002000220E4B10B51A700D4A0E4C4D
:105E60001388204623F040031B041B0C13800521DC
:105E70000222FFF7D9FB204602220621FFF7D4FBBE
:105E80002046BDE8104002220721FFF7CDBB00BF2E
:105E9000510900200030014000000240064B074A33
:105EA000988111781A461889C00701D40029FAD1BF
:105EB0009089C0B2704700BF0030014051090020F6
:105EC000054AD36823F4E0631B041B0C43F0BF6353
:105ED00043F40033D360704700ED00E0202200213E
:105EE000114B10B5C3F88420104B114C1A6A204690
:105EF00042F480421A625A6942F480425A615A69F5
:105F000022F480425A610B4A91811A6A092122F4D3
:105F100080421A620222FFF787FB2046BDE810404C
:105F200002220A21FFF780BB00E100E000380240B6
:105F3000000002400038014010B50B4C40F22551E2
:105F40002046FEF764FC48B12046FEF73EFC074BB6
:105F5000C0B21B6833B1BDE810401847A388044A9B
:105F6000DBB2137010BD00BF00380140540900209F
:105F70000450002010B5044680210848FEF741FC7B
:105F80000028F9D021460548FEF71BFC034C4021B0
:105F90002046FEF736FC0028F9D010BD003801403D
:105FA00010B5441E14F8010F00B910BDFFF7E2FF51
:105FB000F8E7000008B50248FEF707FCC0B208BDCC
:105FC000003801402DE9F0410D46012188B080469E
:105FD000084617461C46FEF769FB01214FF4804036
:105FE000FEF770FB4FF4C0630122029300260223E8
:105FF00002A933488DF80C308DF80D308DF80F2044
:106000008DF80E60FEF7D6F9072209212C48FEF71D
:1060100013FA07220A212A48FEF70EFA092F0ABFAF
:106020004FF48053ADF81460ADF81430052CCDF862
:10603000108033D14FF48053452DADF8163038D150
:106040004FF480630024ADF818300C2304A91D48D8
:10605000ADF81A30ADF81C40FEF758FB224640F26E
:1060600025511848FEF7B5FB01211648FEF79EFBA7
:10607000FFF7A0FF25238DF804309DF838308DF808
:1060800006408DF8053001238DF80730FFF718FF23
:1060900001A8FDF7C3FF08B0BDE8F0810F2C02D1C5
:1060A0004FF44053C8E7022C0CBF4FF400530023B9
:1060B000C2E74F2D0CBF4FF4C0630023C2E700BFFF
:1060C00000000240003801400E2307B5082200936B
:1060D0004E210123FFF776FF03B05DF804FB0000BB
:1060E000402200210D4B0E48C3F884200D4B5A6A04
:1060F00042F400325A629A6942F400329A619A6913
:1061000022F400329A61084A91815A6A032122F4EA
:1061100000325A620222FFF787BA00BF00E100E0B6
:1061200000000240003802400044004008B5024828
:10613000FEF74BFBC0B208BD004400402DE9F04F14
:1061400000271D46262389B09DF84880894692463F
:106150008DF8043083469DF84C409DF850608DF8D2
:1061600005808DF806708DF80770FFF7A9FE01A86D
:10617000FDF754FF01210846FEF798FA01214FF47C
:106180000030FEF7ABFAACB10823029302238DF87E
:106190000E708DF80C300327012302A949488DF8B1
:1061A0000F308DF80D70FEF705F907223946454886
:1061B000FEF742F9B6B10423029301238DF80F30A4
:1061C000002302278DF80E30032302A93D488DF8E5
:1061D0000C708DF80D30FEF7EDF80722394639487E
:1061E000FEF72AF9BAF1090F0CBF4FF480530023D0
:1061F000052DCDF810B0ADF814303CD14FF48053DC
:10620000B9F1450FADF8163040D14FF48063002549
:10621000ADF81830ADF81C50002E3ED1ADF81A6024
:106220005CB1BDF81A30002243F0040340F225515E
:106230002548ADF81A30FEF7CCFA04A92248FEF73B
:1062400065FA01212048FEF7B1FA0CB1FFF76EFFA5
:1062500026238DF8043000238DF8063001238DF8B5
:1062600005808DF80730FFF72BFE01A8FDF7D6FE5D
:1062700009B0BDE8F08F0F2D02D14FF44053BFE7B6
:10628000022D0CBF4FF400530023B9E7B9F14F0FB3
:106290000CBF4FF4C0630023B9E708232A4640F23D
:1062A00027710948ADF81A30FEF793FA40F22661DB
:1062B0000548FEF7CBFA2A4640F226610248FEF76F
:1062C00088FAADE70000024000440040F8B50546FA
:1062D0000024134E134F80211348FEF792FA68B141
:1062E00029461148FEF76DFA00240F4D0C4E0D4F54
:1062F00040212846FEF785FA48B1F8BD0134B44282
:10630000E9D940F219113846FDF76AFCE3E7013498
:10631000B442EDD94FF491713846FDF761FCE7E7DF
:10632000FFFF0F004F7401080044004008B5064B02
:106330000246186000B1012240F225510348FEF7E1
:1063400048FA012008BD00BF580900200044004061
:1063500010B540F226611148FEF759FA40B140F2FB
:1063600026610E48FEF772FA0D4B1B6803B1984781
:106370000A4C40F225512046FEF749FA48B1204622
:10638000FEF723FA074BC0B21B6833B1BDE81040DB
:106390001847A388044ADBB2137010BD00440040C4
:1063A0005C0900205809002004500020BFF34F8FE3
:1063B0000449054BCA6802F4E0621343CB60BFF3A3
:1063C0004F8FFEE700ED00E00400FA0510B5441E13
:1063D000E3B2052B03D90E211148FDF701FCFEF7AE
:1063E000A1FE45F255520F4B1A60DA68D207FCD471
:1063F000052C06D8DFE804F003090B0D0F1101226C
:106400005A604CF6CC421A6010BD0222F8E7032213
:10641000F6E70422F4E70522F2E70622F0E700BFE0
:106420009674010800300040F8B50E46054680B16C
:106430004F1C384600F040FF044640B13A46002168
:106440000CF08AF93246294620460CF061F92046C4
:10645000F8BD0446FBE738B50D46044628B10DF0FB
:106460004FF823462044834201D1002038BD13F861
:10647000012BAA42F7D10120F8E737B504460D46B3
:106480000CF02EF8002201A9026020460DF064F9FC
:1064900004460CF025F80368222B08D0019B1B78DA
:1064A0002BB9002C03DB20462B6003B030BD012349
:1064B00000202B60F9E700002DE9F04F05464FF072
:1064C000010B002687B0CDE9031206F10903122B58
:1064D0008CBF0320022000F0EFFE0090E8B13246AE
:1064E00036490CF0DBFF039B53F82690EDB90024EE
:1064F000009800F0CBFEBBF1000F02D1284600F05F
:10650000C5FE84B1049B0136B34225464FF0000B13
:10651000DBD1204607B0BDE8F08FBBF1000F02D100
:10652000284600F0B3FE0024F3E7254B4FF00008A7
:10653000B9F1000F08BF994648460CF0E1FF019001
:1065400000980CF0DDFF0290284649460DF007F850
:10655000B8B928460CF0D4FFDDE9012301309B1ABD
:1065600008FB030000F0A8FE04460028BFD0034645
:106570002F4618F1FF3809D2394618460CF0B8FFFB
:10658000B6E7019B08F101081844DEE749463846A2
:1065900005930CF0E4FF059BA0EB070A5246394631
:1065A00018460CF0C7FF009950440CF0A1FF019A67
:1065B000029B9244C3185744DBE700BFC67501082D
:1065C000C763010830B580B10346021F00F118040B
:1065D00052F8045F8D4208D0A242F9D11C301A460D
:1065E00014680433013401D1116030BD8342F6D107
:1065F000FBE770B5044680B1064600EB8105AE426C
:1066000004D12046BDE8704000F040BE56F8040BAF
:106610000028F4D000F03AFEF1E770BD2DE9F74F05
:1066200089460092002838D00027C45D8CBB0546FF
:106630008346264600EB070AD34538D104B101361C
:10664000002E6FD00137384600F036FE8346002812
:1066500066D03A4600210CF07FF8B00000F02CFE26
:106660000446002860D04FF000084146AA4532D1C8
:1066700031B15846FFF7D8FE002855D044F828001D
:10668000584600F003FE009B1E60204603B0BDE8A4
:10669000F08F0137B7F5807FC7D10024264620460A
:1066A00000243146FFF7A5FF009B1C60EDE79BF837
:1066B00000304B4505D10CB1002401360BF1010B24
:1066C000BAE70BF0E7FF9BF80030184443781B074C
:1066D00058BF0134F2E72B784B4513D181B15846AE
:1066E000FFF7A2FE00B308F1010344F828000021DF
:1066F0003A46584601930CF02FF8019B002198462A
:106700000135B3E701910BF0C5FF2B7801991844CF
:10671000407810F0080F04BF0BF801300131EFE7AB
:106720000446BCE73446B0E7584600F0AFFDB6E794
:106730002DE9F743002506460820884691461F4666
:10674000009500F0B9FD0446002868D0C0E9005566
:1067500030460CF0D5FE01280FD133782A2B0CD10E
:1067600009F1FF33C4F80080636022684A4502D211
:1067700063684B4543D32B4B0EE02D213046FFF78A
:106780006AFE0546C0B902A941F8040D3046FFF77C
:1067900074FE019B63B1244B3B6000992846FFF7D0
:1067A00028FF002C37D0204600F070FD002432E096
:1067B000C4E900001D46D8E76A462D213046FFF7A0
:1067C0002DFF009B0546013B012B01D9174BE3E749
:1067D000002302AE46F8043D31460068FFF74DFE47
:1067E0002060019B0BB1124BD6E731466868FFF77A
:1067F00044FE6060019B002BB7D00E4BCCE74245B6
:1068000001D3434501D20C4BC6E700992846FFF758
:10681000F0FE00233B60204603B0BDE8F083054650
:10682000BBE700BF81750108FB7401081A750108F8
:106830004375010862750108A175010838B590B16A
:10684000451E15F8014F0CB9204638BD0BF022FF4C
:1068500023462044427802F00302022A08BFA4F132
:1068600020032B70EDE70120EFE708B520B34A1CA9
:1068700022D0062920D8DFE801F0040D10131619E4
:106880001C00002303600CF049F80840431C5842E8
:10689000584108BD00234360F5E700238360F2E719
:1068A00000238361EFE70123C360ECE7002303616A
:1068B000E9E700234361E6E70120EAE770B5064611
:1068C0000D1F01F1180455F8041F4B1C03D1A542FC
:1068D000F9D1002070BD3046FFF7C7FF0028F6D081
:1068E000F8E708234A4291FBF3F302F0070201F0B4
:1068F000070158BF51420122DBB2C9B202FA01F1CD
:10690000C25C1143C154704708234A4291FBF3F320
:1069100002F0070201F0070158BF51420122DBB229
:10692000C9B28A40C15C21EA0201C1547047082300
:1069300091FBF3F3DBB2C05C4B4203F0070301F0C1
:10694000070158BF5942C9B2084100F00100704721
:106950002DE9F047089E8A4690461D46DDF82890AE
:10696000074610B11446A24507D875B90122002484
:106970000B9B1A602046BDE8F08721463846FFF79A
:10698000D6FF002861D10134EDE7099B023B042BBF
:1069900004D8DFE803F0282C2C3034006B68013376
:1069A0006B6028460BF0BAFF013108BFB0F1FF3F22
:1069B000DCD031462846FFF758FF0028D6D12FB348
:1069C000044621463846FFF7B2FF002841D1013482
:1069D000A245F6D10446013E042E19D8DFE806F0A0
:1069E0002B2D2F313300AB680133AB60D9E7EB6857
:1069F0000133EB60D5E72B6901332B61D1E76B697C
:106A000001336B61CDE7002DE5D1AFE73C46E2E70E
:106A10002C6028460BF082FF013108BFB0F1FF3F28
:106A2000A4D0B9F1000FA1D049462846FFF746FF90
:106A300000289FD09AE76C60EBE7AC60E9E7AC61B7
:106A4000E7E7EC60E5E72C61E3E7A045DBD14446EE
:106A500090E7A045BFD1FAE700232DE9F04F0646A5
:106A60008BB01C200C469046099300F025FC05468F
:106A7000002800F0E4801C2000F01EFC07460028DF
:106A800000F0DD804FF0FF31021F2B1F05F11800D1
:106A900043F8041F984242F8041FF9D10023012152
:106AA000D4F800A00DF12409CDE90031CDE9027937
:106AB0003C21234652463046FFF74AFF09990029F8
:106AC0006ED1824502D12846FFF77CFD02234FF0AC
:106AD000010AD4F804B0CDE900A3CDE90259234658
:106AE0005A463C2106F10800FFF732FF099B002BB4
:106AF00056D183454CD151462846FFF763FD032309
:106B00004FF0020AD4F808B0CDE900A3CDE902594C
:106B100023465A46182106F11000FFF719FF099B7A
:106B2000002B3DD1834546D151462846FFF74AFD0B
:106B300040F26F1BA3690593E368049306F1140305
:106B40000693DDF810A006F113030793514606984B
:106B5000FFF7EDFE28B105990798FFF7E8FE00283A
:106B600036D1BBF1010B33D0E36820460133E3603B
:106B70000BF0D4FE013108BFB0F1FF3F24D0A36970
:106B800029462046D4F80CA00593FFF797FEDDE7D1
:106B9000424621463046FFF75FFF09900028AED0FD
:106BA000284600F073FB17B1384600F06FFB0998D8
:106BB0000BB0BDE8F08F424621463046FFF74CFF50
:106BC00009900028ECD1B3E701234FF0000A0993A4
:106BD000099B002BE4D1049B534520D10421284676
:106BE000FFF7F0FC05230622D4F810A0CDE900320F
:106BF000CDE90259234652460C2106F11800FFF751
:106C0000A7FE099B002BCBD18245C9D06369A3EBBA
:106C10000803042B0CD94FF0FF330993C0E7424619
:106C200021463046FFF718FF09900028B8D1D9E770
:106C3000424621463046FFF70FFF0990B0E74FF07C
:106C4000FF330993002DB2D00027A9E72DE9F04FBB
:106C5000002487B0924606AA894642F80C4D2C21A2
:106C60009846109DFFF7DAFC074688B93E4B2B602B
:106C700003993846FFF7BDFC07B0BDE8F08FD0F8A8
:106C800000B072685A451CD2304600F0FFFA013459
:106C9000039BA342ECD957F824602F213046FFF71D
:106CA000DAFBA8B92B46304642465146FFF740FD75
:106CB0002B680646002BE2D00028D9D000F0E6FA77
:106CC000D6E759464846FFF70CFE0BF1010BD8E713
:106CD00000232F21304604AA0493FFF79FFC049958
:106CE00006464B1E012B04D9204B2B60FFF781FC7D
:106CF000BEE742462B4651460068FFF719FD2A6859
:106D000083462AB108B100F0C1FA04993046EDE794
:106D10002D213068FFF79FFB18B908F1FF32CBF83F
:106D20000420002306A941F8043D7068FFF7A5FB85
:106D3000059A00901AB10E4A58462A60E3E7DBF83C
:106D40000020DBF80410914205D230460499FFF789
:106D500050FC584699E7114648460192FFF7C1FD9D
:106D6000DDE900321A44ECE7C9750108DB7501085A
:106D7000007601082DE9FF4100230E4603931446D7
:106D800002B902AC236048B90546564B236003990B
:106D90002846FFF72EFC04B0BDE8F08103AA2021AD
:106DA000FFF73CFC039B0546062B02D04E4B2360AD
:106DB000EDE71A22002130460BF0CEFC00940022B1
:106DC0003C2331462868FFF741FF2268002ADED1C4
:106DD00000943C2306F108016868FFF737FF22683A
:106DE000002AD4D10094182306F11001A868FFF7F7
:106DF0002DFF2368002BCAD16869FFF71FFD07220A
:106E00003A496869FFF758FB80460CF079FB012886
:106E100006F1130706D198F800303F2B04BF2A2350
:106E200088F8003000220823394640460094FFF7D6
:106E30000DFF404600F02AFA2268002AA7D1072158
:106E40003846FFF774FD30B111463846FFF749FD6B
:106E50000721FFF759FDEF6806F1140838460CF0DA
:106E60004FFB012804D13B783F2B04BF2A233B7002
:106E700020230022414638460094FFF7E7FE002118
:106E80004046FFF741FD2368002B80D12F6938462B
:106E9000FFF7D4FC00287FF47AAF38460D2214495E
:106EA000FFF70AFB074600283FF471AF183600943D
:106EB0000D2301223146FFF7C9FE384600F0E6F9FE
:106EC000012421463046FFF732FD30B1611E3046C5
:106ED000FFF707FD2146FFF717FD01340D2CF0D118
:106EE00055E700BFA5740108BD74010830000020FB
:106EF0004C000020F0B58DB0CDE90023054628B93F
:106F00004FF0FF304FF0FF310DB0F0BD24220021D3
:106F100003A80BF021FC03A968460BF00BFB044609
:106F20000028EDD00BF0FAFC4A1C08BFB0F1FF3F7F
:106F300006460F46E4D0626921462846FFF78CFDDD
:106F40000028DDD120460BF0E9FC4B1C08BFB0F156
:106F5000FF3FD5D08F4208BF864203D020460BF0BA
:106F6000DDFCD1E723682046013323600BF0D6FC1B
:106F7000013108BFB0F1FF3FC2D062692146284607
:106F8000FFF76AFD0028E9D0BAE770B53C258AB062
:106F9000DDE90E64019496FBF5F405FB146402949C
:106FA000182493FBF4F505FB1433CDE90330481E98
:106FB0000C2190FBF1F301FB13010023CDE9073312
:106FC0009DF84030A2F26C7201A8059106920993D7
:106FD0000BF0A4FC0AB070BDF7B5044602A860E946
:106FE00002230BF095FA0269037A551C426990F866
:106FF00004C0077B02F26C71067EC2690068A37050
:107000000033207018BF01232046013284F801C0EC
:10701000E7702571A4F80510E6712272637203B05F
:10702000F0BD30B5457A85B0C4788378B0F80520D6
:107030000179029505780195407800902046FFF788
:10704000A4FF05B030BD904271EB0303B4BF012033
:1070500000207047032210B5104986B00B78013329
:1070600093FBF2F202EB42029B1A0D4A0B7052F8AC
:1070700023400278B0F80530049242781A21039236
:1070800082780292C2780192027920460092054AE3
:107090000CF0D0F9204606B010BD00BFAE090020AC
:1070A000A47601086F7601081FB502460B4601A8B9
:1070B000FFF792FF01A8FFF7CDFF05B05DF804FBD5
:1070C0002DE9FF4703220D462B4900280B78044683
:1070D00003F1010393FBF2F202EB4202A3EB020382
:1070E000264A0B7052F8236075F100033EDA4FF028
:1070F000010A444265EB4505214A00232046294602
:107100000EF00AFB1E4A07460023204629460EF0D1
:1071100003FB104619464FF4616200230EF0FCFA9F
:107120004FF4616280460023204629460EF0F4FAAF
:10713000104619463C2200230EF0EEFA3C2281460E
:107140000023204629460EF0E7FACDF80080CDE96D
:1071500001923B46BAF1000F0BD00A4A1A21304681
:107160000CF068F9304604B0BDE8F0874FF0000A33
:10717000C2E7054AF2E700BFAE090020A476010885
:10718000805101008D7601088E7601080FB404B09D
:10719000704700000FB437B51B4C256855B9032262
:1071A0002946012002F00CFD2B462A462946206084
:1071B00002F02AFD154D2A68013A03321ED86421D7
:1071C000206802F00DFF8022002111480BF0C4FA64
:1071D00007AB069A80210E4801930CF02DFD7F2805
:1071E00003DD0C490C480CF083F92B6808489847DC
:1071F000002320681A46194602F006FD03B0BDE8D8
:10720000304004B0704700BF380A0020B0090020A9
:10721000B809002005A80108330A00200FB410B5F2
:107220000D4CA2B02268013A033210D825AB249A43
:10723000802102A801930CF0FFFC7F2804DD0749A0
:107240000DF183000CF054F9236802A8984722B08E
:10725000BDE8104004B07047B409002005A801083B
:1072600070B50446074E4518AC4204D1BDE87040E5
:107270000548FFF78FBF14F8011B3046FFF78AFF60
:10728000F2E700BF1E670108C663010810B5044697
:1072900070B102F0EFFA204602F090FB02F0C2F962
:1072A000BDE81040034A93880133938002F0DAB9B5
:1072B00010BD00BF0650002070B5214C8AB0226876
:1072C00006460132632A22601E4D0BDD03F016FED6
:1072D0000523002201A903F0C3FD03F0CBFA00232C
:1072E0002860236003F0C6FA2B6803F57A7398428E
:1072F00004D903F0BFFA002328602360124A134C1C
:1073000013781BB9236063600123137002F0B2FA93
:10731000304602F0C1FA054668B1324600210BF052
:107320001BFA02F07FF923880133238002F09AF9D7
:1073300028460AB070BD638801336380F8E700BF58
:10734000400A0020440A00203C0A00200650002089
:1073500038B50D46044602F08DFA284602F02EFBA1
:10736000A3880133A38038BD38B50D46044602F02A
:1073700081FA284602F090FA18B12388013323805D
:1073800038BD638801336380FAE7A0F14103052B20
:1073900002D83738C0B27047A0F16103052B01D87D
:1073A0005738F7E73038C0B20A2828BFFF207047A7
:1073B0000022013910B50144441E8C4204D014F857
:1073C000010F08B1002A01DA104610BDFFF7DDFFFA
:1073D0000F2802D840EA0212EFE74FF0FF32F3E73E
:1073E0000068704700687047006800BA704783788B
:1073F00042781B04007843EA02231843704742781E
:10740000007840EA022070470B12017043700B14A1
:1074100009168370C170042070470B12037041700D
:107420000220704738B505460C460BF0BFFF611BC4
:10743000013190FBF1F303FB1100284438BD38B54E
:10744000451E15F8014F04B938BD0BF023F923464A
:107450002044427802F00302012A08BF20332B7037
:10746000EFE72DE9F04106460CF04AF830B300276B
:1074700034180BF00FF914F8013C354618444378E2
:10748000621E19070DD42F463B78A4EB0508013581
:107490005BB908F1010239463046BDE8F0410BF016
:1074A00042B904F8017C1446E3E70BF0F3F815F851
:1074B000013C184443781B07E5D4EAE7BDE8F081B6
:1074C00008B50CF00BF8B0FA80F0400908BD007860
:1074D000013070470FB404B0704700002DE9FF473A
:1074E0000F46002104AC254E44F8041D8046924608
:1074F00030682246994602F023FE0128039B31D1D1
:107500003BB14FF080521E4B1A60BFF34F8FBFF359
:107510006F8FB7F5C87F88BF4FF4C87741463A46AA
:1075200018480BF0F5F8184D164B21463068AF801F
:107530002B60A5F806A085F8089002F075FC039B67
:107540003BB14FF080520E4B1A60BFF34F8FBFF329
:107550006F8F0E480094002301220421006803F07D
:107560008FFE039B3BB14FF08052054B1A60BFF377
:107570004F8FBFF36F8F04B0BDE8F087440C00203D
:1075800004ED00E0AC0A0020A00A00204C0C002012
:107590000348002301220221006803F007BE00BF58
:1075A0004C0C00201FB500230C4904AA42F8043DEE
:1075B00008700B48009240210122006803F060FE31
:1075C000039B3BB14FF08052064B1A60BFF34F8FC5
:1075D000BFF36F8F05B05DF804FB00BF940A002075
:1075E0004C0C002004ED00E01FB5002304AA42F873
:1075F000043D0A48009280210122006803F040FE09
:10760000039B3BB14FF08052054B1A60BFF34F8F85
:10761000BFF36F8F05B05DF804FB00BF4C0C00207A
:1076200004ED00E01FB5104B1C680346A8B1002311
:1076300004AA42F8043D009208210122204603F0EA
:107640001FFE039B3BB14FF08052084B1A60BFF303
:107650004F8FBFF36F8F04B010BD01220821204669
:1076600003F0A4FDF7E700BF4C0C002004ED00E0A0
:107670001FB5002304AA42F8043D009201220948E4
:107680001146006803F0FCFD039B3BB14FF08052B4
:10769000054B1A60BFF34F8FBFF36F8F05B05DF8D6
:1076A00004FB00BF4C0C002004ED00E01FB50023DC
:1076B00004AA42F8043D0A48009210210122006801
:1076C00003F0DEFD039B3BB14FF08052054B1A6087
:1076D000BFF34F8FBFF36F8F05B05DF804FB00BFA2
:1076E0004C0C002004ED00E0004870478C0A00209C
:1076F000114810B5002303224FF48071006803F095
:1077000055FD4FF080520D4B1A60BFF34F8FBFF302
:107710006F8F0B4C206802F05FFD40B1BDE8104058
:10772000002308481A461946006802F06DBA012085
:1077300003F0F2F9EEE700BF4C0C002004ED00E08E
:10774000480C0020400C0020F8B5104B014618688A
:1077500002F046FC0446B8B14FF080560C4F0D4D78
:10776000002303224FF40071386803F01FFD2E60E0
:10777000BFF34F8FBFF36F8F386802F0F1FF2E60B9
:10778000BFF34F8FBFF36F8F2046F8BD400C002032
:107790004C0C002004ED00E070B5044678B103788D
:1077A000032B0CD1436853B10025054E1868F269CC
:1077B00090476068F369056098476560257070BD03
:1077C000680A002010B50A480A4C00230522214609
:1077D000006802F019FA48B9074B217807485B693D
:1077E00098472046BDE81040FFF7D6BF10BD00BF48
:1077F0003C0C0020980A0020680A0020C876010886
:1078000073B50024094E00226946306802F056FB29
:10781000651C30B9064BE1B25B690648984702B077
:1078200070BD6846FFF7B8FF2C46ECE73C0C002023
:10783000680A0020EF760108014B1868704700BF06
:107840003C0C002010B50446064B010AA3F84A0080
:10785000202000F059FCE1B22120BDE8104000F0EA
:1078600053BC00BF1050002008B5FFF7EBFF01220A
:10787000014B83F8522008BD10500020002238B57B
:107880000B4B05461D2083F84E100C4683F84C2008
:1078900000F092FC20F0060040EA4401C9B21D202D
:1078A00000F032FC2946BDE83840232000F02CBC13
:1078B00010500020000000002DE9F74F5E4C1546E7
:1078C000226C8246022A0F461E4600F2A3805B4BC2
:1078D00003EBC203D3E900890120636C9840F9F7F8
:1078E00091FB02460B46404649460DF099FC024684
:1078F0000B46002052490DF093FC804689463FB16B
:1079000049A3D3E900230DF061FB0DF0F9FD3860C8
:10791000B4F84A00F9F776FB00224A4BF9F726FA49
:1079200042464B460DF052FBCDE900013EB13EA36D
:10793000D3E900230DF04AFB0DF0E2FD3060636CEB
:1079400094F84C104FEA830B94F84E000029CBF1C9
:107950001C0202EB001214BF1420002002EBCA0A22
:10796000AAEB0000F9F73EFB94F848200646002AEF
:1079700014BF02200020ABEB00000F46F9F732FBEA
:1079800002460B46304639460DF04AFC0EF080F8B0
:1079900006460F4694F849000430F9F733FB3246A7
:1079A0003B460DF013FB0022002306460F460DF068
:1079B0009DFDA0B30022244B30463946F9F7D6F995
:1079C0004B4642460DF002FB0C9B06460F4643B168
:1079D00015A3D3E900230DF0F9FA0DF091FD0C9BEE
:1079E0001860A5B1DDE9000132463B46F9F7BEF962
:1079F0000DA3D3E900230DF0E9FA0DA3D3E9002389
:107A0000F9F7B4F90EF0CCF80DF07AFD286003B068
:107A1000BDE8F08F4FF000084FF000095CE7002050
:107A20000949CDE7AFF300800000000080842E41BB
:107A30002B8716D9CEF7EF3F10500020B076010803
:107A40000000F03F000011400000204013B5164C2C
:107A50000120A3689847002341F6FE720093009B23
:107A6000934218DDA36802209847002341F6FE7276
:107A70000193019B934212DD0C4BB5211C6C4020FD
:107A8000A047A0214120A04700210120234602B0A9
:107A9000BDE810401847009B01330093DFE7019BCE
:107AA00001330193E5E700BF680A0020247A01084A
:107AB000094B07B51B6CC2213B209847002341F6B8
:107AC000FE720193019B934202DD03B05DF804FB5B
:107AD000019B01330193F5E7247A01088E488F4B0F
:107AE0002DE9F04F03608E4B8E4F83608E4B8F4C91
:107AF00043608F4B85B0C3608E4B8F4D03618F4BBE
:107B0000DFF86CA283618E4BDFF86892C3613B683B
:107B1000984763698B489847002328681A46194696
:107B200002F072F8DFF850B29AF8040068B94FF02A
:107B3000FF33194603AA03F0F5FA68B9666903F042
:107B4000CDF901468048B047EEE741F2883303AAF9
:107B50004FF0FF310020EEE7039BDE0516D500F065
:107B600091FA002000F032FEFB6A9847FFF748FECA
:107B70006369764898470023D9F800001A461946E9
:107B800002F042F8002003F03FF8CDE7980510D549
:107B900000F078FAFFF78CFFFB6A9847FFF730FE9A
:107BA00063696B4898476421D9F8000002F018FA1D
:107BB000BAE7D9F8000002F00FFB012803D163698E
:107BC00064489847B0E7DBF8003023B94FF4977169
:107BD0006148FCF705F8039B190604D507225F4BA3
:107BE0001A70FFF7EFFD039B5A0752D50021286852
:107BF00002F0F6F901284CD1A3690C2098470646FB
:107C000088B963690C215648984733463246314655
:107C1000286801F0F9FF002886D140F241114E4852
:107C2000FBF7DEFF80E7DFF85481A369B8F80400B2
:107C300098470346A0B9B8F8041001906269494812
:107C40009047E26930469047019B28681A461946DA
:107C500001F0DAFF00287FF467AF40F24911DEE758
:107C600008F1040203CA33607060B1601846D8F8A6
:107C70000010B8F804200AF04BFD0322374B1A70AD
:107C80005E60FFF79FFD002328681A46194601F041
:107C9000BBFF039BDB0706D50122304B1A70002285
:107CA0005A60FFF78FFD039BDE0606D505222B4B9E
:107CB0001A7000225A60FFF785FD039B180706D54E
:107CC0000422264B1A7000225A60FFF77BFD039BAB
:107CD000990706D50222214B1A7000225A60FFF73D
:107CE00071FD039B9A0606D506221C4B1A701E4A8C
:107CF0005A60FFF767FD039B5B067FF515AF1B4BD3
:107D00001A78164B32B108221A7000225A60FFF717
:107D100059FD09E70922F7E7480A002071760008B3
:107D2000DD740008247A010891750008680A0020B3
:107D300025760008AD760008440C0020A5750008E3
:107D4000E9750008E9780108FF7801081D79010844
:107D5000457901085C79010872790108980A0020C8
:107D6000B6790108EC790108950A0020940A0020F0
:107D70008C0A0020480C00203C0C0020A00A0020A7
:107D8000044B10B55B6998470446FFF75FFE204639
:107D900010BD00BF247A0108F0B56B4C064625469D
:107DA0000F460FCE0FC596E80F0085E80F0097E845
:107DB00003006369654E013B033388BF644B85B0A4
:107DC00088BF6361636886E80300013B033307D91A
:107DD00060486369984740F27A215F48FBF700FFEB
:107DE0002368013B033307D95C486369984740F235
:107DF0007E215948FBF7F4FEA368013B033307D902
:107E000057486369984740F282215348FBF7E8FEE0
:107E1000E368013B033307D952486369984740F24E
:107E200086214D48FBF7DCFE2369013B033307D96C
:107E30004D486369984740F28A214748FBF7D0FED6
:107E4000E369013B033304D940F28E214248FBF73A
:107E5000C7FEA369013B033304D940F292213E4897
:107E6000FBF7BEFE414B0FCB8DE80F0094E80F00EF
:107E700000F0DEF823689847FFF7E8FD3C4B42200E
:107E80005B6C984722280146636931D1394898478D
:107E900003220021012001F093FE374B18600120DE
:107EA00001F056FF354B186020B940F2AD212A4849
:107EB000FBF796FE012001F04BFF314D286020B901
:107EC00040F2B1212448FBF78BFE4FF0FF312868C8
:107ED00002F086F800220821032001F071FE294BF0
:107EE000186078B963692848984740F2B72103E0E1
:107EF000264898474FF429711748FBF771FE002078
:107F000005B0F0BD224B234A1A6033680BB9042335
:107F10003360214B1D680DB10120F1E701933368F7
:107F2000FA2200931D4901231D4802F081FA01281D
:107F3000F2D063691B489847074840F2C921FBF714
:107F40004FFE2846DCE700BF680A00208C0A0020AC
:107F5000D57400082077010872790108617701085B
:107F600098770108D077010809780108780A00207D
:107F7000247A010845780108440C0020400C0020B8
:107F8000480C00203C0C0020777801085C78010840
:107F9000880A0020CF7400084C0C0020AB78010840
:107FA000DD7A0008B378010870B5084C05462268F0
:107FB0000E4622B940F2D9210548FBF711FE23688D
:107FC00031462846BDE87040184700BF880A0020A7
:107FD0007279010800F046B8034B0344034883421A
:107FE0008CBF0020012070470071BDCCFF6789095C
:107FF0000120704708B5FFF777FB4379002B0CBFD2
:108000008020002008BD0000002310B5074951F86A
:108010003340DA00844203D80A449468844203D887
:108020000133152BF3D1FEE7107910BD907A0108CA
:1080300084B030B503AC84E80F00064C03AD0FCD1F
:108040000FC495E80F0084E80F00BDE8304004B08D
:10805000704700BFF00D0020014B1878704700BF3B
:1080600010500020642307B50093002304481A46EB
:108070000321006803F030FA03B05DF804FB00BF91
:10808000580C002013B5104C0120A368984700231A
:108090000093009BB3F5CC7F0FDDA36800209847C9
:1080A000002342F6FE720193019B934208DD0220F9
:1080B000A36802B0BDE810401847009B0133E7E712
:1080C000019B01330193EFE7F00D00202DE9F04112
:1080D00007460C4C0D46E368002016469847236976
:1080E00047F080009847013D2E44B54204D1E36833
:1080F0000120BDE8F0411847236915F8010F9847A2
:10810000F3E700BFF00D002007B502AB03F8011D37
:1081100001221946FFF7DAFF03B05DF804FB000007
:10812000134A10B55060134A904219D0F8F75AFF1D
:108130000DA3D3E900230DF073F80DF0E1F9044627
:10814000C4F307410620FFF7DFFFC4F30721072030
:10815000FFF7DAFFE1B20820BDE81040FFF7D4BF17
:10816000054CEDE7AFF300800000000080844E4036
:1081700010500020F01FCB33CD3CD9002DE9F04149
:1081800007460C4C0D46E3680020164698472369C5
:1081900007F07F009847013D2E44B54204D1E368C3
:1081A0000120BDE8F041184723690020984705F8F1
:1081B000010FF2E7F00D002007B501220DF10701D4
:1081C000FFF7DCFF9DF8070003B05DF804FB00003B
:1081D00001282DE9F84F884603D0022852D000200C
:1081E00049E06B4C2720A58BFFF7E6FF20F0F80055
:1081F00001302844F8F706FFA37F0022002B3CD172
:10820000644BF8F7B3FD064630200F46FFF7D4FF66
:1082100030F0F9030CBF00235E4B00223046394694
:10822000F8F7A4FD064640460F46F8F7EBFE024677
:108230000B4630463946F8F799FD94F82030002275
:10824000EBB90023F8F792FD0022534B0CF0BEFE71
:108250000646A0690F46F8F7C5FE02460B463046B3
:1082600039460CF0DDFF00224C4B0CF0AFFE0DF058
:108270001BFD0DF045F9BDE8F88F0023C1E74FF075
:108280008043DFE7424C226C022A76D8444B03EB52
:10829000C203D3E900670120656CA840F8F7B2FE7D
:1082A00002460B46304639460CF0BAFF02460B46F2
:1082B000002038490CF0B4FF06460F46B4F84A00D7
:1082C000F8F7A0FE0022374BF8F750FD32463B4648
:1082D0000CF07CFE94F84C30AD00824694F84E00D1
:1082E000002B8B46C5F11C0101EB001114BF1420BB
:1082F000002001EBC801081AF8F774FE94F8483022
:108300008046002B14BF02200020281A8946F8F767
:1083100069FE02460B46404649460CF081FF0DF0CF
:10832000B7FB8046894694F849000430F8F76AFEA6
:1083300042464B460CF04AFE0022002304460D46FE
:108340000DF0D4F8E0B10022134B20462946F8F78F
:108350000DFD32463B460CF039FE52465B46F8F7BF
:1083600005FD00220D4B0CF031FE07A3D3E90023DD
:10837000F8F7FCFC0DF014FC7BE7002600278AE7E9
:1083800000200549E5E700BF2B8716D9CEF7EF3F60
:10839000105000200000F03F0000204000408F40BF
:1083A000787A010800001140012808B504D002289D
:1083B0000AD04FF0FF3006E01120FFF7FDFEC0F3BA
:1083C0004700404200B208BD1B20FFF7F5FE8B3886
:1083D000F8E700000B4B10B55B68044660B902205B
:1083E00098470120FFF7E8FE00F0F8012143012043
:1083F000BDE81040FFF788BE03280CBF0120002015
:10840000EEE700BFF00D002013B5642400230F48F1
:1084100000941A460321006803F05EF800230C481C
:1084200000941A460321006803F056F80023094817
:1084300000941A460321006803F04EF80020FFF76D
:10844000C9FF0022044B1A7002B010BD580C002066
:10845000EC0D0020540C00201050002013B56424B3
:1084600000230F4800941A460321006803F034F8F3
:1084700000230C4800941A460321006803F02CF8EE
:108480000023094800941A460321006803F024F8E9
:108490000120FFF79FFF0022044B1A7002B010BDAD
:1084A000580C0020EC0D0020540C0020105000202F
:1084B00007B50022144B8DF807201A87DA869A85B3
:1084C00083F82E2093F8223023B903B05DF804EB33
:1084D000FFF79ABF3F20FFF76FFE8DF807009DF86A
:1084E0000730DB0603D510213F20FFF70DFE0D20DE
:1084F000FFF762FE40F040010D20C9B203B05DF805
:1085000004EBFFF701BE00BF10500020044B1A8897
:1085100040F201139A4201D1FFF7CABF704700BF72
:1085200010500020F7B5604C06466378012B03D04D
:10853000022B6AD0002730E0402094F82270FFF729
:108540003BFE0C214020FFF7DFFD4120FFF734FE0A
:1085500060F00E01C9B24120FFF7D6FD3520FFF7CC
:108560002BFE00F0C00141F01F013520FFF7CCFDCC
:108570003520FFF721FE00F03F0084F83A000D207F
:10858000FFF71AFE00F0400141F0B9010D20FFF79E
:10859000BBFD0023A3852387E38600214FF4C87227
:1085A00042480AF0D9F801232370414B4FF0FF31C4
:1085B0001868002E6AD04FF47A7505FB06F2009118
:1085C0000023B2FBF5F2042102F086FF6478012C4F
:1085D00061D10520FFF7FEFE0D20FFF7EDFD40F015
:1085E0002001C9B20D20FFF78FFD67B1314B1D6827
:1085F00002F040F94FF0FF3302460093214600237A
:10860000284602F069FF03B0F0BD94F851303320E2
:108610002BB3FFF7D1FD40F04101C9B23320FFF782
:1086200073FD19213B20FFF76FFD94F84F3094F84C
:108630005270FBB11D211120FFF766FD4020FFF7AE
:10864000BBFD00F033014020FFF75EFD00210F204D
:10865000FFF75AFD00210D20FFF756FD9DE7FFF7BC
:10866000ABFD00F0BE0141F001013320FFF74CFDEE
:108670001D21D7E70F211120FFF746FD4020FFF70E
:108680009BFD00F03C0141F00101DCE70091334625
:108690003246032198E72FB1052003B0BDE8F04032
:1086A000FFF798BE0620F8E7105000205C0C002071
:1086B000580C0020540C002037B54FF47A72642314
:1086C00050432C4D2C4C0093B0FBF2F200230421BC
:1086D000286802F001FF6378012B14D0022B2CD004
:1086E000022323702C6802F0C5F80523024600938C
:1086F00001210023204602F0EFFE032003B0BDE875
:108700003040FFF767BE4020FFF756FD00F0030141
:1087100041F010014020FFF7F7FC4120FFF74CFD2E
:1087200000F03E014120FFF7EFFC3520FFF744FD4C
:1087300000F03F0084F83A00D2E794F84F3073B16C
:10874000F5211120FFF7E0FC4020FFF735FD00F098
:10875000330141F040014020FFF7D6FCC0E7F7218C
:108760001120FFF7D1FC4020FFF726FD00F03F016C
:10877000EFE700BFEC0D00201050002010B5114CA9
:108780006378012B04D0022B09D040F2E53101E0DF
:1087900040F2CE31BDE810400B48FBF721BAFA2178
:1087A0001120FFF7B1FC4020FFF706FD00F0FC01AF
:1087B0004020FFF7A9FC032307202370BDE81040E9
:1087C000FFF708BE10500020497B010808B51A4B7E
:1087D0005A7882422ED0022858704FF0000013D0F1
:1087E000FFF7F8FD0120FFF7E7FC00F07F01012013
:1087F000FFF78AFC00214020FFF786FC3021412052
:10880000BDE80840FFF780BCFFF7E4FD0120FFF75B
:10881000D3FC60F07F01C9B20120FFF775FC002195
:108820004020FFF771FC00214120FFF76DFC432140
:108830003120E5E708BD00BF10500020254B13B5DF
:1088400018600023244C1A4600944FF47A71234890
:1088500002F020FE224B186018B9FF212148FBF7D7
:10886000BFF9002300941A464FF47A711E4802F0B3
:1088700011FE1E4B186020B940F201111948FBF798
:10888000AFF91B4B012200934FF4FA610023194802
:1088900002F000FE184B186020B940F20311114895
:1088A000FBF79EF9FFF7EEFB0020FFF78FFF00209C
:1088B000FFF790FD4FF4C8720021104809F04CFFFB
:1088C000002201210E4B83F8282083F829101A700A
:1088D00002B010BD500C0020B58E0008407B01088E
:1088E000EC0D0020497B0108437B0108580C002057
:1088F0000D850008467B0108540C00205C0C00200C
:108900001050002073B50E4614460546FFF75EFF73
:108910003046FFF705FC0520FFF75CFD00230193BF
:10892000019BB3F5CC7F0BDD2846FFF73DFD0546E7
:10893000FFF76AFDA542CCBF0020012002B070BD48
:10894000019B0133EBE773B500240220FFF73EFFE4
:10895000FF211120FFF7D8FB0520FFF73BFD25463F
:1089600026460196019BB3F5CC7F0DDD2C20FFF749
:1089700023FC00F00100A0400134202C45EA000552
:10898000EFD1284602B070BD019B01330193E9E7A6
:108990002DE9F04F824687B00093109B0C4601935F
:1089A0009DF85C309DF85810029393469DF8643012
:1089B0009DF8602003930492BDF84450BDF84890A0
:1089C0009DF84C609DF850709DF854800591FFF71C
:1089D000FDFEDDE90332BAF1010F06D0BAF1020F54
:1089E00005996DD007B0BDE8F08FDFF810920199BE
:1089F000C9F818B089F8212089F822305846C9F8FA
:108A00001040C9F8141089F81E6089F81F7089F8A1
:108A10002080A9F81C50F8F7E5FA0B46024674A12D
:108A2000D1E900010CF0FCFB0CF06AFD1FFA80FBA1
:108A30004FEA1B210220FFF767FB5FFA8BF103204F
:108A4000FFF762FB2046FFF7DFFA01461220FFF72F
:108A50005BFB0198FFF7D8FA01461320FFF754FBA0
:108A6000290A2520FFF750FBE9B22620FFF74CFB2F
:108A7000B9F81E30012B20D0002340F297115E4838
:108A800089F82930FBF7ACF839463220FFF73CFB78
:108A90003020FFF791FB002E14BF00216FF07F0103
:108AA00000F06F0040EA0818302041EA0801C9B21E
:108AB00007B0BDE8F04FFFF727BB89F82930E3E79F
:108AC0004E489DF800C080F84F109DF80810BBF18B
:108AD0000C0FC0E9104B80F849C0A0F84A5080F84C
:108AE0004C6080F84D7080F84E8080F8501080F80F
:108AF000512080F85230824673D8BBF1050F61D9FE
:108B000024B9ABF10B03012B5ED804E0012C5BD13F
:108B1000BBF10C0F58D101231D208AF84830FFF714
:108B20004BFB9AF84810009B41EA480141EA860154
:108B300041EAC30141EA8411C9B21D20FFF7E4FAFA
:108B40001E20FFF739FBC9F3012100F00C0001439F
:108B500041EA0B11C9B21E20FFF7D6FA5FFA89F17C
:108B60001F20FFF7D1FA290A2020FFF7CDFAE9B23A
:108B70002120FFF7C9FA1EB139462220FFF7C4FAB7
:108B80009AF84F306BB14B20FFF716FB60F07F0176
:108B9000C9B24B20FFF7B8FA9AF850102420FFF71B
:108BA000B3FABBF1060F4FF031000FD1FFF704FB12
:108BB00000F0F80141F005013120FFF7A5FA0C2182
:108BC000372075E74FF0060B0023A5E7FFF7F4FA0F
:108BD00000F0F80141F003013120FFF795FA0A2176
:108BE000EEE74FF00C0B012C8EE700BFAFF30080D7
:108BF0000000000080847E41497B01081050002065
:108C00002DE9F04F89B01E469DF84C300791019335
:108C10009DF85C30009202939DF860308346059386
:108C20009DF86430129D03931A9BBDF85070049315
:108C30009DF854809DF85890FFF7C8FD0920FFF774
:108C4000BBFA04465A20FFF7B7FA994A82465068A1
:108C50000692FFF7CFF904F07F04204340B2069A52
:108C60000028144620F00F00079933DA1129CBBFF2
:108C70004AF007030AF0F8035FFA83FA43F0040AA4
:108C80000AF00702072A40B21BD11429A8BF1421F9
:108C900005290A46B8BF0522511F0843C1B2092061
:108CA0000692FFF731FA51465A20FFF72DFABBF131
:108CB000010F069A17D0BBF1020F6AD009B0BDE8C8
:108CC000F08F1129A8BF112102290A46B8BF02223C
:108CD000911EE2E70E29A8BF0E2141EAE172511C64
:108CE0000143C9B2DBE7009B2272C4E903369DF859
:108CF0000C3084F8209084F82130049BA5616362D5
:108D0000A78384F81E800098F8F76CF964A3D3E970
:108D100000230CF085FA0CF0F3FB84B2210A042046
:108D2000FFF7F2F9E1B20520FFF7EEF92846F8F770
:108D300059F902460B465CA1D1E900010CF070FA2A
:108D40000CF0DEFB84B2210A0220FFF7DDF9E1B26C
:108D50000320FFF7D9F9390A2520FFF7D5F9F9B231
:108D60002620FFF7D1F93020FFF726FAB8F1000FDF
:108D70000CBF6FF07F01002100F06F0040EA09197D
:108D8000302041EA0901C9B209B0BDE8F04FFFF750
:108D9000BBB9474B0C2D83F83C209DF80420C3E958
:108DA000106583F849209DF80820A3F84A7083F8DD
:108DB0004F209DF8142083F84C8083F850209DF8B4
:108DC0000C2083F84E9083F85120049A9A465A65F5
:108DD00061D8052D51D926B9A5F10B03012B4DD82A
:108DE00003E0012E4AD10C2D48D101238AF84830E6
:108DF000029B6BB14B20FFF7DFF960F07F01C9B236
:108E00004B20FFF781F99AF850102420FFF77CF9E6
:108E10001D20FFF7D1F994F84810019B41EA490160
:108E200041EA880141EAC30141EA8611C9B21D2025
:108E3000FFF76AF91E20FFF7BFF900F00F0141EAC2
:108E40000511C9B21E20FFF75FF9390A2020FFF78C
:108E50005BF92120F9B2FFF757F9062D4FF03100E9
:108E60000ED1FFF7A9F900F0F80141F0050131201A
:108E7000FFF74AF90C21372086E706250023B5E7DE
:108E8000FFF79AF900F0F80141F003013120FFF7F4
:108E90003BF90A21EFE70C25012EA0E7AFF3008094
:108EA0000000000080844E400000000080847E416D
:108EB0001050002010B5214C2378012B02D0022B3A
:108EC0002FD010BD6378012B24D100230B213E202D
:108ED000A3852387E386FFF717F910213F20FFF7CB
:108EE00013F994F822309BB10D20FFF765F940F09B
:108EF0002001C9B20D20FFF707F9114B1B68002BA9
:108F0000DFD0DB68002BDCD0BDE810400020184724
:108F10002370F2E794F85230002BEED0FFF79EFA60
:108F2000EBE700232370064B1B68002BC9D05B685E
:108F3000002BC6D0BDE81040184700BF10500020DD
:108F4000500C00202DE9F04107460D4C0D46E3681A
:108F5000002016469847236907F07F009847013D97
:108F60002E44B54204D1E3680120BDE8F041184722
:108F7000236900209847C04305F8010FF1E700BFBF
:108F8000F00D00200A4601460020FFF79FB80000C0
:108F9000F7B5374C064663780D46012B03D0022BFC
:108FA00027D0002017E000232387A37FE18613B199
:108FB0003220FFF7A9F86B1E3F2B11D884F83B50E5
:108FC000304694F83B10FFF7DDFF228F94F83B30DA
:108FD000606A1344238703B0BDE8F040FFF76CBB21
:108FE0002A463146234809F093FB202384F83B307E
:108FF000E6E794F85130332023B3FFF7DDF800F0B3
:10900000BE013320FFF780F819213B20FFF77CF8E1
:109010002946222084F85C50FFF776F800210E20C4
:10902000FFF772F800210D20FFF76EF80120FFF71F
:10903000C3F830F0F80710D030462946FFF7A2FFFA
:10904000606DC8E7FFF7B8F800F0BE0141F001011C
:109050003320FFF759F81D21D7E7FFF7FFF90197F4
:10906000019BB3F5CC7FE7DC019B01330193F7E76C
:10907000105000205C0C00200A4601460020FFF73B
:109080007DB80A4601460020FFF75CBF38B50546AB
:109090000C46FFF79BFB012D02D0022D0AD038BDF4
:1090A000064B9B7F002BFAD121463220BDE8384089
:1090B000FFF72AB821462320F8E700BF1050002010
:1090C0007FB50022614C8DF80B2023780392012B91
:1090D000254604D0022B00F0988004B070BD637860
:1090E000012B32D0022BF8D140211220FFF70CF8CF
:1090F0001220FFF761F88DF80B009DF80B30544EED
:1091000013F0200F27D020211220FEF7FDFF94F846
:10911000523003B9237000224E48009203AB08215D
:10912000006802F0D9F9039B3BB14FF080524A4BE3
:109130001A60BFF34F8FBFF36F8F3368002BCCD013
:109140001B69002BC9D09847C7E740F2EE4143485E
:10915000FAF746FDC1E71920FFF72EF840B20028C4
:1091600084F85800BFBF40428010404244B2A8BFBC
:1091700084101A20FFF720F8002C40F30B139BB249
:10918000B5BF00198B38A0F18B04C018B4BFE41828
:10919000A5F85A004FF01300B8BFA5F85A40FFF7E2
:1091A0000BF885F85C001020FFF706F801460D204B
:1091B000FEF7AAFF95F85C102948FFF75DFF95F8C8
:1091C00052208AB923482A70009203AB0821006814
:1091D00002F082F9039B3BB14FF080521E4B1A60A4
:1091E000BFF34F8FBFF36F8F3368002B3FF475AF22
:1091F0009C68002C3FF471AF95F95830B5F95A20AE
:1092000095F85C101648A04767E71648009203AB34
:109210000821006802F060F9039B3BB14FF08052D7
:109220000D4B1A60BFF34F8FBFF36F8F6B78022B1C
:1092300003D108211220FEF767FF00232B70044B97
:109240001B68002B3FF449AF1B687AE710500020E1
:10925000500C0020580C002004ED00E0497B010870
:109260005C0C0020EC0D0020002230B5544D85B080
:109270002B780392012B8DF80B202C4604D0022B67
:1092800000F0848005B030BD6B78012B22D0022B1A
:10929000F8D14C48009203AB0821006802F01CF999
:1092A000039B3BB14FF08052474B1A60BFF34F8F87
:1092B000BFF36F8F80211220FEF726FF002323705B
:1092C000424B1B68002BDDD0DB68002BDAD001207D
:1092D0009847D7E73F20FEF76FFF8DF80B009DF80A
:1092E0000B309B06CED595F8293023B940F28E512C
:1092F0003748FAF775FC238F364894F83A1018442B
:1093000094F82830022B17D1FFF7BBFE238FB3B19F
:10931000228F94F83A30E18E13449BB28B4223871C
:10932000B0D32A4B1B68BBB19D68ADB1002394F943
:109330002E202848A8470FE0FFF79EFEE6E794F8A6
:109340002D304BB194F83A102248FEF72DFEE086FE
:109350000138B0F5C77FDBD9FFF7AAF81E4B1C68B0
:1093600001F08EFA002302460093072103AB20464A
:1093700002F0B2F8039B002B84D04FF08052124BC6
:109380001A60BFF34F8FBFF36F8F7BE76B78012BB2
:109390007FF478AF2A8FEB8E95F83B100D489B1A1F
:1093A0008B42104407DDFFF7EDFD95F83B302A8F27
:1093B00013442B8766E7D9B2FFF7E4FDEB8EF8E79D
:1093C00010500020580C002004ED00E0500C00204C
:1093D000497B01085C0C0020540C002010B5184C8F
:1093E0002378012B02D0022B28D010BD61780129EF
:1093F00018D00229F9D194F84F30002BF5D0122063
:10940000FEF782FE0F4B1B68002BEED05C69002C30
:10941000EBD01C20FEF7D0FE2346BDE8104000F044
:109420003F00184700231120238784F82D10FEF7F2
:10943000C3FE4008404284F82E00D6E76178D8E7A2
:1094400010500020500C00201F4B70B55A78022A93
:1094500004D11B78012B02D0032B13D070BD122036
:10946000FEF7AAFEC306F9D510211220FEF74CFE26
:10947000164B1B68002BF1D0DB69002BEED0BDE84A
:10948000704018471220FEF797FE10F001050F4CB0
:109490000DD005211220FEF737FE2368002BDDD00A
:1094A0009B69002BDAD00120BDE8704018470421E9
:1094B0001220FEF729FE2368002BCFD09B69002BDA
:1094C000CCD02846F0E700BF10500020500C002000
:1094D000074B5A78012A0AD11A78012A07D183F852
:1094E0002C20002202213E201A87FEF70DBE704775
:1094F0001050002070474FF0FF3200F10803436026
:10950000C0E9022303610023036070470023036165
:10951000704743689A684B608A609A6851609960A6
:10952000036808610133036070470A6830B5531C53
:109530000AD103695A684A6091608B605960036878
:1095400008610133036030BD00F108035C682568E1
:109550009542EFD82346F9E70369D0E901128A6002
:10956000826851605968814208BF5A6000220261D6
:109570001A68013A1A6018687047000006480068C7
:10958000006880F3088862B661B6BFF34F8FBFF3FF
:109590006F8F00DF00BF000008ED00E0002307B57B
:1095A00001930B4B1B68013303D0CA210948FAF71A
:1095B00017FB4FF0500383F31188BFF36F8FBFF396
:1095C0004F8F019B002BFCD003B05DF804FB00BF64
:1095D00080000020967B01084FF0807340F8043C27
:1095E000054B21F0010140F8081C40F80C3C40F804
:1095F000202C4038704700BF9D95000800000000F7
:10960000074B19680868B0E8F00F80F30988BFF3CA
:109610006F8F4FF0000080F311884EF00D0E7047F1
:10962000304A00204FF0500383F31188BFF36F8F4F
:10963000BFF34F8F084A13680133012B136009D120
:10964000064B1B6813F0FF0F04D040F2751104485D
:10965000FAF7C6BA704700BF8000002004ED00E0B2
:10966000967B010810B5074C236823B94FF4BE71EF
:109670000548FAF7B5FA2368013B23600BB983F379
:10968000118810BD80000020967B010800000000BA
:10969000EFF30980BFF36F8F0D4B1A6820E9F00FCD
:1096A00010602DE908404FF0500080F3118801F060
:1096B00059FA4FF0000080F31188BDE8084019689E
:1096C0000868B0E8F00F80F30988BFF36F8F704728
:1096D000304A002008B54FF0500383F31188BFF3E0
:1096E0006F8FBFF34F8F01F0D3F818B14FF0805256
:1096F000024B1A60002383F3118808BD04ED00E0DB
:109700000022054B05491A600A6041F26701044ACC
:10971000116007221A60704710E000E018E000E0D6
:1097200014E000E013B5264B264C1A78D2B2019211
:10973000FF221A701B78244ADBB28DF803309DF8A3
:10974000033003F0500313700723002223609DF8B9
:109750000310581E090629D402B123602368032B85
:1097600004D04FF49B711948FAF73AFA2368144A67
:109770001B0203F4E06323600024019BDBB213703F
:10978000134B1A6842F470021A601A6842F0704271
:109790001A60FFF7B5FF0F4B1C60FFF7EFFE01F0FB
:1097A000E1F9FFF7FBFE204602B010BD9DF8033043
:1097B00001225B00DBB28DF803300346C7E700BF30
:1097C00000E400E0140E0020100E0020967B01083B
:1097D00020ED00E08000002008B5EFF305830F2B9B
:1097E0000AD90D4A9B5C0D4A12789A4204D940F27C
:1097F000A5210B48FAF7F4F90A4B0B4A1B681268CB
:1098000003F4E063934206D9BDE8084040F2B52175
:109810000348FAF7E5B908BDF0E300E0100E0020B8
:10982000967B01080CED00E0140E002010B50F4BE4
:109830001A68824218D35C681919884201BF4168CE
:10984000184609195960446801198A4207D1084924
:1098500009688A421FBF516812680919416098421D
:10986000026018BF186010BD1346E1E7284A0020C7
:10987000180E002038B5064B064D1C68246804B944
:1098800038BD6307FAD077212846FAF7A9F9F5E73A
:10989000284A0020EE7B01082DE9F843074600F036
:1098A000E1FF3F493F4D0B680BBB3F4A3F4E50071E
:1098B0001DBFD01D20F0070002F570534FF4705308
:1098C0001CBF02461B1A00201344083B23F0070369
:1098D00070603260C3E90000981A0B60C2E9003082
:1098E000334B1860334B18604FF000432B602B68EC
:1098F0001F4252D1002F41D007F1080462071CBF5C
:1099000024F007040834002C47D02A4B1A689846E4
:10991000A24242D3254B1E687268A24202D230682E
:10992000002837D10968B14237D01F683168121B4F
:10993000102A07F10807196010D906EB040919F07D
:10994000070F03D0D5211C48FAF74AF97368484637
:109950001B1BC9F804307460FFF768FF1449726874
:10996000D8F8003008689B1A8342C8F8003038BF26
:109970000B602B68134373600023336001F018F809
:109980007B0704D040F215110B48FAF729F9384645
:10999000BDE8F88333460646BEE70027EEE700BF82
:1099A000180E00201C4A00201C0E0020284A00200F
:1099B000244A0020204A0020EE7B010838B50446E6
:1099C00070B3184D50F8041C2A68114204D140F2BB
:1099D00029111548FAF704F954F8083C23B14FF45B
:1099E00095711148FAF7FCF854F8043C2A681342C0
:1099F00016D054F8081C99B923EA020344F8043C31
:109A000000F030FF094A54F8043C1168A4F1080042
:109A10000B441360FFF70AFFBDE8384000F0C8BFF1
:109A200038BD00BF1C4A0020EE7B0108204A002000
:109A300010B50446FFF7F6FDA46BFFF713FEB4FA6A
:109A400084F0400910BD70B51546026C0446866B63
:109A500042B905689DB9806801F0B8FAA560013681
:109A6000A66370BD6DB9406808F052FE6368226C51
:109A70001344A2686360934201D3236863600020AB
:109A8000EDE7C06808F044FE236CE2685B422168A1
:109A90001A448A42E2603EBFA2689B18E360022D2E
:109AA000EDD10EB1013EEAE73046D8E703461A6C25
:109AB00010B4084662B1D9689C681144A142D960CB
:109AC00028BF196810BC28BFD960D96808F020BE2B
:109AD00010BC704770B50446FFF7A4FD94F84550DC
:109AE00004F124066DB2002D14DCFF2384F8453008
:109AF000FFF7B8FDFFF796FD94F8445004F1100607
:109B00006DB2002D12DCFF2384F84430BDE87040B4
:109B1000FFF7A8BD636A002BE7D0304601F018F9C3
:109B200008B101F097F9013D6DB2DCE72369002B24
:109B3000E9D0304601F00CF908B101F08BF9013D94
:109B40006DB2DEE738B50D46044620B940F2031188
:109B50001948FAF745F8FFF765FDD4E90F314B4393
:109B60002268D0185B1A1344A060E3600020FF2332
:109B7000A063626084F8443084F8453095B9236965
:109B800063B104F1100001F0E3F838B14FF08052F6
:109B90000A4B1A60BFF34F8FBFF36F8FFFF762FD61
:109BA000012038BD04F11000FFF7A5FC04F12400EA
:109BB000FFF7A1FCF2E700BF447C010804ED00E0E0
:109BC000F8B50D461746064620B94FF4BB710D484F
:109BD000FAF706F805FB06F05030FFF75DFE044685
:109BE00048B155B92060C4E90F6501212046FFF74F
:109BF000A9FF84F84C702046F8BD00F150030360C3
:109C0000F1E700BF447C01082DE9FF478846019237
:109C10001E46044620B940F2F1214B48F9F7E0FF17
:109C2000B8F1000F06D1236C23B140F2F22146486F
:109C3000F9F7D6FF022E07D1E36B012B04D040F2D7
:109C4000F3214148F9F7CCFF01F05EF930B9019BEF
:109C500023B140F2F6213C48F9F7C2FF0027B9468C
:109C6000DFF8E8A0FFF7DEFCA26BE36B9A4201D3BA
:109C7000022E19D1324641462046FFF7E4FE636AC0
:109C80001BB104F1240001F063F838B14FF08052A9
:109C90002E4B1A60BFF34F8FBFF36F8FFFF7E2FCBD
:109CA000012004B0BDE8F087019D1DB9FFF7DAFC83
:109CB0000020F6E717B902A801F08AF8FFF7D2FCF6
:109CC00000F0D0FDFFF7AEFC94F84430FF2B08BF46
:109CD00084F8449094F84530FF2B08BF84F84590F1
:109CE000FFF7C0FC01A902A801F07EF828BBFFF72E
:109CF00099FCA26BE36B9A420ED1FFF7B3FC01997A
:109D000004F1100000F0EAFF2046FFF7E3FE00F048
:109D10004FFE48B10127A5E7FFF7A4FC2046FFF757
:109D2000D9FE00F045FEF5E74FF08053CAF8003049
:109D3000BFF34F8FBFF36F8FECE72046FFF7CAFEEC
:109D400000F036FEB4E700BF447C010804ED00E0FB
:109D500010B5024600210120FFF732FF044638B15A
:109D6000002383600360C3601A461946FFF74CFF67
:109D7000204610BD2DE9F843894690461F4604460B
:109D800020B940F2C3312748F9F72AFFB9F1000F93
:109D900006D1236C23B14FF471712248F9F720FFEB
:109DA000022F07D1E36B012B04D040F2C5311D48CF
:109DB000F9F716FFFFF710FDEFF311864FF0500390
:109DC00083F31188BFF36F8FBFF34F8FA26BE36BE9
:109DD0009A4201D3022F22D194F845503A466DB2EF
:109DE00049462046FFF72FFE6B1C13D1636A0BB95F
:109DF00001200BE004F1240000F0AAFF0028F7D0B6
:109E0000B8F1000FF4D00120C8F8000086F31188E3
:109E1000BDE8F88301356DB284F84550E8E70020CD
:109E2000F4E700BF447C010870B50D46044620B934
:109E30004FF48C612048F9F7D3FE236C23B140F234
:109E400064411D48F9F7CCFE236833B9A36823B1F8
:109E500040F269411848F9F7C3FEFFF7BDFCEFF384
:109E600011864FF0500383F31188BFF36F8FBFF358
:109E70004F8FA26BE36B93421CD994F845300132AB
:109E80005BB2A2635A1C10D1636A0BB9012009E0CE
:109E900004F1240000F05CFF0028F7D0002DF5D07D
:109EA0000120286086F3118870BD01335BB284F80D
:109EB0004530EBE70020F5E7447C01082DE9F0434D
:109EC00085B00F460192044620B94FF4A061424884
:109ED000F9F786FE37B9236C23B140F204513E48AE
:109EE000F9F77EFE01F010F830B9019B23B140F282
:109EF00009513948F9F774FE0026B046DFF8DC90C6
:109F0000FFF790FBA56BD5B139462046013DFFF721
:109F1000CDFDA563236963B104F1100000F018FFC3
:109F200038B14FF080522D4B1A60BFF34F8FBFF303
:109F30006F8FFFF797FB012005B0BDE8F083019D0F
:109F40001DB9FFF78FFB0020F6E716B902A800F055
:109F50003FFFFFF787FB00F085FCFFF763FB94F8FA
:109F60004430FF2B08BF84F8448094F84530FF2B21
:109F700008BF84F84580FFF775FB01A902A800F02F
:109F800033FFF0B92046FFF753FDA0B1019904F16A
:109F9000240000F0A3FE2046FFF79CFD00F008FD22
:109FA00038B94FF08053C9F80030BFF34F8FBFF37B
:109FB0006F8F0126A4E72046FFF78CFD00F0F8FC28
:109FC000F7E72046FFF786FD00F0F2FC2046FFF79A
:109FD0002FFD0028EDD0B6E7447C010804ED00E039
:109FE0002DE9FF410446019120B940F291515248B8
:109FF000F9F7F6FD236C23B140F295514E48F9F77D
:10A00000EFFD00F081FF30B9019B23B140F29A517E
:10A010004948F9F7E5FD00252F462E46DFF81C815B
:10A02000FFF700FBA36BE3B1013BA363236813B904
:10A0300001F06CF8A060236963B104F1100000F036
:10A0400087FE38B14FF080523C4B1A60BFF34F8F00
:10A05000BFF36F8FFFF706FB0125284604B0BDE86C
:10A06000F081019B4BB925B140F2E1513248F9F73B
:10A07000B7FDFFF7F7FA0025EFE717B902A800F0E0
:10A08000A7FEFFF7EFFA00F0EDFBFFF7CBFA94F82D
:10A090004430FF2B08BF84F8446094F84530FF2B10
:10A0A00008BF84F84560FFF7DDFA01A902A800F0B7
:10A0B0009BFE40BB2046FFF7BBFCF0B123683BB9D9
:10A0C000FFF7B0FAA06800F02FFF0546FFF7CAFAC5
:10A0D000019904F1240000F001FE2046FFF7FAFC8C
:10A0E00000F066FC38B94FF08053C8F80030BFF379
:10A0F0004F8FBFF36F8F012792E72046FFF7EAFCEF
:10A1000000F056FCF7E72046FFF7E4FC00F050FCB7
:10A110002046FFF78DFC0028EDD0002D9DD0FFF7E5
:10A1200081FA616A19B1236B1968C1F10501A06850
:10A1300000F098FF9DE700BF447C010804ED00E0BB
:10A140002DE9F84389469046054620B940F2FB6167
:10A150002048F9F745FDB9F1000F06D12B6C23B16A
:10A1600040F2FC611B48F9F73BFDFFF735FBEFF3CD
:10A1700011874FF0500383F31188BFF36F8FBFF344
:10A180004F8FAC6B1CB395F84460494676B22846B5
:10A19000FFF78CFC013C731CAC6313D12B690BB92A
:10A1A00001200BE005F1100000F0D2FD0028F7D0EF
:10A1B000B8F1000FF4D00120C8F8000087F311882F
:10A1C000BDE8F883013676B285F84460E8E72046BA
:10A1D000F4E700BF447C010810B5044620B940F202
:10A1E0008A710548F9F7FCFCFFF71CFAA46BFFF72E
:10A1F00039FA204610BD00BF447C010838B5054639
:10A2000020B940F2A4710648F9F7EAFCFFF70AFA10
:10A21000A86BEC6B241AFFF725FA204638BD00BF67
:10A22000447C0108002330B5064A52F8335002EB53
:10A23000C3041DB942F83310606030BD0133052BF3
:10A24000F3D1FAE770500020002310B5074A02EB63
:10A25000C3014C68844204D1002042F833004860B6
:10A2600010BD0133052BF2D1FAE700BF705000207A
:10A2700010B5044620B94FF4F8610548F9F7B0FC71
:10A280002046FFF7E1FF2046BDE81040FFF796BBF0
:10A29000447C010870B504460D461646FFF7C2F926
:10A2A00094F84430FF2B04BF002384F8443094F822
:10A2B0004530FF2B04BF002384F84530FFF7D2F967
:10A2C000A36B2BB93246294604F1240000F020FD8F
:10A2D0002046BDE87040FFF7FDBB0000064A13684A
:10A2E0001968064B19B94FF0FF321A6070471268AF
:10A2F000D268D2685268F8E7344A0020E44A002065
:10A3000010B5044620B940F2F2610848F9F768FC3C
:10A310006269074B9A4207D1A06A064B984203D064
:10A32000B0FA80F0400910BD0020FCE7887C0108ED
:10A33000044B0020EC4A0020F8B51B4B1B4E1C6858
:10A34000054630680F460430FFF706F9334640B93A
:10A3500001203168164EC96A3268884022EA00023C
:10A3600032606A1C07D137B1196812480431BDE860
:10A37000F840FFF7CEB81A686419546007D30E4A44
:10A3800010681968BDE8F8400431FFF7CEB80B4AF1
:10A39000106819680431FFF7C8F8094B1A68A2421F
:10A3A00088BF1C60F8BD00BF2C4B0020304A002045
:10A3B000B44A0020044B0020384A0020344A0020D0
:10A3C000E44A002080B5DFF86480144F144C154E29
:10A3D000236863B9144B1B68012BF8D94FF08053E5
:10A3E000C8F80030BFF34F8FBFF36F8FEEE7FFF772
:10A3F00019F9FB68DD68281DFFF7AEF83368013BEB
:10A4000033602368013B2360FFF72CF9286BFFF7CB
:10A41000D5FA2846FFF7D2FADAE700BF184B00203A
:10A42000A44A0020A04A00203C4A002004ED00E09D
:10A430002DE9F84F4FEA820A804650460D4699466C
:10A440000B9EFFF729FA0746002800F0AB805C203E
:10A45000FFF722FA0446002800F0A180076325B91F
:10A460004FF458715648F9F7BBFB5246A521206BB3
:10A4700008F072F9236BAAF1040A9A442AF0070A39
:10A480006B1E04F134020F3513F8011F02F8011B93
:10A49000197809B1AB42F7D10A9D4FF0000B042D9A
:10A4A00028BF0425271DE562C4E9135B384684F8FC
:10A4B00043B0FFF72BF8C5F1050504F11800FFF7CD
:10A4C00025F8C4F854B02461A561646284F858B0DA
:10A4D0004A4641465046FFF77FF8206006B1346097
:10A4E000FFF7A0F8374B384E1A68DFF818810132B1
:10A4F0001A603268002A58D134601B68012B25D1BC
:10A500003248FEF7F8FF3248FEF7F5FF3148FEF714
:10A51000F2FFDFF8F4903048FEF7EDFF2F4D3048A2
:10A52000FEF7E9FF4846FEF7E6FF2846FEF7E3FFA1
:10A530002C48FEF7E0FF2C48FEF7DDFF2B48FEF726
:10A54000DAFF2B4BC3F800902A4B1D6001252A4AE5
:10A550002A491368086801331360E26A636405FAE4
:10A5600002F3034314200B60184B394600FB023002
:10A57000FEF7CFFFFFF776F8D8F8003063B1336805
:10A58000DA6AE36A9A4207D24FF080521C4B1A6093
:10A59000BFF34F8FBFF36F8F2846BDE8F88F384663
:10A5A000FFF70CFA4FF0FF35F6E7D8F80030002B34
:10A5B000CCD13368DA6AE36A9A4298BF3460C5E75F
:10A5C000887C0108A04A0020304A00203C4A002034
:10A5D000504A0020644A0020784A0020CC4A0020DB
:10A5E0008C4A0020EC4A0020184B0020044B00202D
:10A5F000344A0020384A0020B04A0020B44A0020E3
:10A6000004ED00E0004B0020B84A002070B504467D
:10A61000284DFFF707F804B92C68261D3046FEF7D1
:10A620009BFF60B91421E06A234B41435B5833B967
:10A630000122224982400B6823EA02030B60A36ACD
:10A640001BB104F11800FEF787FF1D4A13680133A0
:10A6500013602B68A34220D131461A48FEF759FFF8
:10A66000194A136801331360FEF7FCFF174B1B6890
:10A6700093B12B68A3420FD1154B1B6823B140F255
:10A68000B6411448F9F7ACFA4FF08052124B1A60F9
:10A69000BFF34F8FBFF36F8F70BD104A206B1368ED
:10A6A000013B1360FFF78AF92046FFF787F9FFF7B0
:10A6B00015FED9E7304A00203C4A0020B44A002069
:10A6C000B04A0020184B0020A44A0020004B002074
:10A6D000AC4A0020887C010804ED00E0A04A00207C
:10A6E000F8B5054620B940F24C511748F9F778FA09
:10A6F000164B1B68AB4220D0FEF794FF144B6C69DD
:10A700001F68144B1E68FEF7ADFFBC4217D0B44261
:10A7100015D0114B9C4208D1AB6A83B995F85830DB
:10A72000012B0CBF02200320F8BD0C4B9C4208D02B
:10A73000002C0CBF04200120F6E70020F4E70220E3
:10A74000F2E70420F0E700BF887C0108304A0020CF
:10A75000344A0020384A0020044B0020184B0020C7
:10A7600070B5044620B940F21C711948F9F738FA5F
:10A77000184D2B68A34229D044B3FEF753FF20465F
:10A78000FFF7BEFDF0B1261D3046FEF7E5FE0123C2
:10A790001149E26A08689340034314200B600F4B91
:10A7A000314600FB0230FEF7B4FE2B68E26ADB6A3A
:10A7B0009A4207D34FF08052094B1A60BFF34F8F74
:10A7C000BFF36F8FBDE87040FEF74CBF70BD00BF98
:10A7D000887C0108304A0020B44A00203C4A00200E
:10A7E00004ED00E013B50024174B009401935022B0
:10A7F000234616491648FFF71BFE012818D100F022
:10A8000023FE012814D14FF0500383F31188BFF3C6
:10A810006F8FBFF34F8F4FF0FF320E4B1A600E4B0E
:10A8200018600E4B1C6002B0BDE81040FEF77ABF06
:10A83000013007D140F60401094802B0BDE81040DC
:10A84000F9F7CEB902B010BDE04A0020CC7C010877
:10A85000C5A30008E44A0020004B00202C4B002038
:10A86000887C0108024A136801331360704700BFF7
:10A87000AC4A0020014B1868704700BF2C4B0020E9
:10A8800008B5FEF7A9FF014B186808BD2C4B002046
:10A890002DE9F84F3A4B1B68002B6AD1394B1C68E5
:10A8A00001341C609CB9384D2B681B6823B140F6FD
:10A8B00062213648F9F794F9354B2A6819682960FE
:10A8C0001A60344A136801331360FFF707FD324DF5
:10A8D0004FF0000B2B68314FA34211D93A68304B2F
:10A8E000D16A14224A439A58022A28BF4FF0010B1A
:10A8F0002C4A1268002A0CBF58460120BDE8F88F88
:10A90000DFF884A0DFF8A490DAF8002012681AB902
:10A910004FF0FF322A60E1E7DAF80020D268D6680B
:10A9200071688C4201D22960D8E706F104084046DC
:10A93000FEF712FEB16A19B106F11800FEF70CFE1F
:10A9400001224FF0140CF06AD9F8003002FA00F13D
:10A950001943134BC9F800100CFB00304146FEF7B9
:10A96000D8FD3868F16AC26A914228BF4FF0010BE6
:10A97000CAE70D4A4FF0000B136801331360B7E7C5
:10A98000AC4A00202C4B0020344A0020887C01086F
:10A99000384A0020E84A0020E44A0020304A0020DB
:10A9A0003C4A0020304B0020A84A0020B44A002036
:10A9B0002DE9F8432E4C236823B940F668012D4851
:10A9C000F9F70EF9FEF72EFE2368013B2360246899
:10A9D0002CB10024FEF746FE2046BDE8F883264B46
:10A9E0001B68002BF5D0254D254EDFF8A8801FE011
:10A9F000EB680127DC6804F1040904F11800FEF794
:10AA0000ABFD4846FEF7A8FD1420E26A316807FA5C
:10AA100002F30B4300FB028049463360FEF779FDE9
:10AA2000184BE26A1B68DB6A9A4201D3164B1F601F
:10AA30002B68002BDCD10CB1FFF750FC134D2C68B8
:10AA400044B10127104EFFF723FF00B13760013CEE
:10AA5000F9D12C600C4B1B68002BBAD04FF0805200
:10AA60000B4B1A60BFF34F8FBFF36F8F0124B1E719
:10AA7000AC4A0020887C0108A04A0020EC4A002053
:10AA8000B44A0020304A0020304B0020A84A002061
:10AA900004ED00E03C4A002038B50C46054620B9DC
:10AAA00040F2CA411848F9F79BF824B940F2CB416B
:10AAB0001548F9F795F8154B1B6823B140F2CC41C6
:10AAC0001148F9F78DF8FFF7CDFE114B2A68186889
:10AAD00014192CBF0121002182422C600CD961B9CC
:10AAE000FFF766FF38B94FF080520A4B1A60BFF388
:10AAF0004F8FBFF36F8F38BD09B9A042F0D200214C
:10AB0000201AFFF719FCEBE7887C0108AC4A00200B
:10AB10002C4B002004ED00E010B5044640B94FF086
:10AB200080520D4B1A60BFF34F8FBFF36F8F10BD74
:10AB30000A4B1B6823B14FF4A4610948F9F750F898
:10AB4000FFF790FE00212046FFF7F6FBFFF730FFEE
:10AB50000028E4D0EBE700BF04ED00E0AC4A0020A1
:10AB6000887C0108224B70B51A68224B12B1012271
:10AB70001A6070BD204E1A6033681B6B1A68B2F100
:10AB8000A53F0BD15A68B2F1A53F07D19A68B2F13F
:10AB9000A53F03D1DB68B3F1A53F04D0306831682D
:10ABA0003431F8F7EDFF154B1C68B4FA84F4142324
:10ABB000E4B2C4F11F046343114DEB5823B940F6CE
:10ABC00088311048F9F70CF8142202FB04F3E91855
:10ABD0004868083340682B44984202FB045408BF7D
:10ABE0004368486008BF4B606368DB683360C0E758
:10ABF000AC4A0020304B0020304A0020B44A0020EC
:10AC00003C4A0020887C010870B504462A4EFEF7B5
:10AC100009FD04B93468251D2846FEF79DFC60B97E
:10AC20001421E06A254B41435B5833B90122244982
:10AC300082400B6823EA02030B60A36A1BB104F194
:10AC40001800FEF789FC29461E48FEF762FC94F8BE
:10AC500058301D4D012B04BF002384F85830FEF7F7
:10AC600001FD2A682AB1FEF7DDFCFFF737FBFEF78E
:10AC7000F9FC3368A34211D12B6883B1134B1B68D5
:10AC800023B14FF4D9611248F8F7AAFF4FF0805270
:10AC9000104B1A60BFF34F8FBFF36F8F70BD094A1F
:10ACA00011680D4A1268914201D13360F6E7BDE8A0
:10ACB0007040FFF757BF00BF304A00203C4A0020D9
:10ACC000B44A0020044B0020004B0020AC4A002076
:10ACD000887C010804ED00E0A04A002038B50D464C
:10ACE000044620B940F69F310748F8F779FF074B33
:10ACF000204619681831FEF718FC2846BDE8384090
:10AD00000121FFF719BB00BF887C0108304A0020F1
:10AD100070B50E461446054620B940F6CA310A48B9
:10AD2000F8F75EFF094B284619681831FEF7F1FB6A
:10AD3000002C214608BF3046BDE8704018BF4FF0D8
:10AD4000FF30FFF7F9BA00BF887C0108304A0020C5
:10AD500038B5C368DC6824B940F6FA311548F8F70D
:10AD60003FFF04F118052846FEF7F6FB124B1B685F
:10AD7000E3B9251D2846FEF7EFFB01230F49E26AE0
:10AD800008689340034314200B6029460C4B00FBDA
:10AD90000230FEF7BEFB0B4BE26A1B68DB6A9A428D
:10ADA00085BF0120084B0020186038BD29460748A0
:10ADB000EFE700BF887C0108AC4A0020B44A0020BD
:10ADC0003C4A0020304A0020304B0020EC4A002052
:10ADD000034B1B680360034B1B684360704700BF55
:10ADE000E84A00202C4B002070B50C46054620B9DF
:10ADF00040F665411448F8F7F3FE24B940F6664181
:10AE00001148F8F7EDFEFEF70DFC104B1A682368A9
:10AE1000591C0FD00E482E6800686968864201D020
:10AE200091420ED9521A934209D99B1A236028469F
:10AE3000FFF7CEFF0024FEF715FC204670BD00236F
:10AE400023600124F7E700BF887C01082C4B002019
:10AE5000E84A00200122014B1A607047304B002065
:10AE600070B50C461646054608B91B4A156805F12B
:10AE700034026260EA6A052B22612A6B2560E26176
:10AE80006A6CA260EA6C62614FF00002A2611BD0A2
:10AE900011490968A9420BD12273D6B1296B0A4620
:10AEA000531A12F8010BA528FAD09B08238470BD11
:10AEB000032B2373F1D1FFF7D5FCAB6A0BB102234F
:10AEC0002373FFF775FDE8E72846FFF709FC2073B9
:10AED000E3E72684EBE700BF304A002008B9064BC1
:10AEE0001868026B1346981A13F8011BA529FAD0AB
:10AEF000C0F38F00704700BF304A0020014B186834
:10AF0000704700BF304A0020054B1B6833B1054B2A
:10AF10001B68002B0CBF02200020704701207047E7
:10AF2000004B0020AC4A00202DE9F04104460028E7
:10AF300036D0234AC36A11681746C96A8B4237D292
:10AF4000142682691F4D002AA8BF3A6806FB0353E6
:10AF5000A2BFD26AC2F10502826142699A4221D13E
:10AF600000F104084046FEF7F7FA174B48B9E06ACB
:10AF70004643AA592AB901211A68814022EA0102EE
:10AF80001A603A681968D26AE262012404FA02F08F
:10AF9000084318601420414600FB0250FEF7B9FA3E
:10AFA000204603E03B68DB6AC3620120BDE8F08114
:10AFB0001368C06CDC6AA0422CBF00200120F5E7BA
:10AFC000304A00203C4A0020B44A0020F8B504462C
:10AFD00008B90020F8BD1F4B1B68834204D040F61F
:10AFE0007A711D48F8F7FCFD236D23B940F67B719B
:10AFF0001948F8F7F5FD236DE16AE26C013B9142D7
:10B000002365E6D0002BE4D1251D2846FEF7A4FADF
:10B01000124E134A50B91421E76A794373582BB979
:10B0200001201368B84023EA00031360E36CC3F106
:10B030000501A161E3620124116804FA03F00843E9
:10B0400010601420294600FB0360FEF762FA2046D8
:10B05000C0E700BF304A0020887C01083C4A00203D
:10B06000B44A0020F8B50D460446002845D0036DCB
:10B0700023B940F6C9712148F8F7B2FDE36C9D424F
:10B0800038BF1D46E36AAB4237D0236D012B34D164
:10B090001B4B1B68A34204D140F6E4711748F8F734
:10B0A0009FFD1426A269E36A002AE562A4BFC5F1E8
:10B0B0000505A561134D626906FB03539A421CD135
:10B0C000271D3846FEF748FAE26A0F4C40B956434E
:10B0D000AB592BB901212368914023EA0103236076
:10B0E00001231420216893400B432360394600FB61
:10B0F0000250BDE8F840FEF70CBAF8BD887C0108A4
:10B10000304A00203C4A0020B44A0020044B1A6810
:10B110001AB119680A6D01320A651868704700BFD4
:10B12000304A00202DE9F0411E4C1E4680460F4655
:10B130001546FEF777FA236893F85830022B14D09F
:10B14000012123685A6D22EA08025A65236883F8B0
:10B15000581056B13046FFF7EFF84FF08052124BBF
:10B160001A60BFF34F8FBFF36F8FFEF77BFAFEF7C6
:10B1700059FA15B123685B6D2B602368002293F8A0
:10B180005830022B09BF012500252368596D04BFE3
:10B19000B9435965236883F85820FEF763FA2846B7
:10B1A000BDE8F081304A002004ED00E0F8B50E461D
:10B1B00017461D46044620B941F219212B48F8F7DD
:10B1C0000FFDFEF72FFA0DB1636D2B60022394F88B
:10B1D000585084F85830EDB2042F16D8DFE807F045
:10B1E0000A0307051100636D1E43666502E0636D87
:10B1F00001336365012D11D00124FEF733FA204697
:10B20000F8BD022DF1D10024F7E7636D0133F1D0D1
:10B2100041F24A211548F8F7E3FCEBE7261D3046DA
:10B22000FEF79AF91420124AE36A11689D400D4313
:10B230001560104A314600FB0320FEF76AF9A36A45
:10B2400023B141F259210948F8F7CAFC0A4BE26AD6
:10B250001B68DB6A9A42CFD94FF08052074B1A60C5
:10B26000BFF34F8FBFF36F8FC6E700BF887C010825
:10B27000B44A00203C4A0020304A002004ED00E09F
:10B280002DE9F843DDF820800E4691461D46044620
:10B2900020B941F28C213548F8F7A2FCFEF79CFA60
:10B2A000EFF311874FF0500383F31188BFF36F8FD3
:10B2B000BFF34F8F0DB1636D2B60022394F858508C
:10B2C00084F85830EDB2B9F1040F16D8DFE809F070
:10B2D0000A0307051100636D1E43666502E0636D96
:10B2E00001336365012D11D0012087F31188BDE87A
:10B2F000F883022DF1D10020F7E7636D0133F1D01F
:10B3000041F2CF211948F8F76BFCEBE7A36A23B1B0
:10B3100041F2DA211548F8F763FC154B1B6803BBB3
:10B32000251D2846FEF718F901231249E26A08682C
:10B330009340034314200B6029460F4B00FB02305F
:10B34000FEF7E7F80D4BE26A1B68DB6A9A42CBD93D
:10B350000123B8F1000F01D0C8F80030084A13608B
:10B36000C2E704F118010748EAE700BF887C01083A
:10B37000AC4A0020B44A00203C4A0020304A002059
:10B38000304B0020EC4A002038B5054608B9084B80
:10B390001D680024FEF746F995F85830022B04BFCB
:10B3A00085F858400124FEF75DF9204638BD00BFFE
:10B3B000304A0020F8B50F4CFEF734F92568ADB9D6
:10B3C0000D4F0E4E3846FEF796F83046FEF793F8CE
:10B3D0000B4B2A461F600B4B0C210A201E60FEF708
:10B3E000EFFB206010B10849FEF71CFFBDE8F840F4
:10B3F000FEF738B9684B00203C4B0020504B002032
:10B40000344B0020384B0020D17C0108914208B514
:10B41000416000610AD8D21A83699A420DD2084B62
:10B42000011D1868FEF781F8002008BD9A4201D27C
:10B43000994202D2011D034BF3E70120F5E700BF5B
:10B44000384B0020344B002007B5FFF7B3FF0C4BFF
:10B450001B6843B90B484FF48971F8F7C1FB002012
:10B4600003B05DF804FB084BC82201930123074990
:10B47000009307480023FEF7DBFF0028EAD0EFE740
:10B48000684B0020D67C01086C4B00201B7D010816
:10B49000ADB500082DE9F04180462C200D46174639
:10B4A0001E46FEF7F9F9044688B125B94FF4B67186
:10B4B0000848F8F795FBFFF77DFF069BC4F800806E
:10B4C000C4E9065726626362201DFEF71FF8204676
:10B4D000BDE8F081D67C01082DE9FF410D4690467C
:10B4E0001F46064620B94FF4C3710F48F8F778FBA2
:10B4F0000E4C206878B1052DCDE9015803960DDC7E
:10B50000FFF702FD002302280CBF0A9A1A4601A980
:10B510002068FEF779FB04B0BDE8F08100233A46CD
:10B5200001A9FEF727FCF6E7D67C0108684B00204E
:10B530002DE9F74300271A4DDFF86C802B681A6855
:10B5400032B9184A11681360296003B0BDE8F0836E
:10B55000DB68DC681E6804F104094846FDF7FCFF5F
:10B56000636A20469847E369012BE7D1A369334416
:10B570009E4206D26360246149462868FDF7D5FFE4
:10B58000DCE700230097324619462046FFF7A4FF68
:10B590000028D3D140F272314046F8F721FBCDE7C5
:10B5A000344B0020384B0020D67C01082DE9F04FA9
:10B5B0004FF00108624D89B0DFF898B1DBF8002048
:10B5C000136843B30024D368D3F80090FFF74AF917
:10B5D000FFF750F95B4B82461A681F4690425A4E5D
:10B5E0001CD31860002C4CD0584B1B681A68B2FA58
:10B5F00082F25209A9EB0A013068FEF74BFEFFF711
:10B60000D7F998B94FF08052514B1A60BFF34F8F62
:10B61000BFF36F8F0AE001249946D7E70393FFF742
:10B6200087FF039BC3F800A0FFF7C2F9002205A91A
:10B630003068FEF743FC0028BED0059B002BF5DBED
:10B64000079C636913B1201DFDF786FFFFF712F910
:10B650003B688146984201D2FFF76AFF059BC7F815
:10B660000090092BE2D808FA03F313F4047A57D1B7
:10B6700013F0C70F33D19B06D8D52046FEF79EF9AD
:10B68000D4E7814529D8FFF793F9DBF80030DB6870
:10B69000D3F80CB00BF10400FDF75EFFDBF81C30B3
:10B6A000012B15D1DBF818104B4652464944584639
:10B6B000FFF7ACFE60B1009423464A462146584647
:10B6C000FFF70AFF20B94FF4F4712846F8F788FA1B
:10B6D000DBF8243058469847A8E722468AE7A16954
:10B6E000069B4A4619442046FFF790FE00289DD04D
:10B6F000636A20469847E369012B97D1A2690699AE
:10B70000CDF800A00A44534651462046FFF7E4FE18
:10B7100000288BD140F201312846F8F761FA85E71D
:10B72000069BA36123B94FF446712846F8F758FAEF
:10B73000A1694B464A4649442046FFF767FE75E734
:10B74000D67C0108644B0020684B0020384B002059
:10B7500004ED00E0344B0020021C18BF0122002140
:10B760000148F9F7F1BF00BF00040240FAF796BBA9
:10B7700038B505460C460020FFF7EEFF45F0800087
:10B78000FFF7F4FF2046FFF7F1FFBDE83840012046
:10B79000FFF7E2BF08B50120F9F7C8FD0A20F9F765
:10B7A000C5FD0B20F9F7C2FD0720F9F7BFFD052005
:10B7B000F9F7BCFDBDE808400420F9F7B7BD00006B
:10B7C000204B70B59D780446EDB958B902211E484A
:10B7D000F9F7B4FF23461A460221BDE870401A4823
:10B7E000F9F7E4BE012805D102211748F9F7A0FFB7
:10B7F0002B46F0E7022823D102460146BDE87040FF
:10B800001148F9F711BF012D14D138B904210E48A0
:10B81000F9F794FF002304211A46DEE7012804D13A
:10B8200004210948F9F784FFF4E7022808D1024609
:10B830000421E3E76821BDE870400448F8F7D0B977
:10B8400070BD00BF704B002000000240237D010846
:10B8500008B50020FFF7B4FFF9F7AAFC0120FFF7B5
:10B86000AFFFF9F7A5FC0220FFF7AAFFBDE80840EB
:10B87000F9F79EBC08B500210120FAF791FA0120E2
:10B88000FFF76AFF0023094819461A46F9F78EFEAA
:10B89000B5214020FFF76CFFA0214120FFF768FF92
:10B8A000BDE8084000210120FFF762BF000402400C
:10B8B00010B5FFF76FFF0120FFF74EFF00233A4856
:10B8C0001A461946394CF9F771FE00210120FAF7A2
:10B8D00067FA22787AB1002306211A463248F9F72E
:10B8E00065FE06213048F9F723FFF9F761FC1921BD
:10B8F0005820FFF73DFFFFF7ABFFFFF7BBFF637873
:10B900005BB1002304211A462948F9F74FFE0023B2
:10B910000D211A462748F9F749FE00220121224845
:10B92000F9F782FE00220A211F48F9F77DFE002266
:10B930000B211D48F9F778FE002207211A48F9F774
:10B9400073FE002205211848F9F76EFE002204213B
:10B950001548F9F769FE0E23022201211248F9F772
:10B9600003FD0E2302220A210F48F9F7FDFC0E23E6
:10B9700002220B210C48F9F7F7FC0E2302220721C3
:10B980000948F9F7F1FC0E23022205210648F9F7D0
:10B99000EBFC094B1B782BB9BDE81040BC210748D4
:10B9A000F8F71EB910BD00BF00040240704B002024
:10B9B0000000024000080240734B0020237D010874
:10B9C00082B0019002AB33F8041D054A9B781180C8
:10B9D00093700122034B1A7002B0FFF769BF00BFDA
:10B9E000704B0020734B00201A4B10B55B78D3B11D
:10B9F0000128194C18D104211848F9F799FE0D2196
:10BA00001748F9F79BFE23786BB1002304211A46EF
:10BA10001248F9F7CBFD00230D211A461048F9F71B
:10BA2000C5FD0023237010BD40B904210B48F9F770
:10BA300085FE0D210A48F9F77BFEE4E70222042186
:10BA40000648F9F7F1FD02220D210548F9F7ECFD52
:10BA50000123E7E7704B0020840000200000024033
:10BA60000008024008B5FFF795FEFFF7F1FEFFF76B
:10BA700001FFFAF7EFF9012200211F48F9F7D4FD81
:10BA80000220FFF7B1FF0220FFF79AFE02220121F8
:10BA90001948F9F7C9FD02220A211748F9F7C4FD30
:10BAA00002220B211448F9F7BFFD02220721124898
:10BAB000F9F7BAFD022205210F48F9F7B5FD022278
:10BAC00004210D48F9F7B0FD0C4B1B781BB9E021A0
:10BAD0000B48F8F785F80B4B1B785BB10023062168
:10BAE0001A460548F9F762FDBDE8084006210248FC
:10BAF000F9F724BE08BD00BF00040240734B0020CC
:10BB0000237D0108704B002010B5064C0222204610
:10BB10000021F9F789FD2046BDE8104002220121ED
:10BB2000F9F782BD00140240014BDB68184700BFE3
:10BB3000744B00200120704701B1096818B1806A78
:10BB4000431A58425841704710B5044618B9CF21DE
:10BB50000748F8F745F8074B5B689847D4E9062390
:10BB6000904271EB0304B4BF101A002010BD00BF57
:10BB70006E810108744B00202DE9F849884604467F
:10BB800010B10369012B03D1E0211748F8F728F819
:10BB9000D4E906BC5BEA0C0323D0D4E90867BBEB0D
:10BBA00006006CEB0701F5F767FB054620690138D5
:10BBB000F5F748FB01462846F5F750FC0546404698
:10BBC000F5F740FB2946F5F795FB2946F5F788FA86
:10BBD000F5F7E0FC321847F1000310461946C4E9B6
:10BBE0000601BDE8F88900BF6E81010838B50C4B2D
:10BBF0000546186800F0C9FB10B90023184638BD87
:10BC00004FF47A7403686C431A68A242F6D000F0CD
:10BC1000B3FB0028F1D003681A689442F6E700BF2E
:10BC2000744B002041F65832A0F55223A3F6183386
:10BC3000934224D8A0F55423A3F1F902622A1ED915
:10BC40006FF454729A18C62A19D9A3F21353302BE1
:10BC500015D9104B984214D903F6B833984212D92B
:10BC600003F51673984210D903F5167398420ED94E
:10BC700003F5E173984294BF052006207047002029
:10BC8000704701207047022070470320704704204E
:10BC9000704700BFE8320D00F8B5054618B9EC2131
:10BCA0002248F7F79DFF224E306800F06EFB002817
:10BCB0003BD0002D39D003681A79AA4231D11F7BBD
:10BCC00000F05AFB20BB87B3062D03D93D2117484E
:10BCD000F7F786FF174B53F8354024BBF72113487D
:10BCE000F7F77EFF306800F050FB0646E8B17C4372
:10BCF00037683B79AB4204D121463846FFF73CFF19
:10BD00003C61304600F038FB06460028F0D10CE0DC
:10BD100003681A79AA42D3D11B7B002BD0D00137FC
:10BD2000CEE70027CCE7012CDCD1F8BD6E810108FD
:10BD3000744B0020347D01082DE9F04F044687B094
:10BD400058B3254B00681D69F5F77CFAF5F76CF9D7
:10BD50001FA3D3E9002309F063FA227B06460F46AE
:10BD60002379D4F82890D4F81080D4F808A0BAB178
:10BD7000062B98BF194A204694BF52F823B0DFF82B
:10BD800068B0FFF7E1FE32463B46CDE90198CDE9C8
:10BD900003A01348CDF800B0A84707B0BDE8F08F66
:10BDA000062B98BF0D4A204694BF52F823B0DFF807
:10BDB00038B0FFF7C9FECDE90189CDE903A0CDF880
:10BDC00000B032463B460748E6E700BFAFF30080CD
:10BDD0000000000080842E41744B00206C7D01081F
:10BDE00055800108AA8001084780010810B5104C51
:10BDF000206820B923690F48BDE81040184700F0BB
:10BE0000CDFA2369014660B10B489847206800F0DD
:10BE1000BCFA044638B9204600F0AEFA044610B920
:10BE200010BD0648E8E72068FFF786FFF3E700BF8C
:10BE3000744B0020C87F0108E67F010820800108BC
:10BE4000F8B5134D06462B7E0F4623B940F25B1121
:10BE50001048F7F7C5FE2C6824B96B690E4898475F
:10BE60002046F8BD0D4B2046002E08BF1E4600F0B0
:10BE70008CFA054608B90024F2E7046839462046E2
:10BE8000B0470028ECD1284600F076FAF1E700BF71
:10BE9000744B00206E810108897F010835BB0008C2
:10BEA0002DE9F0472F4D81462B7E0E46904623B953
:10BEB00040F28B112C48F7F793FE2C682CB96B6974
:10BEC0002A4898472046BDE8F087294B2046002E97
:10BED00008BF1E4600F059FA824620B96B69254812
:10BEE00098475446EEE70468237B6BB94FF0FF3761
:10BEF0000024504600F040FA824690B9B8F1000F95
:10BF0000E0D0C8F80070DDE7A3684B45EEDB002108
:10BF10002046B0470028E9D02046FFF715FE074627
:10BF2000E7E7DAF800502B7B002BE2D0AB684B45FB
:10BF3000DFDB00212846B0470028DAD02846FFF78B
:10BF400003FE6CB187420AD8D3D1D4E90823D5E9DE
:10BF50000801FBF778F8002818BF2C46C9E7074608
:10BF60002C46C6E7744B00206E810108897F0108CA
:10BF700035BB0008AD7F01082DE9FF470D4604469B
:10BF800020B94FF4E6712A48F7F72AFE236923B94E
:10BF900040F2CD112648F7F723FEDFF89CA04FF0C2
:10BFA0000009DAF80430984702460B460646C4E911
:10BFB000082320690F46F5F745F92946F5F79AF960
:10BFC0002946F5F78DF8F5F72FF817A3D3E90023E5
:10BFD00009F026F909F05CFD09F092FA361847EBF2
:10BFE0000907C4E9066780462068F5F72BF9F5F7DD
:10BFF0001BF80DA3D3E9002309F012F906462846E1
:10C000000F46CDE90289F5F70FF83246CDE9000178
:10C010003B46DAF810100748884704B0BDE8F047FF
:10C02000FFF7E4BEAFF300800000000080842E41E3
:10C030006E810108887D0108744B002008B5FFF768
:10C04000F1FD003018BF012008BD000038B50D4DCE
:10C0500004462A7E22B940F207210B48F7F7C0FDBB
:10C0600074B1237B63B1002320792373FFF714FE9F
:10C070002B69064898472046BDE83840FFF75CBE6C
:10C0800038BD00BF744B00206E810108587F010845
:10C0900038B50D4D04462A7E22B940F213210B48D3
:10C0A000F7F79EFD74B1237B63B9012320792373D5
:10C0B000FFF7F2FD2B69064898472046BDE8384057
:10C0C000FFF73ABE38BD00BF744B00206E810108F7
:10C0D000717F0108F8B5194D06462B7E23B940F251
:10C0E0001F211748F7F77CFD2C6824B96B691548A8
:10C0F0009847204601E00EB90020F8BD204600F028
:10C1000044F904460028F7D023689E420CD13779C1
:10C110003046FFF709FD2146286800F04DF9384602
:10C12000FFF7BAFD0120E8E7204600F025F90446B4
:10C130000028E9D16B690448DAE700BF744B00209E
:10C140006E81010826810108488101082DE9F84324
:10C15000384D06462B7E8846914623B94FF4F2713E
:10C160003548F7F73DFD3046FFF768FF044630B924
:10C170006B693146314898472046BDE8F883304620
:10C18000FFF734FD044630B12D482B6931469847FE
:10C190002046FFF79FFF2B7E1BB973212648F7F738
:10C1A0001FFDAB6830209847044640B96B692548AD
:10C1B00098476B693146244898470024DCE73022D1
:10C1C000002106F0C9FA3046FFF72CFD0746207122
:10C1D00038B9EB68204698476B6931461B48984749
:10C1E000E7E7062803D93D211348F7F7F9FC184B78
:10C1F000214603EBC70253F83730526823614FF4EE
:10C200007A73A2605E4300220023C4E9062301235F
:10C2100026602373C4E90A89286800F097F820791A
:10C22000FFF73AFD2B690B4898472046FFF784FD3E
:10C23000A2E700BF744B00206E810108407E010818
:10C24000777E0108AC7E01081D7F0108DA7E0108B7
:10C25000347D0108057F010870B50F4C0546237E2B
:10C2600023B940F25B210D48F7F7BAFC23685BB1B4
:10C270000B4E29463046FFF7E3FD50B923692946A6
:10C28000BDE870400748184763690748BDE870403B
:10C290001847FFF749FCECE7744B00206E8101085A
:10C2A00039BB00080081010826810108014B187E76
:10C2B000704700BF744B002084B070B504AC84E8B4
:10C2C0000F00154B1A7E1C462AB1BDE870405B6911
:10C2D000124804B018471D1D04AE0FCE0FC53368B9
:10C2E0002B600BB90E4B636123690BB90C4B2361B7
:10C2F000E3680BB1A36833B923690A4898470A4B2E
:10C30000E3600A4BA36000F013F80123206023765A
:10C31000BDE8704004B07047744B0020CC7D01082C
:10C320008D710008057E0108C1260108B1260108AB
:10C3300010B50820FAF7C0FF0446FEF793FA002371
:10C34000C4E90034FEF734FB204610BD70B5054645
:10C350000C200E46FAF7B0FF044660B10660FEF707
:10C3600081FA002363606B68A3601C6004346C6016
:10C37000FEF71EFB012070BD10B50446FEF772FAF1
:10C380006468FEF715FB204610BD10B50446FEF7A5
:10C3900069FA2468FEF70CFB204610BD10B5044670
:10C3A000FEF760FA236800241BB9FEF701FB204664
:10C3B00010BD01345B68F7E738B50C460546FEF75B
:10C3C00051FAD4E901324BB19A60A2681360FEF7CA
:10C3D000EFFA2046BDE83840FAF758BF6A60F4E744
:10C3E000044B1A7F22B993F82A0080F001007047AD
:10C3F000002070478800002070B590B00C464022A5
:10C4000000210546684606F0A7F906F0CFFF06466C
:10C41000204606F0A7FF002406F0C8FF0DEB04033A
:10C420000134102C1872F7D1002406F0BFFF0DEB79
:10C4300004030134102C83F82000F6D1002406F008
:10C44000B5FF0DEB04030134102C83F83000F6D156
:10C45000002406F0ABFF0DEB04030134082C187622
:10C46000F7D1304606F07EFF2C466B4610AE1A46DA
:10C4700003CAB24220606160134604F10804F6D199
:10C48000284610B070BD000084B070B58AB00EAC04
:10C4900084E80F00664CA8222546002104F12800FC
:10C4A0000EAE06F059F90FCE0FC5336813AE2B60F0
:10C4B00004F114050FCE0FC533682B600E9B0BB92A
:10C4C0005C4B23600F9B0BB95A4B2360109B1BB92D
:10C4D000BD215948F7F784FB129B1BB9C12156486F
:10C4E000F7F77EFB119B1BB9C5215348F7F778FB83
:10C4F000636923B923685148984703236361A3699B
:10C500000BB90A23A361A37F0BB90123A37701F021
:10C5100079FDE37F0BB90123E37701F06BFD636ADB
:10C520000BB9474B636201F059FDFBF785F9C4F87D
:10C53000C0000138033004D963684248984700209E
:10C540006DE0032200210120FDF73AFBC4F8C8008A
:10C5500018B9EE213848F7F743FB00220421A069FF
:10C56000FDF72EFB606318B9F2213348F7F738FB6B
:10C57000002204210120FDF723FBA06318B9F52157
:10C580002D48F7F72DFB082384F8A330042384F803
:10C59000A430FFF78BFE05AD68B9A3682269059347
:10C5A000236807920893E26863680692009395E80F
:10C5B0000F00FFF781FE01F04BFD2368224E079329
:10C5C000636806F150020893236904960693E368B2
:10C5D000883605930AAB43F81C2D93E803008DE8D9
:10C5E000030095E80F0002F019FE019663694FF40D
:10C5F000CD720093154901231548FDF719FF012855
:10C60000054611D1002303220421D4F8C400FEF70B
:10C61000CDFD104823689847284684F829500AB071
:10C62000BDE8704004B0704763680B4886E700BF00
:10C63000880000208D7100081183010851830108D2
:10C6400008E6D3339A830108C4000020CD83010893
:10C6500011C80008D5830108F283010810B5154CF4
:10C66000D4F8C43023B94FF490711348F7F7B8FAEF
:10C67000042100230322D4F8C400FEF797FD0F48DD
:10C680002368984742F21071D4F8C800FDF7A8FC5F
:10C6900020B940F229110848F7F7A2FA0023D4F88C
:10C6A000C8001A461946FDF7AFFA23680448BDE8EA
:10C6B000104018478800002011830108DE8401081B
:10C6C0000585010838B50E4DD5F8C83023B940F2BC
:10C6D00031110C48F7F784FA0021D5F8C800FDF7AE
:10C6E0007FFC0128044608D10023D5F8C8001A466B
:10C6F0001946FDF789FA204638BD0020FCE700BF47
:10C70000880000201183010810B5FFF7DBFF0B4CF8
:10C7100078B1002303220821D4F8C400FEF746FDB7
:10C72000236807489847D4F8C400BDE81040FEF7D6
:10C7300017B823680348BDE8104018478800002058
:10C740002085010842850108014B1863704700BF2E
:10C7500088000020002307B502A941F8043D044BDE
:10C760000246986BFDF7AAFB019803B05DF804FB45
:10C770008800002070B5FFF7A5FF1F4E054620B1C9
:10C7800073681E489847002070BD706BFDF724FD4C
:10C79000B369834202D233681948F3E72946284631
:10C7A00002F06CFD044610B933681648EAE70570DC
:10C7B00000F0F4FB054618B9204602F09FFDE2E7C1
:10C7C000114A1368013313608BB913680133136086
:10C7D0006B6001236B70022328462B7000F014FC61
:10C7E00038B9284600F0ECFB73680848CAE71368BC
:10C7F000EEE76868C8E700BF8800002022840108CF
:10C800004E84010880840108904B0020BD840108FB
:10C8100001232DE9F041534D534F544E85F82830F4
:10C820000A23514A4FF0FF310020FEF77BFC01281C
:10C8300048D1386843071AD533781BB1FAF758FF47
:10C8400000233370FCF7EEFE2B6849489847FCF74D
:10C8500009FF022385F828300023D5F8C8001A46BE
:10C860001946FDF7D1F90020FEF7CEF9D8E710F010
:10C87000080024D0337883B941F28830FAF764FF96
:10C8800018B94A213B48F7F7ABF901233A4833700E
:10C890002B689847394BDB6A98470020FEF774FDF8
:10C8A0004FF4FA61D5F8C800FDF79AFB18B9512189
:10C8B0003048F7F795F9012385F82830B0E7FEF7FF
:10C8C00063FDADE73378002BAAD000F0AFFB044640
:10C8D0000028A5D003781BB962212648F7F780F914
:10C8E000032385F828302378D5F80080032B96BFE2
:10C8F000234A244A52F8232061682348C0472378FA
:10C90000012B09D001D3032B1ED96B681F48984710
:10C91000204600F055FB83E7FFF762FD60B11C483D
:10C920002B689847204600F06FFB10B9204600F0B6
:10C9300047FBFFF71FFF73E7204601F0F9F938B115
:10C94000204600F03DFB08E0204600F07DFFF6E7C2
:10C95000204600F059FB0028F2D0084BDB6A9847CC
:10C960005EE700BF88000020984B0020944B002019
:10C970005C8201081183010879820108247A010888
:10C980004482010854820108A9820108EE8201084C
:10C99000C7820108024B93F8980001F02DBD00BF3B
:10C9A000880000202DE9FF4180460F461546ADF86E
:10C9B0000430FFF787FE384E044638B173683748B5
:10C9C00098470024204604B0BDE8F081706BFDF765
:10C9D00003FCB369834203D2336831489847F1E7D7
:10C9E000FFF7D8FF8742014605D9336896F89820AB
:10C9F0002C489847E6E715B933682B48E0E7DF2D68
:10CA000002D933682948E9E73946404602F036FC46
:10CA1000044610B933682648E0E79DF80530B3B105
:10CA2000042323709DF804303BB10D2304A901F8C1
:10CA3000013D0122204600F07DFE6577204600F092
:10CA4000ADFA054628B9204602F058FCB9E70223A2
:10CA5000E7E70023174A83601368013313609BB92B
:10CA60001368013313606B600A9B28462B61012316
:10CA70006B702B7000F0B6FA044638B9284600F007
:10CA80009FFA73680C48A9E71368ECE73368696894
:10CA90000A4898476C6895E78800002022840108BE
:10CAA0004E84010872850108CE850108F3850108CE
:10CAB00035860108904B002070860108A286010887
:10CAC000082808BF0120024B987783F89800704728
:10CAD00088000020024BD87783F89900704700BF88
:10CAE0008800002008B5FAF77FFC014BD86308BD29
:10CAF00088000020034630B5054C00F110052246A1
:10CB000018685968083303C2AB421446F7D130BDE8
:10CB1000C8000020034630B5054C00F11005224640
:10CB200018685968083303C2AB421446F7D130BDC8
:10CB3000D80000200246024B0068516803C37047CA
:10CB4000F80000200246024B0068516803C370479A
:10CB500000010020034630B5054C00F110052246C7
:10CB600018685968083303C2AB421446F7D130BD88
:10CB7000E8000020014B5877704700BF8800002074
:10CB800038B50D461446FFF7ADFF2846FFF7B2FF54
:10CB90002046FFF7BFFF0122014B1A7738BD00BFC7
:10CBA0008800002038B50D461446FFF7C3FF28461D
:10CBB000FFF7C8FF2046FFF7CDFF0022014B1A7791
:10CBC00038BD00BF880000202DE9F04186B08046C6
:10CBD0000C468DF80F202BB101220DF10F01002022
:10CBE000FBF774FA0025284B20469DF80F109B6A2E
:10CBF0009847264F05AB9DF80F00009304AA2B46DB
:10CC00002946234ECDE90455FAF756FEDDE9042303
:10CC10009DF80F101F483C68A04740F6B8323146D7
:10CC2000D7F8C000FDF74AF938B3FDF723FE337893
:10CC30000446012B30461CD1FAF7AEFD0498F4F7F8
:10CC400001FB01464046FFF797F9D8F80000F4F7DA
:10CC5000F9FAF4F7E9F90AA3D3E9002308F0E0FAB6
:10CC60003D6802460B460C48A847204606B0BDE882
:10CC7000F081FAF791FD2C46F7E70446F5E700BF8F
:10CC80000000000080842E41247A010888000020E2
:10CC90009C4B0020C4870108F48701082DE9F84F58
:10CCA0003C4C1F46636B0546884691469847A34611
:10CCB000394E3A4CDFF8FCA04FF47A7202FB05F3D0
:10CCC00003F5C333A033B3FBF2F23449D6F8C00006
:10CCD000FDF7F4F828B9DBF8303098474FF0FF3013
:10CCE00036E02378072B0DD1FBF774F92046FAF7CD
:10CCF00053FD3568FDF7BEFD01465046A8474FF489
:10CD00007A65D9E7032BDBF830A023D13568FDF72E
:10CD1000B1FD01462248A847656828792968814500
:10CD200028BF814640464A4605F0F2FC366895F930
:10CD30000830B5F90620A9881A48B0471FB1EB881A
:10CD40003B802B7ABB701548FAF726FDD047484642
:10CD5000BDE8F88F042B0BD13468FDF78BFD01463D
:10CD60001148A0470D48FAF717FDD0470020EFE71C
:10CD7000052B0AD13468FDF77DFD01460B48A0471D
:10CD80000648FAF709FDD047A8E7B7210848F6F7A3
:10CD900027FFF5E7247A010888000020A44B002033
:10CDA00011870108268701085B870108738701083E
:10CDB00089870108F78601082DE9F04FC3B002AF5B
:10CDC000894616463946FF229B46DDF8348102F03B
:10CDD000B5FA644C054630B923686348984700208B
:10CDE00043B0BDE8F08F94F8993094F89820D9F8C2
:10CDF0000010002001F0B2FB00232A4639464846C5
:10CE0000FFF7E2FE019010B923685848E6E7FF22D9
:10CE10000021384605F0A0FC94F8982094F89A3048
:10CE2000D9F8001093429ABFD21AD2B20022062338
:10CE3000012001F093FB2568FDF71CFD4FF47A7982
:10CE4000019A0146323A32444948A84709FB06F1A3
:10CE5000A1F543415039B1FBF9F101A8FDF71CFEE2
:10CE6000D4F800A0FDF706FDABEB0606A6F16405BD
:10CE70002A4601463F48D047FF22434639462846C6
:10CE8000FFF70CFFD4F800B00546FDF7F3FC0146B0
:10CE90003948D8476A1C02D1236838489EE7002DDC
:10CEA00025DD2368294636489847B8F1000F02D09F
:10CEB000012388F8033000264C9BB5421E6014DD28
:10CEC000E9B2384602F0B0FB4C9BDFF8CC8018602A
:10CED00023682C489847B95D236840460136984737
:10CEE000B542F8D1236828489847012078E70623FF
:10CEF00094F89B20D4F89C10012001F02FFB2568AA
:10CF0000FDF7B8FC09FB06F601462048A847B6FB2A
:10CF1000F9F101A8FDF7C0FD2568FDF7ABFC40F66F
:10CF2000B83201461348A8474346FF22394640F627
:10CF3000B830FFF7B3FE26680546FDF79BFC0146B7
:10CF40000D48B0476B1C02D12368114846E7002DFD
:10CF5000B1DD236829460F489847B8F1000FAAD0E1
:10CF60000223A6E7880000203088010850880108C5
:10CF70006E8801089B880108B7880108C8880108E5
:10CF8000F188010886890108C66301081389010830
:10CF90003A890108638901081E67010838B5074B03
:10CFA0000546DB6818209847044620B1142200216A
:10CFB00005F0D2FB6561204638BD00BF8800002027
:10CFC00010B5044650B1406902F098F9002363613E
:10CFD000034B2046BDE810401B69184710BD00BF39
:10CFE00088000020002307B502A941F8040D054878
:10CFF0001A46406BFCF708FE431E5842584103B0E6
:10D000005DF804FB8800002007B502A941F8040D73
:10D01000054801230022406BFCF7F6FD431E5842F1
:10D02000584103B05DF804FB8800002007B50022DA
:10D03000054B02A941F8042D586BFCF73FFF0198FE
:10D0400003B05DF804FB00BF88000020064B10B55C
:10D05000DB6878209847044618B17822002105F053
:10D060007BFB204610BD00BF8800002070B5044641
:10D070000C4D0D482B68984794B1236E2BB12B684B
:10D080000A4898472B69206E9847206F18B102F024
:10D0900035F9002323672B692046BDE87040184707
:10D0A00070BD00BF880000200F8801082288010899
:10D0B0001FB50E4C0190A06BFDF7A0F8024638B9E1
:10D0C00003A9A06BFCF7FAFE10B10398FFF7CEFF9F
:10D0D000002301A91A46A06BFCF796FD20B94FF476
:10D0E00087710348F6F77CFD04B010BD880000206E
:10D0F00089870108F8B50423437003780646022B9C
:10D100000ABF104B04691C6BFFF7A0FF054620B94E
:10D1100040F21D110C48F6F763FD012733782F709C
:10D120006B7054B129467068A0472846FFF79EFFF0
:10D13000FA20FDF7F1FC3846F8BD2846FFF7B8FFA6
:10D140002046F9E78800002089870108F8B50378B0
:10D150000646022B08BF124B0F460CBF1C6B04691E
:10D16000FFF774FF054620B940F235110D48F6F778
:10D1700037FD02232B7033786F606B7054B12946F2
:10D180007068A0472846FFF771FFFA20FDF7C4FC3E
:10D190000120F8BD2846FFF78BFF2046F9E700BFC6
:10D1A0008800002089870108064A1378FD2BDFBF1D
:10D1B00000780549C8540133DABF012013700020FC
:10D1C000704700BFAD4C0020AE4B002038B1007856
:10D1D000032803D0431F584258417047012070472D
:10D1E000084B07B51B6808489847052302A800F8B4
:10D1F000013DFFF7D9FF0548FFF7D6FF03B05DF803
:10D2000004FB00BF88000020ED8C0108AC4B00201F
:10D210002DE9F04F00258FB0CDE905019DF860B0F4
:10D22000079202935D4557D2029B974F5E195B5D53
:10D2300096480393039A3B68013AD2B20E2A96BFEE
:10D240009349944A51F8222003999847039B033B42
:10D250000C2B00F25582DFE813F00D00DE013701E0
:10D26000EC009A0114021602C00153021802BA001F
:10D270001C024F020024ABEB0503DBB2824F089384
:10D280008DF82C40089A231D934202DA335D032B5C
:10D2900025D0ACB103230EA800F8083DFFF784FFAA
:10D2A0000BA8FFF781FF9DF82C107B4801F00103CC
:10D2B0000093754BC1F380021E68C1F34003B04771
:10D2C0002C44E4B2A54240F01D826F4BABEB05024B
:10D2D0001B680399714898470FB0BDE8F08F06EBC3
:10D2E000040999F80180A01C4FEA181130440991F3
:10D2F000FAF785F899F804900999C9F302130534EF
:10D30000062908F00F088246049309F00F09E4B2D9
:10D3100036D90F293B6839D19DF82C3043F00203F0
:10D320008DF82C3008F1FF32042A3B6831D9B8F16E
:10D330000F0F36D19DF82C3043F004038DF82C30BC
:10D340003B68B9F1000F06D04A4697F8A51054483B
:10D35000984787F8A590049A3B6832BB51465148DC
:10D360009847504600F044FF9DF82C3043F00103ED
:10D370008DF82C303B68524604994B48984781E71A
:10D3800087F898103B6849489847C5E74848984748
:10D39000C8E7424697F899104648984787F8998019
:10D3A000C8E7414644489847CAE7049A062AE1D1AB
:10D3B0004FF6FF713B4898474FF6FF7000F018FF9B
:10D3C0009DF82C3043F001038DF82C305AE7ABEB7D
:10D3D0000503DBB2052B40F21C8133780D2B40F0A6
:10D3E0001881701CF9F7FEFF079B8046012B4FF058
:10D3F000000913D11EA4D4E9003413EB08039846A6
:10D4000044EB0904A14605993B684246096D2B4847
:10D410009847059BC3E91489062451E7079B022B13
:10D4200003D015A4D4E90034E7E715A4D4E9003407
:10D43000E3E73378062B40F0EC800EA800F80C3DB3
:10D44000FFF7B2FE069B0EAC03F01F0204F8082D96
:10D4500097F8A6101A483E68B0471A48FFF7A4FE8E
:10D460002046FFF7A1FE01242AE700BFAFF30080AA
:10D47000813DD51200000000803DD5120000000063
:10D48000823DD5120000000088000020D8890108E4
:10D4900094890108D0890108C88A01085B8C0108B9
:10D4A0006B8A0108848A01089D8A0108F9890108AC
:10D4B0001A8A0108378A0108508A0108FE8A010881
:10D4C0001C8B01082E010020ABEB0503DBB2042B03
:10D4D00040F29F803478052C40F09B80D6F80120E4
:10D4E0003B680C9297F89A10C2F30212864898474C
:10D4F0009DF83020854EC2F3021387F89A303378B6
:10D5000002F00F0243F00403052A33703B682ED863
:10D5100097F89B107E4898479DF83030C3F303037B
:10D5200087F89B30337843F002030DF131003370FC
:10D530004FF06408F9F75BFF08FB00F84046FAF784
:10D540004BFD8146D0B1734E42463368D6F89C10ED
:10D55000714898476D4AC6F89C80137843F00103E0
:10D56000137001226D4B1A70FFF73AFEA8E61146C0
:10D570006B48984733786FF34103D6E73B684146E1
:10D5800068489847337869F300033370E9E7ABEBF9
:10D590000503DBB2052B3CD93478072C39D133464F
:10D5A00053F8010FF1781A793379090241EA0341FE
:10D5B000B3780C9019436423707859438DF8342064
:10D5C00000F098FD8DF828000EA800F80C4DFFF72C
:10D5D000EBFD0AA8FFF7E8FD1EE7ABEB0503DBB2A6
:10D5E000042B16D934780A2C13D16421D6F8010003
:10D5F000030A5943C0B200F0C5FD8DF82C000EA8F7
:10D6000000F8084DFFF7D0FD0BA8FFF7CDFD05246E
:10D6100056E6002454E6AC1CE4B20234E4B2023410
:10D62000E4B2ABEB0403DBB2012B30D9029A029BCC
:10D6300012F804902344B9F10C0F28D14FF0010ADD
:10D640005E7897F8A3104FEA16180AFA08F806F061
:10D650000F063B68424634480AFA06FA98473B6888
:10D66000524697F8A410314887F8A38098470EA82F
:10D6700000F8089D87F8A4A0FFF796FD02231C443C
:10D680001FE62C46C9E72C46C9E72C46C9E700230C
:10D69000F5E7EC1CE4B2ABEB0403DBB2012B2DD9B4
:10D6A000029A029B12F804802344B8F10F0F25D18F
:10D6B0005E78BB68984701223309C7E92A010A331B
:10D6C0000EA802FA03F306F00F0600F8088DC7F85B
:10D6D000B0308DF82C20C7F8B460FFF765FD0BA8BB
:10D6E000FFF762FD02231C44E4B23B68ABEB04028B
:10D6F00003990F489847E5E52C46CCE70023F2E76D
:10D700002C46F2E725468DE5408B0108AC4B002006
:10D710006F8B010888000020BD8B0108AD4B0020F5
:10D720009B8B0108EA8B0108118C0108368C0108DB
:10D730005B8C0108037A70B51B09D61804460F2EBE
:10D7400000F10C00154618440D4E0BDC04F0E0FF10
:10D75000237A0C4865F307132372294633689847E8
:10D76000012070BDC3F10F0204F0D2FF237A0648F6
:10D7700043F0F00323722946336898470020F0E70E
:10D7800088000020938C0108B78C010810B5044C68
:10D79000227822B10349FFF7CDFF0023237010BD8B
:10D7A000AD4C0020AE4B002030B585B0039104464F
:10D7B000174B30B91B78FBB105B0BDE83040FFF71F
:10D7C0000FBD00259DF90E109DF80F201D70FFF76D
:10D7D000FDFC88B10F48237A457F2DB113F0010578
:10D7E00018BF012580F8A1501B0907D0009304F150
:10D7F0000C032046FFF70CFD05B030BD637F002B06
:10D80000FAD1237F002BF7D00093A36CF1E700BF80
:10D81000AD4B00208800002010B5044678B1836A23
:10D82000012B0CD1C36A1BB90D210648F6F7D8F9B4
:10D83000E36A587802288CBF0020012010BD002028
:10D84000FCE700BFB48D01082DE9F04F06468BB010
:10D8500018B10378023B012B03D91F219648F6F734
:10D86000BFF973690BB11B781BB120219248F6F701
:10D87000B7F90025DFF88C929048D9F8002090473E
:10D8800099F89B3099F899800393D9F89C3099F8CE
:10D8900098B0049399F89AA000F0ACFB00F0B2FBAA
:10D8A0000AAA42F80C5D86494046FEF7F9FA4C4652
:10D8B000074640B98348D9F8003098473046FFF70B
:10D8C00019FC01270AE0079BCBB1FEF78FFA0799F5
:10D8D000042907D93046FFF739FC2F4638460BB0EC
:10D8E000BDE8F08FD9F80030774898470798774B14
:10D8F00043434FF47A70B3FBF0F0FDF70DF9B368D2
:10D900000133012BB36009D1D4F88C300133C4F852
:10D910008C306F4B5B699847A4F88000B4F8803076
:10D9200094F89B500133A4F88030002384F89B3096
:10D93000089309AB019308AB0093394641F2707329
:10D9400041F288327069FFF737FA074658B9236801
:10D95000604898473046FFF7CDFB089801F0CEFCB1
:10D9600084F89B50ADE7089A84F89B50236812B165
:10D970001278012A08D0584898473046FFF7BAFB7A
:10D98000089801F0BBFCA9E754489847236854481D
:10D990009847089BE16BDA685248E263236898472E
:10D9A000089BDFF864C103F1320203F1420E6546C1
:10D9B00010685168083203C57245AC46F7D14A4D2C
:10D9C00003F122023233AC46106851680832ACE8E9
:10D9D00003009A426546F6D1236894F85F2094F8D4
:10D9E000501042489847236894F84F2094F840100C
:10D9F0003F489847089BE16A9A683E48E26223687C
:10DA00009847089B94F89B101A7C3B48C2F303028A
:10DA100084F89B2023689847089B94F89A101A7CF6
:10DA20003648C2F3021284F89A20236898470023EC
:10DA3000D4F88C10C4E92433C4F88C302268304800
:10DA4000059390470898123000F012FC2268234892
:10DA50009047FEF7CBF9012284F82A20FFF7F6FA67
:10DA6000054658227169183004F052FE089A059B49
:10DA70002A6794F82A206B722B662A752B709DF802
:10DA80000C203378EA736B70049A236B85F80CB022
:10DA900085F80D8085F80EA02A614BB12946706883
:10DAA00098476420FDF738F82846FFF7DFFA15E7B6
:10DAB0002846FFF7FDFA11E7B48D0108EF8D010844
:10DAC00019D800080F8E01086994010840420F0020
:10DAD000247A0108458E01087F8E0108B58E010861
:10DAE000FD8E0108248F0108C8000020508F010816
:10DAF0008E8F0108CC8F0108F98F0108279001084B
:10DB00005890010888000020D800002028B1836ABE
:10DB1000012B01D1007B7047002070472DE9F341B4
:10DB20000546414C414A424823680E4600290CBF35
:10DB3000014611463F48984723683F489847696C1B
:10DB400023683E4898472B783D48072B96BF3D4AAF
:10DB50003D4952F8231027686A78B84723683B4844
:10DB600098472368697F3A4898472368297F39484E
:10DB7000984723686989384898472368696837480F
:10DB80009847297A0B090193C1F3C003009336B378
:10DB9000C1F38003C1F34002266801F0010130485F
:10DBA000B0472B7A13F0F00F3BD023682D486FF06D
:10DBB0000B079847DFF8B88005F10C067F1B297A20
:10DBC000BA19B2EB111F236804DB274802B0BDE885
:10DBD000F041184716F8011B40469847EFE7C1F39C
:10DBE0008003C1F34002266801F001011F48B047DD
:10DBF0002B7A13F0F00F14D023681A486FF00B073C
:10DC00009847DFF86C8005F10C067F1B297ABA195A
:10DC1000B2EB111F2368D8DA16F8011B404698476B
:10DC2000F4E702B0BDE8F08188000020A890010868
:10DC3000AF900108B8900108D4900108EA9001085B
:10DC4000F990010888900108548201080D9101089B
:10DC50001A910108309101084F910108679101085C
:10DC600080910108C5910108C6630108D59101089A
:10DC70001E67010870B5114C0546637FEBB1037A4E
:10DC8000266843F00103037294F8A32094F8A210CD
:10DC900094F8A4300A48B04794F8A21094F8A3204E
:10DCA00091420AD92B7A246843F002032B72A446CE
:10DCB000BDE8704001230348604770BD8800002024
:10DCC0009C920108DC92010837B5164C10B1002374
:10DCD00084F8A230637F13B394F8A21094F8A320C1
:10DCE00091421CD994F8A4308D1A95FBF3F003FBF4
:10DCF0001050A0B90C482568A84700F08BF920B94E
:10DD000000F096F908B900F0A3F9A07F94F89830D4
:10DD1000E27F94F89910009024680448A04703B06B
:10DD200030BD00BF88000020179201086D920108E5
:10DD30002DE9F04F044689B010B10378012B03D0D0
:10DD4000A6218848F5F74CFF63691BB9A7218548D0
:10DD5000F5F746FF63691B78042B05D0022B03D02F
:10DD6000A8218048F5F73CFF0027DFF820927E4885
:10DD7000D9F80020904799F89B3099F89980029340
:10DD800008AAD9F89C3042F80C7D7849404699F8A9
:10DD900098B099F89AA00393FEF782F84D4606468C
:10DDA00058B9D9F80030724898472046FFF7A2F9D1
:10DDB0000126304609B0BDE8F08F059BB3B1FEF7F0
:10DDC00015F80599042904D92046FFF7BFF9002664
:10DDD000EFE7D9F80030674898470598664B43430A
:10DDE0004FF47A70B3FBF0F0FCF796FEA3680133B2
:10DDF000012BA3600FD1D5F88C3060690133C5F8D1
:10DE00008C3095F8A230013385F8A230FFF732FF4D
:10DE10006069FFF7BBFCEB6B60694360D5F88C3041
:10DE2000438195F8A03033B1002385F8A030037A00
:10DE300043F00403037200270121FFF76FFE07ABD5
:10DE4000019306AB009331464FF4FA634FF47A72B4
:10DE500060690697FEF7B0FF064610B92B68474881
:10DE6000A2E7FCF707FDE060069848B13946FFF7E6
:10DE700055FE069B1B78052B04BF012385F8A030B7
:10DE80000698FFF721FFDDE90601FFF78DFC069AF2
:10DE9000002A61D0137A13F0040707D037462B68A5
:10DEA00051893748984795F8A530A360069B33B150
:10DEB00063691B78022B04BF95F8A530A360FFF7B8
:10DEC000C5F8814620B940F207112648F5F788FECB
:10DED0005822616909F1180004F01AFC0022069921
:10DEE0009DF80830C9F87010217889F80920C9F820
:10DEF000602089F8002095F82A2089F80F3089F8E9
:10DF00001420039B226989F80CB089F80D8089F8E8
:10DF10000EA0C9F8103089F8011089F80870EAB12C
:10DF20004946606890476420FCF7F6FD4846FFF7D5
:10DF30009DF895F8A520A1682F681248B84795F874
:10DF4000A520A1689142BFF434AF2A680E489047DB
:10DF5000032289F800203AE71746A7E74846FFF76B
:10DF6000A7F8E6E7CB9301080A9401080DDB000847
:10DF70002E9401086894010840420F00969401080D
:10DF8000D4940108F09401080D9501088800002040
:10DF9000437882781B02007843EA024303430A2055
:10DFA000B3FBF0F07047000038B5044681B10D783E
:10DFB00084B1A36A012B0DD1E36A1BB95321064832
:10DFC000F5F70EFEE36A5878431B5842584138BDB6
:10DFD000FF25EDE70020FAE758950108044B93F878
:10DFE000202083F89B205A6AC3F89C20704700BF0A
:10DFF00088000020024BDA7F83F89920704700BF29
:10E0000088000020024B9A7F83F89820704700BF59
:10E0100088000020054BDA7F93F8991091423ABFAF
:10E02000012083F899200020704700BF880000205D
:10E03000064A92F89830917F99423DBF03F1FF3331
:10E04000012082F898300020704700BF880000202F
:10E0500010B5FFF7C3FF0120FEF7FEF85023164C62
:10E06000012123700023224614486370FEF76EF8E6
:10E0700018B931211248F5F7B3FD50230121114A97
:10E080001148A370E170FEF761F818B935210C480A
:10E09000F5F7A6FD5023237102230C4A01210C48F9
:10E0A0006371FEF753F828B9BDE8104039210448E0
:10E0B000F5F796BD10BD00BF98500020043F0D003D
:10E0C000589501089A500020CC3F0D009C5000202C
:10E0D00094400D0007B502A901F8010D0448FDF7B1
:10E0E000AFFE08B1FDF7F6FF03B05DF804FB00BF1B
:10E0F000A9DF00082DE9F8431746C7F30312052AE4
:10E10000044689464FF000052FD91A4B07F00F013E
:10E110001B68194898474FF000084FF47A76B9FB0E
:10E12000F6F63046FDF78AFF08B10F2C20D9114BC7
:10E1300049461B6811489847002368F3000563F3BC
:10E14000410505F00303032B0CD12046FFF7C2FF66
:10E150000B4B012103EB4402547003F8147030465A
:10E16000FDF7F4FF2846BDE8F8834FF00108D4E737
:10E170000123E2E788000020DA950108FA950108FA
:10E18000985000200F282DE9F04105460F461FD872
:10E19000164B03EB40035C78231A5C425C414FF45E
:10E1A0007A78B7FBF8F0FDF749FF4FF0000360F312
:10E1B000000364F3410303F00303032B064609D075
:10E1C0004FF0000066F3000064F34100BDE8F08109
:10E1D0000024E4E72846FFF77DFF044A012102EB13
:10E1E000450208FB07F0FDF7B1FFE9E79850002072
:10E1F0002DE9F743194D01462B6804461848984706
:10E200000023184FDFF86080DFF860908DF807304A
:10E210009DF807300F2B02D903B0BDE8F0830DF154
:10E2200007013846FDF70CFE064648B1E2072B68A9
:10E230009DF807100BD5484698473046FDF728FF54
:10E240009DF80730640801338DF80730E0E7404659
:10E2500098473046FDF7FAFEF2E700BF880000203D
:10E2600095950108A9DF0008C2950108AB95010842
:10E2700038B504460320FFF72DFF0420FFF72AFFDF
:10E280000520FFF727FF0620FFF724FF0720FFF7F1
:10E2900021FF2046FFF77CFE0546FDF7CFFE48B183
:10E2A0005023294A012193710323063253702846D3
:10E2B000FDF74CFFE01CFFF76BFE0546FDF7BEFEC9
:10E2C00048B15023204A01211372042308325370AD
:10E2D0002846FDF73BFFA01DFFF75AFE0546FDF758
:10E2E000ADFE48B15023184A0121937205230A322A
:10E2F00053702846FDF72AFF04F10900FFF748FE96
:10E300000546FDF79BFE48B150230F4A01211373C8
:10E3100006230C3253702846FDF718FF04F10C0059
:10E32000FFF736FE0446FDF789FE58B15023064A32
:10E33000204693730723D3730121BDE838400E3282
:10E34000FDF704BF38BD00BF985000200738C0B2A9
:10E3500005289ABF014B185C0820704733950108C7
:10E3600006289ABF014B185C0020704739950108B8
:10E37000052804D90628034818BF00207047024822
:10E38000704700BF90D0030048E80100052810B591
:10E39000044604D940F237110348F5F721FC034B3A
:10E3A00013F9240010BD00BF5895010840950108DD
:10E3B000142810B504460FDD4FF49E710D48F5F793
:10E3C0000FFC0A2C10DD0C2C10DD0E2C10DD152C92
:10E3D000B4BF0020062010BD062803DD0828F0DCAD
:10E3E0000420F8E70520F6E70320F4E70220F2E72F
:10E3F0000120F0E7589501080F280DD8DFE800F05C
:10E400000D0D0D080F0F0F0A0A0C0C0C0C0C0C0A4A
:10E410007320704700207047704733207047DE201C
:10E4200070470000000000002DE9F04F8DB01E463F
:10E43000169F434B81469F428A46934608D0414BE4
:10E440009F4203D0A5214048F5F7CAFB002100E018
:10E4500001213E4D0B91EB6A9847EB685046984777
:10E46000B9F1010F4FF000040A95DFF8EC800B9929
:10E4700033D108230A22CDE90132AB6932461D4669
:10E4800002204B46CDE90899CDE90644CDE9044484
:10E4900003940094A8472146FF20F9F7EFF950466E
:10E4A000F2F7D0FEF2F7C0FD23A3D3E9002306F074
:10E4B000B7FED8F80030CDE900013A46314624488D
:10E4C00098470820F9F7D0F9342139200A9B1B6CB2
:10E4D0000A930DB0BDE8F04F18474FF47A634FF040
:10E4E0000109CDE907430823CDE901930A9B2246A0
:10E4F000DB69CDE905441D46CDE903490B4600968D
:10E5000059460220A8474946FF20F9F7B7F9504677
:10E51000CDF808B0F2F796FEF2F786FD06A3D3E930
:10E52000002306F07DFED8F80030CDE900013A4620
:10E53000314608489847C4E70000000080842E4117
:10E5400090D0030048E8010020960108247A0108D1
:10E550005A9601088D960108880000202DE9F7439E
:10E560000546104614460F469946FFF701FF8046C0
:10E570002046FFF7F5FEC6B21EB9C8210C48F5F7D4
:10E580002FFB95B94846FFF701FF0246334639464F
:10E590002846CDF80080FFF747FF2146054B064887
:10E5A0001B6803B0BDE8F04318470022EEE700BF48
:10E5B0002096010888000020139601080A68036865
:10E5C000534003604A684368534043608A688368E5
:10E5D00053408360CA68C3685340C36070470B6888
:10E5E00010B514686340036054684B68634043602F
:10E5F00094688B6863408360CB68D2685340C36083
:10E6000010BD0000A1F11003DBB2102B2DE9F04783
:10E610000C46154608D84FF0010909FA03F303F038
:10E62000013323F080732BB90023FF2085F8F030ED
:10E63000BDE8F0870A460146284604F069F804F16F
:10E640001C0E4FEA8E0E5FFA8EFE4FEA1E13013B40
:10E6500085F8F03023462749B3FBF4F204FB12326D
:10E66000E81812F0FF0210F804AC10F803CC10F810
:10E67000027C10F8016C32D111F80C804FEAD912EB
:10E6800089EA080811F807C08F5D11F80A604FEA9F
:10E69000420A5244C24602EBC20282EA49025FFACF
:10E6A00082F91A1BD2B215F802802A448AEA080AB3
:10E6B00005F803A092F8018004338CEA080C80F876
:10E6C00001C092F802C0DBB287EA0C078770D278EB
:10E6D0009E4586EA0206C670BED80020A8E7182C20
:10E6E000DFD9102A01BF11F80AA011F80CC0CF5DC4
:10E6F0008E5DD6E7CC9D01082DE9F04F92F8F03001
:10E70000A1B01A911892002B00F05D8101461CA85F
:10E71000FFF765FF4FF00108AC4CAD4DAD4E189BB7
:10E720009DF875E003EB081319939DF870309DF880
:10E730007AA00093009A9DF87F90A05C9DF87420C9
:10E7400014F80A100192019F9DF87920E75D02926A
:10E750000697029F9DF87E20E75D03920797A25CD3
:10E760009DF87870049208979DF873209DF87D704D
:10E77000059214F8093014F80EC0A25C09979DF8B0
:10E7800072700A97E75D0B979DF877700C97E75DBD
:10E790000D97089FE75D0E97099FE75D0F979DF81E
:10E7A0007C7010979DF8717011979DF87670129794
:10E7B000E75D13979DF87B701497E75D1597109FA1
:10E7C000E75D1697119FE75D1797189F97F8F07010
:10E7D00047453ED88DF870009DF818008DF87210EE
:10E7E0008DF874009DF82C109DF838008DF87A1083
:10E7F0008DF878009DF810109DF858008DF876106F
:10E800008DF87C009DF84C109DF81C008DF87E1052
:10E810008DF875009DF854109DF83C008DF87F1020
:10E820008DF879009DF834109DF85C008DF87B1010
:10E830008DF87D008DF877201A98199A1CA98DF80B
:10E8400071C08DF87330FFF7CAFE002021B0BDE81B
:10E85000F08F81EA03071B97009F434015F807B02C
:10E860001B9F80EA0C008BEA070716F80EB081EABE
:10E870000C0187EA0B078DF8707015F80E707B405D
:10E8800016F80A707B408DF8713015F80A30584040
:10E8900016F809305840009B8DF8720016F803C036
:10E8A000049B8CEA010115F809C0534081EA0C0170
:10E8B0008DF8731001991CA8695C4B400299715C3A
:10E8C0004B408DF87430069B5A40029BEB5C5A40DB
:10E8D000039BF35C5A408DF87520DDE90632534006
:10E8E000039AAA5C5340059AB25C53408DF8763087
:10E8F000079A049B5340019AB25C5340059AAA5C64
:10E9000053408DF877300D9A0B9B5340089AAA5CC0
:10E910005340099AB25C53408DF87830DDE90D32EE
:10E920005340099AAA5C53400A9AB25C53408DF84E
:10E930007930DDE90E3253400A9AAA5C53400C9AB2
:10E94000B25C53408DF87A300B9B0F9A5340089A73
:10E95000B25C53400C9AAA5C53408DF87B30159AF8
:10E96000139B5340109AAA5C5340119AB25C5340D7
:10E970008DF87C30DDE915325340119AAA5C534082
:10E98000129AB25C53408DF87D30DDE91632534067
:10E99000129AAA5C5340149AB25C53408DF87E30B0
:10E9A000179A139B5340109AB25C5340149AAA5C76
:10E9B000199953408DF87F30FFF700FE08F10103ED
:10E9C0005FFA83F8ABE6FF2040E700BFCC9D01086B
:10E9D000CC960108CC9701082DE9F04F924692F8A9
:10E9E000F02091B00B91002A00F094810AEB021202
:10E9F00001460CA8FFF7F3FD314C9DF830309DF82F
:10EA00003920E35CA25C8DF830309DF834302D4D18
:10EA1000E35C2D4E8DF834309DF83830E35C8DF892
:10EA200038309DF83C30E35C8DF83C309DF83D304B
:10EA30008DF83D209DF83520E35CA25C8DF83920EF
:10EA40009DF831208DF83130A25C9DF832308DF880
:10EA500035209DF83A20E35CA25C8DF83A308DF8C1
:10EA600032209DF83E209DF83630A25CE35C8DF8A4
:10EA700036209DF837208DF83E30A25C9DF833306B
:10EA80008DF833209DF83B20E35CA25C8DF83720A5
:10EA90009DF83F208DF83F30A25C8DF83B209AF81E
:10EAA000F020013AD2B20AEB0218D0450ED10B98F1
:10EAB00042460CA9FFF793FD002011B0BDE8F08F8E
:10EAC000CC9C0108CC9B0108CC99010841460CA8BC
:10EAD000FFF774FD9DF836309DF8319000939DF856
:10EAE00037308D4A01939DF838309DF833E002931A
:10EAF0009DF839309DF834C003939DF83A309DF865
:10EB0000357004939DF83B30A8F1100805939DF8EB
:10EB10003C3006939DF83D3007939DF83E300893B6
:10EB20009DF83F3009939DF8303018469DF83230FB
:10EB3000295C0A9316F8093059400A9BD35C594066
:10EB4000764B13F80EB081EA0B01615C13F800B04C
:10EB50008DF8301015F809108BEA010B0A99715CD9
:10EB60008BEA010112F80EB081EA0B01615C12F828
:10EB700000B08DF8351013F8091012F809908BEADF
:10EB8000010B0A99695C8BEA010116F80EB081EA63
:10EB90000B01615C8DF83A10315C0A9881EA090139
:10EBA00013F80090019881EA090115F80E9015F804
:10EBB0000CE081EA0901615C8DF83F10F15D8EEA9D
:10EBC000010E0099515C8EEA010113F800E081EA20
:10EBD0000E01615C13F80CE08DF83410E95D8EEAEB
:10EBE000010E0099715C8EEA010112F800E081EAE1
:10EBF0000E01615C12F80CE08DF83910D95DD75D1B
:10EC00008EEA010E0099695C8EEA010116F800E0B7
:10EC1000009881EA0E01615C8DF83E1016F80C1028
:10EC200079401F5C019879402F5C7940615C8DF8D8
:10EC300033100299685C0399715C48400499515CF7
:10EC400041400598185C4140615C8DF8381002998C
:10EC5000585C0399695C48400499715C414005988F
:10EC6000105C4140615C8DF83D100299505C039945
:10EC7000595C48400499695C41400598305C4140CA
:10EC8000615C03988DF832100299105C715C414010
:10EC90000498185C48400599695C4840215C0798D5
:10ECA0008DF837100699695C305C41400898105C1B
:10ECB00041400998185C4140615C07988DF83C1010
:10ECC0000699285C595C41400898305C414009989D
:10ECD000105C4140615C07988DF831100699185C12
:10ECE000515C41400898285C41400998305C4140A3
:10ECF000615C07988DF836100699125C715C4A4089
:10ED000008995B5C5340099AAA5C5340E35C8DF818
:10ED10003B30CAE6FF20D0E6CC9A0108CC98010827
:10ED200010B5102204460021F13003F015FD00213A
:10ED30002046C4F81411F022BDE8104003F00CBDC9
:10ED40000B46024610211846FFF75CBC2DE9FF4731
:10ED50000446D0F814010E46154604F2011910B30A
:10ED6000C0F110089045474628BF174648443A4628
:10ED700003F0CEFCD4F814313B440F2BC4F814310B
:10ED80001CD9A8451AD204F1F10319461A78187C47
:10ED9000424003F8012B4B45F8D122460846FFF7C5
:10EDA000ABFC3E44ED1B0DF1100A102D09D82A468C
:10EDB0003146484603F0ACFCC4F8145104B0BDE839
:10EDC000F08704F1F002731E06F10F0013F8017FC3
:10EDD00012F8011F834281EA07011170F6D16A46D9
:10EDE00004F1F103984617469446186859680833A9
:10EDF000ACE803004B456246F6D122463946384618
:10EE0000FFF77AFC43463A4603CA524518605960F8
:10EE1000174603F10803F6D11036103DC5E7F0B5EB
:10EE20000C4689B0102200210546684603F094FC88
:10EE3000224669466846FFF75FFC9DF900306A4646
:10EE4000002B0DF10F013EDA137812F8010F5B0071
:10EE50005BB243EAD013914202F8013CF4D19DF831
:10EE60000F305B0083F087038DF80F30D4F8143136
:10EE7000102B37D1002304F2011211781DF8030082
:10EE800001334140102B02F8011BF6D104F1F102CD
:10EE9000134604F201171178107C414002F8011B5F
:10EEA0009742F8D104AA9446164618685968083360
:10EEB00003C6BB423246F7D1224629466046FFF7D9
:10EEC0001BFC09B0F0BD137812F8010F5B005BB2B8
:10EED00043EAD0138A4202F8013CF4D19DF80F3086
:10EEE0005B00C1E79DF900206846002A28DA027815
:10EEF00010F8016F520052B242EAD612814200F875
:10EF0000012CF4D19DF80F20520082F0870280215D
:10EF10008DF80F20E21882F80111002201330F2B27
:10EF20001DD9C4F81431002304F2011211781DF820
:10EF3000030001334140102B02F8011BF6D1A5E775
:10EF4000027810F8016F520052B242EAD6128142A2
:10EF500000F8012CF4D19DF80F205200D7E7E118FA
:10EF600081F80121DAE770B51025CEB00C460646CF
:10EF70002A460021684603F0EFFB49238DF8003054
:10EF8000A37B08A88DF80530D4F80A301A0A8DF84A
:10EF900006308DF8072023FA05F21B0E8DF8093094
:10EFA00023698DF808201A0A8DF80A308DF80B2095
:10EFB00023FA05F21B0E8DF80D3023898DF80C20F5
:10EFC0008DF80F30FFF7ACFE216808A8FFF7B8FEF8
:10EFD0002A46694608A8FFF7B9FE2289616808A891
:10EFE000FFF7B4FE08A90DEB0500FFF718FF049B1F
:10EFF00033604EB070BD30B50C46CBB0054604A8AA
:10F00000FFF78EFE216804A8FFF79AFE2289616847
:10F0100004A8FFF79BFE04A96846FFF700FF009BCA
:10F020002B604BB030BD70B50C89BEB006460D46A6
:10F03000A4B114F00F0411D101AA10212868FFF720
:10F04000E1FA2889A04201DC3EB070BD6868311940
:10F05000204401AAFFF7C0FC1034F2E74FF0FF3064
:10F06000F2E770B50C89BEB006460D46A4B114F0A7
:10F070000F0411D101AA10212868FFF7C3FA2889CB
:10F08000A04201DC3EB070BD68683119204401AA7D
:10F09000FFF732FB1034F2E74FF0FF30F2E72DE9D3
:10F0A000F0430D89C7B080460E46002D5BD0012489
:10F0B0001022002101A803F04FFBB37B05F00F07DE
:10F0C0008DF80930D6F80A302D091A0A8DF80A3061
:10F0D0008DF80B201A0C1B0E8DF80D3033698DF84E
:10F0E0000C201A0A8DF80E308DF80F201A0C1B0E0A
:10F0F0008DF81130736801358DF804408DF81020BB
:10F1000003F1FF39AC4203DD308947B0BDE8F0833D
:10F1100009AA102130688DF81340FFF773FA09AA85
:10F1200005A901A8FFF7E8FAAC4211DB002F14BFD4
:10F130003B4610234846424643440DF1130C93428C
:10F1400008D80134A4B208F1100809F11009D9E770
:10F150001023EFE710F801EF1CF8011F81EA0E0100
:10F1600002F8011BEBE74FF0FF30CEE770B5C2B0FD
:10F17000144606460D46F122002105A803F0ECFADC
:10F180000023CDE90333636810218DF805301A0A96
:10F190001B0C8DF80730A3688DF806208DF8083019
:10F1A0001A0A1B0C8DF80A30A3898DF809208DF8F6
:10F1B0000B301B0A8DF80C30012305AA20688DF84E
:10F1C0000430FFF71FFA05AA314601A8FFF794FAA9
:10F1D000022305AA102120688DF80430FFF712FAE7
:10F1E00005AA294601A8FFF787FA42B070BD00685A
:10F1F000704782B0034660B16A4659680068013BB7
:10F2000003C207221DF8021012F1FF3203F8011F9A
:10F21000F8D202B070470FB404B0704730B585B073
:10F220006D4685E80F00104C95E80F0084E80F004C
:10F2300004F1100208A903C982E803000BB90B4BC3
:10F24000E360A3680BB9094BA36063680BB1236843
:10F2500033B9A36806489847064B6360064B2360A2
:10F260000123237605B030BDB04C002017F2000812
:10F27000F49E0108C1260108B12601082DE9F041DC
:10F28000194E8046337E0D462BB96821174B184A1C
:10F29000184803F0F9F8DE2903D9174B144A6921FD
:10F2A000F6E7336858209847044680B15822002179
:10F2B00003F052FAB8F1000F12D08DB1336828462E
:10F2C0009847074630B92046736898473C46204621
:10F2D000BDE8F0812A46414603F01AFA2577A76473
:10F2E00000236370F3E700BFB04C0020CC9E010800
:10F2F00061A10108D99E0108E69E010870B50B4C7A
:10F300000546237E2BB90A4B0A4A84210A4803F09A
:10F31000BBF850B1806C636810B198470023AB64B0
:10F3200063682846BDE87040184770BDB04C0020A7
:10F33000CC9E010873A10108D99E01082DE9F04374
:10F340001746B44A91B0137E05460C4690462BB939
:10F350009C21B14BB14AB24803F096F8032F04D870
:10F360000026304611B0BDE8F0830178437843EAC7
:10F37000411323700378022B01D0042B69D10023A1
:10F38000042F8DF81630EBD06B6863706B681B0A26
:10F39000A370EB88E370EB7923716B68CDF81230C2
:10F3A0009DF81630002B40F00081052FD8D02A7A26
:10F3B000C2F3400302F001019B0143EAC11343EA97
:10F3C0001213C2F3800243EA4213062663712A7ABB
:10F3D0001209731C9F42C3DD6989DBB2A15569899B
:10F3E0000236090AE1546B89069352B106EB020911
:10F3F0004F45B5DBA01905F10C0103F089F95FFA5F
:10F4000089F62B7F002B00F0F080BE42A8D26B7FE4
:10F4100006F10109A3556A7F5FFA89F9D8F814301B
:10F42000002A40F0E08004330293AB6C02A90393FE
:10F430002B7F04EB0900ADF81030FFF730FE484495
:10F44000C6B2B74280F0D180764B744A40F2551173
:10F4500081E7032B01D0052B01D1012390E7C3BB2A
:10F46000082F7FF67DAF5669601C324652F8343F54
:10F47000C4F8013053684360FFF7BBFE102F7FF6DE
:10F480006FAF324652F83C3F04F10900C4F809302E
:10F4900053684360FFF7ADFE122F7FF661AFB6F8F9
:10F4A000443002A96374B6F8443001A81B0AA3745F
:10F4B00013232436CDE90264ADF81030FFF79BFD2D
:10F4C000162F7FF64DAF019B1726C4F813306B64DF
:10F4D00047E7012B7FF444AF4368637043681B0A1E
:10F4E000A370C388E3708368237183681B0A637108
:10F4F0004389A371C368E371C3681B0A2372C3897C
:10F500006372C37BA372037C03F07002C3F3030333
:10F510001343E372437C237390F82130002B42D0D5
:10F52000034633F8122F1C26A4F80D209B78E373B2
:10F53000034633F8152F22829B78A374034633F8D1
:10F54000182FA4F813209B786375034633F81B2FFC
:10F55000E2829B78237635F81E3FA4F81930AB7809
:10F56000E376D8F8143002A9243301A8CDE9023497
:10F57000ADF81060FFF73FFD019B02A9A351D8F839
:10F5800014300436243302930134731E07A8039405
:10F59000ADF81030FFF747FDBDF8102007A9204651
:10F5A00003F0B6F8DDE60D26DBE72B78032B01D060
:10F5B000052B15D1052F3FF4D3AE2A7AC2F34003B1
:10F5C00002F001019B0143EAC11343EA1213C2F3A3
:10F5D000800143EA4113C2F3C00243EA0213F4E696
:10F5E00000220526F5E614331EE7F31C9F427FF741
:10F5F000B7AED8F8143002A9043301A8CDE902341B
:10F60000ADF81060FFF7AFFC019BA3510436F6B2D2
:10F61000A7E600BFB04C0020CC9E010888A10108DD
:10F62000D99E0108726801082DE9F047DFF894823D
:10F6300094B098F8189006460F464546B9F1000F69
:10F6400006D1934B934A40F27111934802F01CFF8C
:10F65000022926D9D8F8003058209847044638B9EE
:10F66000D8F80C308D489847204614B0BDE8F08794
:10F670005822002103F070F896F800A04FEA5A1AB9
:10F6800084F800A03378BAF1070F03F00303637026
:10F6900009D1D8F80C3082489847D8F80430204671
:10F6A00098470024E0E7BAF1050F00F29D81DFE8FA
:10F6B0001AF06B01B3000600060006000600701C7D
:10F6C000FFF795FD6060F379B279717942EA032220
:10F6D000D8F81430A7F104080433ADF82080BAF14B
:10F6E000040F6281CDE90636CDF822004FEAD11E23
:10F6F0002869237A4FEA611C02D0BAF1020F34D193
:10F700004FF0000A6EF300034FEAA11E6EF34103AF
:10F710006CF382034FEA211C6CF3C30361F30713FC
:10F720008DF826A000682372030C80B2904284BF3B
:10F7300001339BB202EB034206EB08000A92FFF78B
:10F7400056FD06A9606401A8FFF70DFC019B626CE1
:10F7500093421DD053485449EE68B9F1000F08BFD9
:10F7600001465248B0476B6899E74FF001096EF3C4
:10F7700000036CF382034FEA211C6CF3C30361F3B3
:10F7800007138DF8269040684FF000092372CBE7ED
:10F7900094F8089006F108014FEA19194A4604F155
:10F7A0000C0002F0B5FF09F10C039F4230D909F1BA
:10F7B0000802B25C09F10D039F42627704D1002375
:10F7C0003B482377EB684EE709F10909A8EB0900EC
:10F7D000C0B220776B696AB904334E44069307962A
:10F7E000ADF820002B689847A06428B9EB68314831
:10F7F0009847B8E71433F0E706A9FFF750FC002854
:10F800003FF732AFEB682C4898476B68A06CEFE786
:10F8100000232377A36427E7112F1BD1002384F84B
:10F8200021306B691FFA87F824330693731C079302
:10F8300008F1FF33ADF82030337806A90DF12D0023
:10F840008DF82C30FFF70DFC00280BAE07DCEB68C1
:10F850001A48CDE7212F40F099800123DFE7381FB8
:10F860003044FFF7C4FC6B6960642433A8F10408DA
:10F8700006A901A8CDE90636ADF82080FFF7BBFB4D
:10F88000636C019A9A421FD0EB680D48B0E700BF45
:10F89000CC9E01089EA10108D99E0108319F010854
:10F8A000499F0108289F0108219F0108779F0108AF
:10F8B000BC9F0108F09F010822A0010898A0010840
:10F8C000BCA00108B04C00209DF82F109DF82E30F0
:10F8D000090441EA03219DF82D300DF1330019434D
:10F8E00061609DF832309DF831201B0443EA022309
:10F8F0009DF830201343A360FFF779FCE0609DF88A
:10F900003700227CC60966F3C712061166F3061299
:10F9100060F3030222749DF83820627494F8212069
:10F9200002B314AA32F8170D92786082227514AAD5
:10F9300032F8140D9278A4F81500E27514AA32F882
:10F94000110D92782083A27614AA32F80E0D9278C7
:10F95000A4F81B00627714AA32F80B0D9278E083AA
:10F9600084F820206A69049302F12400B2F844303C
:10F97000CDE9020102AA04F1320104F12200ADF83E
:10F980001430FFF7F3FB6FE6172F02D0EB6818482F
:10F990002EE706F11300FFF72AFCD8F81430606454
:10F9A0002433CDE90636132306A901A8ADF820308B
:10F9B000FFF721FB636C019A9A4203D0D8F80C3010
:10F9C0000C4815E7324652F8013F636053683246EF
:10F9D000A36052F8093FE36053682361B27C737CF3
:10F9E00043EA0223A3823FE6D8F80C300248FFE640
:10F9F00048A00108F1A0010827A1010810B504469C
:10FA000001680748F7F7C6FB616831B10B7823B18D
:10FA10000448BDE81040F7F7BDBB0348F9E700BF55
:10FA2000B6A10108BBA10108C663010810B10121FC
:10FA300001F064BE704708B1F7F73EBC70478068BC
:10FA40007047406870474368012B08D1D0E9043201
:10FA5000934204D01878003018BF0120704700206E
:10FA600070474B6870B5042B04460E464FF00003F8
:10FA700004D0C0E900338360204670BDD1E904257D
:10FA8000AD1AC0E9003383602846FFF7D4FFC4E90C
:10FA900000000544A560D6E90453024629468B427E
:10FAA00005D00AB10E78167001310132F7E75B1B01
:10FAB00018446060E0E742680346022A06D1D3E9B1
:10FAC00004031B1A032B01D9F7F78ABC00207047E7
:10FAD0004368032B06D1D0E904329A4208BF0023C1
:10FAE000184670470023FBE7037870B58168044629
:10FAF000B3B1284A2848F7F74DFB6368022B12D1AF
:10FB00002046FFF7D8FF01462448F7F743FBE1689A
:10FB10000B78002B3CD02248BDE87040F7F73ABB89
:10FB2000204A2148E7E7032B05D12046FFF7D0FF05
:10FB300001461E48E9E7042B0ED100251C4ED4E9EE
:10FB40000431C91A8D4205D2595D3046F7F722FBC0
:10FB50000135F4E71748D8E7012B08D12046FFF715
:10FB600072FF1549154B002818BF1946E1E700251B
:10FB70000F4ED4E904239B1A9D4205D2515D3046B5
:10FB8000F7F708FB0135F4E70D48F7F703FBBEE78D
:10FB90000C48C1E71C5F010824A2010838A2010833
:10FBA000BBA10108C76301082EA201086EAB0108C2
:10FBB0001E67010842A20108D36D01081FA20108B7
:10FBC00048A20108C6630108B1F5705F2DE9F8434A
:10FBD00004460F4602D9174801F066FD066883689F
:10FBE0009B1B994219D9D0F804900846FFF723FFD0
:10FBF00005460346A9EB0608B14505D00BB132789E
:10FC00001A7001360133F7E72068FFF70FFF05EBA5
:10FC1000080325603D446360A56025683DB928461A
:10FC2000C4E90155FFF702FF2846BDE8F88301202B
:10FC3000FBE700BFC2A101082DE9F0410368561A95
:10FC4000904682680446D21A96420D4615D930462F
:10FC5000FFF7F1FE07460346A84505D02A7803B111
:10FC60001A7001350133F7E720683E44FFF7DEFEE6
:10FC7000C4E901662760BDE8F0814768481EFF1AA5
:10FC8000BE420ED81A469D19A91A002904DD10F8A3
:10FC9000011F02F8011BF7E7002EA8BF9B19636044
:10FCA000E9E73D441F44FA1A002A04DD10F8012F49
:10FCB00003F8012BF7E763682E461846B04505D0D8
:10FCC000327800B1027001360130F7E7A8EB050881
:10FCD0004344E4E708B509C81B1AC3F570508842CD
:10FCE00002D2104601F0E0FC994238BF194658187C
:10FCF00005D2B0F5705F28BF4FF4705008BD4FF4C7
:10FD00007050FBE72DE9F8430C46591C2046154678
:10FD10001F46FFF759FF064680B14FF00003EA196E
:10FD200029462046FFF788FFD4E901539D4208D0B9
:10FD30000DB100232B706368013363603046BDE86A
:10FD4000F8831B4A01212046FFF7C4FF23680746BA
:10FD5000A5EB0309FFF76FFE10EB090F1CBF002393
:10FD600000F80930236880461A460146954205D0BE
:10FD700009B11078087001320131F7E7D31A013365
:10FD80004344104619466568954207D019B192F868
:10FD900000C081F800C001320131F5E72D1A1D4481
:10FDA00020684744FFF742FEC4E90085A760C5E725
:10FDB000DDA101081346426810B5032A06D1BDE84B
:10FDC00010400A4600F11001FFF79CBF816802480D
:10FDD000F7F7E0F9002010BD5AA201082DE9F04123
:10FDE00005460E4661B1D0E90132D21A8A4209D3E2
:10FDF00000221E4403B11A700133B342FAD16B6082
:10FE0000BDE8F081114AFFF765FF8046FFF713FE5A
:10FE1000D5E9001407460A460346944205D00BB1C3
:10FE20001078187001320133F7E70023641A3C445C
:10FE3000264404B123700134B442FAD12868FFF794
:10FE4000F5FDC5E900744744AF60D9E73EA301085A
:10FE5000D0E90032D21A914210B503D9891AFFF7BE
:10FE6000BDFF10BD3CBF5B184360FAE770B50C46A0
:10FE7000012120461646FFF7A7FE054628B10121BD
:10FE80002046FFF7E5FF23681E70284670BD00007E
:10FE9000426808B5012A06D1BDE808400A4600F1CB
:10FEA0001001FFF7E3BF81680248F7F773F90020FC
:10FEB00008BD00BFCDA2010810B50C1A134605D02D
:10FEC00001462246184602F02EFC0346181910BDC2
:10FED0002DE9F0410446A2EB01081646A36822680A
:10FEE00008469B1A98450F4615D94046FFF7A3FDD3
:10FEF00005460346BE4205D00BB13A781A70013769
:10FF00000133F7E72068FFF791FD25604544C4E918
:10FF10000155BDE8F0816568AD1AA84504D83146A1
:10FF2000FFF7CAFF6060F4E70D442946FFF7C4FFFE
:10FF3000636829461A468E4205D00AB108781070C7
:10FF400001310132F7E7751B1D446560E1E70000F0
:10FF500070B5D0E9043100F110060446C91A3046E4
:10FF6000FFF732FE054640B1D4E90712914206D1AF
:10FF7000A1680648F7F70EF90025284670BD4FF036
:10FF800000033046FFF7A4FFF7E700BFF7A1010821
:10FF90002DE9F0418368A2EB010817460268044688
:10FFA0009B1A98450E4615D94046FFF744FD054675
:10FFB0000346B74205D0327803B11A7001360133D7
:10FFC000F7E72068FFF732FD25604544C4E9015595
:10FFD000BDE8F0814568AD1AA84505D839463046D8
:10FFE000FFF76AFF6060F3E70D4429463046FFF7EC
:10FFF00063FF636829461A468F4205D0087802B12C
:020000040801F1
:10000000107001310132F7E77D1B1D446560DFE7A9
:1000100037B50D4601A81146F7F7F6F90421284631
:10002000FFF7D2FD044630B14FF0000302AA01A948
:100030002846FFF7ADFF204603B030BDFFF7E8BF0D
:10004000426808B5022A06D1BDE808400A4600F118
:100050001001FFF7DDBF81680248F7F79BF8002029
:1000600008BD00BF05A30108FFF7EABFF7B50E46BC
:1000700004461046154603F043FA00237268C4E9AB
:100080000033013AA360032A12D8DFE802F0022B02
:100090003B412D49284603F021FA20B12B4928463F
:1000A00003F01CFA38B9012221463046FFF7DEFE84
:1000B000204603B0F0BD2649284603F00FFA20B1D0
:1000C0002449284603F00AFA08B90022ECE7002286
:1000D00002A941F8042D284603F03EFB021C18BF7C
:1000E0000122E1E702A941F8043D0022284603F07D
:1000F00033FB019B0246AB42DAD021463046FFF784
:1001000087FFD5E72A462146304600F025F8CFE79D
:1001100010F00106CCD1470839462046FFF754FDC0
:100120000028C5D039462046FFF792FEB742BFD01F
:10013000022105EB4600F7F73BF90028B8DB2368FE
:1001400098550136F2E700BF1FA20108D2A10108AD
:10015000D36D0108D7A10108F0B5436885B0032B22
:100160000D46164615D0014601A8FFF77FFFDDE9D1
:10017000011291420BD04FF000032846FFF7A8FE72
:1001800001240198FFF752FC204605B0F0BD002481
:10019000F7E7104603F0B4F9471C39462846FFF745
:1001A00013FD04460028EFD04FF00003F21931464A
:1001B0002846FFF741FDE7E70A4600F11001FFF787
:1001C000CBBFF8B50D461946284616461F46FFF721
:1001D000FBFC044630B14FF00003F21931462846CB
:1001E000FFF7D6FE2046F8BD1346426810B5042A34
:1001F00006D1BDE810400A4600F11001FFF7E1BF4B
:1002000081680248F6F7C6FF002010BD94A20108DD
:1002100010B10C2101F072BA704710B1012101F048
:100220006DBA704730B513460D460446AC4207D050
:100230001BB194E8070083E807000C330C34F5E7A2
:10024000184630BD10B5044638B1EFF795FF20468B
:10025000BDE81040282101F051BA10BD70B5044628
:10026000006AFFF7D5FFD4E90556AE4204D0284610
:10027000EFF782FF2835F8E7606908B1FFF7E2FF82
:10028000204670BDF8B5054600242826074FD5E95D
:1002900005031B1ADB107B439C4205D206FB0400BE
:1002A000FFF756FE0134F2E7F8BD00BFCDCCCCCC51
:1002B000F8B504462248F6F76DFF2248F6F76AFFC4
:1002C000D4E90531994218D0C91A1F4EC91071439B
:1002D0001E48F6F75FFF00252827D4E905031B1AFF
:1002E000DB1073439D4205D207FB0500FFF7FCFBC3
:1002F0000135F2E71648F6F74DFFD4E90831154EFF
:10030000C91A891071431448F6F744FF00250C27D9
:10031000D4E908031B1A9B1073439D4205D207FBC7
:100320000500FFF76BFB0135F2E70C48F6F732FFEB
:100330000B48F6F72FFFBDE8F8400A48F6F72ABF4A
:100340001EA40108AD670108CDCCCCCC28A40108BF
:100350003AA40108ABAAAAAA73A40108C6630108BB
:1003600083A401086D6201082DE9F043002487B0E1
:1003700006466846CDE90044029400F0A5FF6846B1
:1003800001F03AF84FF028082F4F304DD6E90523F9
:100390009B1ADB107B439C424ED208FB04F302EB1A
:1003A0000309D35C002B43D14846FFF748FB0146C5
:1003B000684601F013F84846FFF743FB042837D896
:1003C000DFE800F03803101A24004846FFF73BFB33
:1003D0000146684600F0B8FF50BBC0212846F3F73D
:1003E000FFFB25E04846FFF766FB0146684600F044
:1003F00091FFE8B9C421F1E74846FFF769FB0146E0
:10040000684600F0EBFF98B9C821E7E7494603A822
:10041000FFF727FBDDE903126846521A00F0B6FF2A
:1004200018B9CD212846F3F7DBFB0398FFF7F5FE5B
:100430000134ABE7D121D1E7684601F005F8029815
:1004400007B0BDE8F08300BFCDCCCCCC73A30108CE
:100450002DE9F04305460E4600244FF028081A4FB8
:100460008DB0D5E905239B1ADB107B439C4224D237
:1004700008FB042931461822684603F05BF8484619
:10048000FFF7DDFA182201460DEB020003F052F8E7
:100490006846F6F7D4FF6846F6F7E3FF06A8F6F7D6
:1004A000CEFF06A8F6F7DDFF182268460DEB020125
:1004B00003F02EF818B10134D3E74FF00009484695
:1004C0000DB0BDE8F08300BFCDCCCCCC2DE9F04F12
:1004D00006460F4600244FF00C09DFF86C808DB003
:1004E000D6E908535B1B9B1008FB03F39C4224D204
:1004F00018223946684603F01DF8182209FB04FB50
:100500000DEB020055F80B1003F014F86846F6F7EF
:1005100096FF6846F6F7A5FF06A8F6F790FF06A82F
:10052000F6F79FFF182268460DEB020105EB0B0A58
:1005300002F0EEFF18B10134D2E74FF0000A504646
:100540000DB0BDE8F08F00BFABAAAAAA10B5144643
:10055000FFF77EFF20B12146BDE81040FFF72CBE1B
:1005600010BD0000F8B50C46064640F2011200210D
:10057000224802F0F1F84FF4807221461F4802F041
:10058000C7F81E491E48F6F705FE1E491B4803F032
:1005900001F81C490546002002F0FCFF29460746E9
:1005A0003046FFF755FFA0B929463046FFF78EFFCA
:1005B000044600B301681448F6F7ECFDA36838461A
:1005C000984701242046F8BD39461048F6F7E2FD69
:1005D000F8E73A4629463046FFF7B8FF04460028B8
:1005E000F2D00B48F6F7D6FD0A48F6F7D3FD3046B1
:1005F000FFF75EFEE6E729460748E7E7504E002092
:100600009CA40108A2A40108A4A40108CDA4010887
:10061000B9A40108C6630108E6A4010810B54FF4A7
:1006200080720649044600F093FF002805DD20464D
:10063000BDE810400149FFF795BF10BD504D0020A7
:1006400038B514461D46FFF703FF28B12A46214658
:10065000BDE83840FFF7AEBB38BD10B51446FFF714
:10066000F7FE20B12146BDE81040FFF7E9BC10BD00
:1006700010B51446FFF7ECFE10B12146FFF708FC59
:10068000002010BD38B514461D46FFF7E1FE28B125
:100690002A462146BDE83840FFF7A6BD38BD000018
:1006A0002DE9F04700248CB0074603A8CDE90344A8
:1006B000059400F009FE214603A8009400F020FFF5
:1006C0000146002834D0214603A800F0A2FE40F2E3
:1006D000E7330446009300263546DFF8F890009B88
:1006E000B34273D9214603A800F0C5FE8246002814
:1006F0006CD1182321460DEB030203A800F04CFE39
:100700000444214603A800F0C4FE8046B0B10CAA00
:10071000214642F828AD03A800F0DCFD029A04440B
:1007200006A93846FFF799FF00B101350136D6E733
:100730006A4603A800F074FE0446CCE7214603A8ED
:1007400000F0F1FE70B10CAA02F8288D214603A832
:1007500000F0EAFD9DF80820044406A93846FFF79A
:1007600087FFE1E7214603A800F0AEFE804668B1AE
:1007700002AB01AA214603A800F01FFEDDE9012318
:10078000044406A93846FFF75BFFCDE7214603A8DE
:1007900000F08CFE90B10CAB43F8288D01AA2146E5
:1007A00003A8CDF8048000F0E0FD9DF80830044473
:1007B000019A06A93846FFF765FFB5E7039B48464F
:1007C000195D01F0E001F6F7E5FCAFE728460CB053
:1007D000BDE8F087ADA3010808B5FFF739FE18B1F1
:1007E000BDE80840FFF72FB908BD10B5044608461C
:1007F0001146FFF72DFE014620B9C4E90000A060B4
:10080000204610BD2046FFF72CF9F9E708B5FFF7A1
:100810001FFE18B1BDE80840FFF74DB908BD08B587
:10082000FFF716FE18B1BDE80840FFF751B908BD43
:10083000002370B5D1E90025AD1A0446C0E90033A4
:1008400083600E46284601D0F6F736FDC4E9000065
:100850000544A560D6E90053024629468B4205D0DF
:100860000AB10E78167001310132F7E75B1B1844AC
:100870006060204670BD38B504460D460B781030D8
:1008800000F8103C4B68103140F80C3C51F8083C23
:1008900040F8083C51F8043C40F8043CFFF7C8FF1E
:1008A00005F11C0104F11C00FFF7C2FF204638BD12
:1008B0002DE9F843D0E90054641B9146A2101F4C67
:1008C00006465443B4F5705F0F4602D11C4800F051
:1008D000EBFE002C14BF22460122A418A1EB050553
:1008E00026D2B4F5705F23D82CB30C206043F6F702
:1008F000E3FC804618EB05031CBF99E8070083E87A
:100900000700424639463068FFF78CFC716800F1F9
:100910000C023846FFF786FC05463068FFF778FC86
:100920000C2303FB0484C6E90085B460BDE8F883AA
:100930004FF47054D9E7A046DCE700BFABAAAAAADF
:10094000DDA101082DE9F043054685B008460C46B7
:1009500017461E4602F0D4FD172803D980212D48E2
:10096000F3F73EF9CDE90147D5E9087803962A4A1D
:10097000A8EB0706B41054430134B4F5705F02D9F4
:10098000264800F091FEAB6ADB1B9B1053439C4250
:1009900015D94FF00C0909FB04F91CB14846F6F7CC
:1009A0008BFC0446224641463846FFF73BFC286A4A
:1009B000FFF72EFC26442C624C446E62AC62AA6A9D
:1009C000D5E9080314491B1A9B10121A4B439210C5
:1009D0004A430133934206D91148F6F7DBFB8A21DB
:1009E0000C48F3F7FDF8D5E9093293420AD023B158
:1009F00004AA12E9070083E807000C336B6205B014
:100A0000BDE8F08301AA194605F12000FFF750FF69
:100A1000F5E700BF73A30108ABAAAAAAC2A1010807
:100A200058A30108002310B50446C0E90533C0E906
:100A30000733C0E90933064B8021036100F081FDD3
:100A40002046044B044A0549FFF77CFF204610BDB1
:100A5000D04C0020990A010809A5010815A5010834
:100A600010B5084C2368DB0709D40748FFF7DAFF05
:100A70000123064A06490448236001F0FFFC0248AE
:100A800010BD00BFCC4C0020544F0020A84F0020C8
:100A90005D020108FFF7E4BF08B5FFF7E1FFBDE81D
:100AA0000840FFF705BC0022C0E90022826010B5B3
:100AB0000C6804600A6042684C6844604A6082685E
:100AC0008C6884608A6010BD70B50E460546144679
:100AD000B54217D09CB12B7805F1100123706B68DB
:100AE00004F110006360AB68A360EB68E360FFF79C
:100AF000DAFF05F11C0104F11C00FFF7D4FF2834D4
:100B00002835E5E7204670BD2DE9F843D0E90064BB
:100B1000A41BE310234C05465C43B4F5705F0F46FD
:100B2000914602D1204800F0BFFD002C14BF23469F
:100B30000123E418A1EB060623D2B4F5705F20D898
:100B400014B328206043F6F7B7FB804618EB060085
:100B500002D04946FFF78FFE394642462868FFF724
:100B6000B3FF696800F128023846FFF7ADFFD5E909
:100B700000690746B14509D03046EFF7FDFA28363F
:100B8000F8E74FF47054DCE7A046DFE7286808B1C7
:100B9000FFF758FB282303FB0484C5E90087AC60FA
:100BA000BDE8F883CDCCCCCCDDA101082DE9F04720
:100BB000D0E9055704460E46DFF80C818AB0AF42F3
:100BC0001BD029466846FFF756FE6846FEF737FFFA
:100BD00081463046FEF733FF01464846F6F770FC83
:100BE00030B13046FEF72BFF01464046F6F7D2FA09
:100BF0006846EFF7C1FA2835E1E7D4E905892E4ABE
:100C0000A9EB0807FD1055430135B5F5705F02D912
:100C10002A4800F049FDE369A3EB0803DB105343C6
:100C20009D4220D94FF0280A0AFB05FA1DB1504613
:100C3000F6F742FB0546494640462A46FFF744FF81
:100C4000D4E90589C14505D04046EFF795FA08F18A
:100C50002808F7E7606908B1FFF7F4FA2F446561E7
:100C60005544A761E561E269D4E9050312491B1AFD
:100C7000DB10121A4B43D2104A430133934206D978
:100C80000F48F6F787FA75210E48F2F7A9FFD4E965
:100C90000603984209D010B13146FFF7ECFDA36975
:100CA0002833A3610AB0BDE8F0870146324604F15B
:100CB0001400FFF729FFF5E7CDCCCCCCC2A1010889
:100CC000FFA3010873A30108CDA3010808B50848D4
:100CD000F6F760FAFFF7C4FEFFF7D4FA0548F6F717
:100CE00059FAFFF7BDFEBDE80840FFF7E1BA00BFC3
:100CF000E7A60108FFA60108F7B505464FF4007006
:100D0000F6F7DAFA044618B926211848F2F768FF10
:100D10004FF400720021204601F01EFD4FF40072D6
:100D200021462846FFF720FB114D124E02AF47F82F
:100D3000040D01461048F6F72DFA7368294604227F
:100D40006868984704226868736839461044984771
:100D500068687368019A2146083098470748F6F793
:100D600019FA2046F6F792FA03B0F0BDB0A50108D3
:100D7000904F0020844F0020F8A5010813A6010819
:100D80002DE9F74FFFF76CFE2E4F06462E48F6F77B
:100D900001FAB846DFF8CC90DFF8CCA0F9F76AFD8D
:100DA0002A4D38602B68AB46294C002B37D003F511
:100DB0006A436033984232D223782BB92548F6F73C
:100DC000E9F92548F6F7E6F9012330462370FFF7E5
:100DD00025FC41F2883352464FF0FF310020FAF7EC
:100DE000A1F90190F9F746FD019BC8F8000023B96D
:100DF000237813B13046FFF711FCDAF80030DA0738
:100E000044BFD8F800202A609B07C7D50023CBF841
:100E10000030D9F80830002BBED09847BCE72378C3
:100E200063B13046FFF768FF0C48F6F7B3F90C489A
:100E3000F6F7B0F9D9F8083003B1984700232370CA
:100E40002B60C6E7A44F002057A60108A04F002042
:100E5000984F00206CA601088FA60108B2A60108D1
:100E6000C4A60108844F00209C4F002010B5FFF756
:100E7000F7FD0446FFF740FF2046FFF719FABDE8EB
:100E8000104003480023012202210068FAF78EB9BE
:100E9000804F002010B5FFF7E3FD0446FFF72CFF5D
:100EA0002046BDE81040FFF703BA00002DE9F341EA
:100EB0000024154D154E884602A941F8084D04221C
:100EC00007463368686898472A6800998A4204D0C0
:100ED0000F48F6F75FF9204613E0042268680DEB2F
:100EE000020110443368984701990A48F6F752F90D
:100EF000019A4245EFD86868336839460830984708
:100F0000019802B0BDE8F081904F0020844F00208E
:100F100022A601083DA6010882B0F0B587B003AC57
:100F200084E807000D93049B1BB9EF215648F2F7A4
:100F300057FE039B1BB9F0215348F2F751FE94E88A
:100F40000700524B83E80700514B0DAA92E80300BB
:100F500083E80300FFF784FD06464E4B4E4A4F4997
:100F6000FFF7F0FC4E4B4F4A4F493046FFF7EAFC83
:100F70004E4B4F4A4F493046FFF7E4FC4FF40070A8
:100F8000F6F79AF9044670B14FF40072002101F0AF
:100F9000E3FB4FF400712046FFF788FF024660B97B
:100FA0002046F6F773F94448F6F7F4F83046FFF7B1
:100FB00069F94248F6F7EEF806E021463046FFF7B9
:100FC0006FFB2046F6F762F94FF40070F6F774F9FC
:100FD00005464FF40072002101F0BEFB4FF4007192
:100FE0002846FFF763FF0746F8B9F6F74FF928469A
:100FF000F6F74CF93248F6F7CDF8FFF731FDFFF779
:101000007BFE304BFA22019301232F4900932F4896
:101010000023F9F70DFA90BB4FF485711A4807B019
:10102000BDE8F04002B0F2F7DBBD4FF40070F6F718
:1010300043F9044618B966211348F2F7D1FD4FF47D
:1010400000720021204601F087FB4FF40072214618
:101050003046FFF789F908B92046C6E78742FBD139
:101060000023E15CEA5C9142F6D101339F42F8D162
:101070002046F6F70BF92846F6F708F9C1E707B05E
:10108000BDE8F04002B07047B0A50108844F0020D1
:10109000904F0020950E010819A5010825A501080B
:1010A000CD0C01082AA5010845A501086D0E01080F
:1010B0004DA5010865A501086AA50108FFA601085C
:1010C0008EA50108804F0020A5A50108810D01080B
:1010D000F0B508B90020F0BD002746684D1CB542A8
:1010E0001760F7D803685C185B5C03F01F03A3F17B
:1010F000180103298FBF38460D49C91811F8180C7B
:101100000544AE42E6D304280DD8DFE800F004031E
:10111000070C0C00637813600130DCE7B4F8013091
:101120005BBA9BB2F7E7D4F801301BBAF3E700BF14
:1011300017A70108F7B51F46436816464A1C9A428E
:1011400005460C4617D803685B5C03F0C003402BD0
:1011500011D196B101AAFFF7BBFF50B1019A044427
:101160006B68A118994206D8296810440C44346071
:101170003A6003B0F0BD0020FBE73046F9E72DE907
:10118000F7439946436817464A1C9A4280460D46E3
:1011900024D803685B5C03F0C003402B1ED1FFB171
:1011A00001AAFFF795FF0446A0B1019E09F10109CC
:1011B000B14513D30544D8F8043072199A420DD8BA
:1011C000D8F8001032462944384601F0A1FA00232D
:1011D0003444BB55204603B0BDE8F0830024F9E752
:1011E0003C46F7E7F0B5002931D0172A1CD8D3B216
:1011F000A3F11804032C8CBF0024164C8D689CBFEF
:10120000E41814F8184C6F1C4E6804EB070CB44536
:101210001DD20E6818438F60705500200130231ACC
:101220005D1C0BD1601CF0BDFF2A05D9B2F5803FD3
:101230002CBF1A231923DBE71823D9E78E680D6822
:10124000DB00771C22FA03F38F60AB55E6E7002042
:10125000E9E700BF17A70108172BF8B50D4616469A
:101260001C4612D8DBB2A3F11802032A8FBF00225A
:10127000144A9B1813F8182CAB680132234413440A
:101280006A6893420BD30020F8BDFF2B05D9B3F554
:10129000803F34BF19231A23E5E71823E3E72246EA
:1012A0002946FFF79FFF07460028ECD02868AB6867
:1012B0003146184401F02CFAAA68E0192244AA60C9
:1012C000E2E700BF17A7010818B10023C0E9001228
:1012D00083607047436873B514464A1C9A420646B9
:1012E0000D4602D9002002B070BD03685B5C13F0AC
:1012F000C00FF7D1002CF5D001AAFFF7E9FE0028B6
:10130000F0D03268019B525D12F0E00F18BFDB4352
:101310002360E8E70A1EABBF014601460020D24326
:10132000B8BF2020FFF75EBF03685B5C03F0E001FD
:10133000E02907D132B1A3F1F5014B424B411370C3
:101340000120704700207047836810B544685A1C1C
:10135000A24208D2002914BFF524F4240168826057
:101360000120CC5410BD0020FCE7F0B446684F1CAF
:10137000B74208D805686C5C04F0E004402C02D148
:10138000F0BCFFF7D7BE0020F0BC704713460A46FA
:1013900001464020FFF760BFF0B446684F1CB742DB
:1013A00008D805686C5C04F0E004602C02D1F0BC45
:1013B000FFF7E5BE0020F0BC7047F0B446684F1C54
:1013C000B74208D805686C5C04F0E004602C02D1D8
:1013D000F0BCFFF7AFBE0020F0BC704770B505460B
:1013E00008460C4602F08CF8224603462946BDE822
:1013F00070406020FFF730BF836841685A1C8A4202
:101400003FBF8260BF220168012034BFCA54002060
:1014100070470368585CA0F1BF03584258417047B9
:1014200013B5036814465B5C03F0E003A02B07D1FF
:1014300042B101AAFFF74CFE019B236002B010BD30
:101440000020FBE71046F9E7836841685A1C8A428E
:101450003FBF8260FF220168012034BFCA540020D0
:10146000704730B18068013888428CBF002001206D
:1014700070470120704708B50246FFF7F2FF30B908
:101480001268505CA0F1FF035842584108BD01208A
:10149000FCE743688B4207D903685B5C13F0C00F1D
:1014A0000CBF0120002070470020704743688B422A
:1014B00008D90368585C00F0E000A0F140035842EE
:1014C000584170470020704743688B4208D9036831
:1014D000585C00F0E000A0F16003584258417047AA
:1014E0000020704743688B4208D90368585C00F0BD
:1014F000E000A0F1A0035842584170470020704717
:1015000010B50446FFF7EEFF50B163688B4208D96F
:101510002368585C00F01F00A0F11F035842584197
:1015200010BD0020FCE743688B4208D90368585C73
:101530000C30C0B201288CBF002001207047002071
:1015400070470023C0E9013303690160C36070473D
:10155000F8B503680446002B0D46164603DC362119
:101560002948F2F73DFB32460021284601F0F4F805
:10157000D4E90170B8420CD00021236801EB070CBC
:101580009CFBF3F203FB12C2904205D1002088427B
:1015900004D14FF0FF3031E00131EFE7C21992FB87
:1015A000F3FE03FB1E2ED4F80CC01CF80EE0BEF1B7
:1015B0000A0F26D128B3013A92FBF3F103FB112263
:1015C000002106F1FF3E71450ED2E7686368FB5CBF
:1015D0006B5467682668013797FBF6F306FB1377B1
:1015E000013188426760EEDA1CF802300D2B4FF0B3
:1015F000000304D1054405F8013C0138F8BD2B5423
:10160000FCE70130C3E700BF1BA7010810B5044683
:101610000846C4E900120021A16001F09DF82046AF
:1016200010BD0000836870B5044640689E1886426D
:10163000154605D907481621F2F7D2FA002070BDE9
:101640002068184401F064F8A26801202A44A260CE
:10165000F5E700BF63A7010807B502AB03F8011D5A
:1016600001221946FFF7DEFF03B05DF804FB0068B6
:1016700070478068704713B5044601A8F5F7CDFEA2
:10168000022201A92046FFF7CDFF02B010BD13B51D
:10169000044601A8F5F7C1FE022201A92046FFF782
:1016A000C1FF02B010BD000008B501460448F5F7BF
:1016B00071FDBDE808400C210248F2F791BA00BF65
:1016C0009BA70108B9A7010808B50448F5F762FD12
:1016D000BDE808401C210248F2F782BA0AA80108B6
:1016E00037A80108F5F7E8BD10B90248F5F752BD73
:1016F000F5F7CCBDF5A70108F5F7DEBDFFF7F4BFA0
:1017000073B50E4C8DF8070023690E4698470546C1
:1017100020B963699847284602B070BD6368D0223B
:1017200001210DF107009847A368D022012130461E
:101730009847636998470125EDE700BF58010020ED
:10174000002373B50A241D4602AE06F8053D314656
:101750000F20FFF7D5FF9DF803305B070ED549F644
:10176000FE720195019B934204DD013CEFD12046BE
:1017700002B070BD019B01330193F3E70120F7E74D
:10178000F7B50B4C074623690E469847054620B926
:1017900063699847284603B0F0BD8DF804708DF852
:1017A00005602368D022022101A898470546EFE78B
:1017B0005801002010B50C4CA37F0BB9637F7BB997
:1017C000E3685A1E03320CD8984728B95921BDE85E
:1017D00010400648F2F704BA012363770023A37789
:1017E00010BD5F21F3E700BF5801002073A8010876
:1017F00007B5FFF7DFFFFFF7A3FF38B90E4B0F4820
:101800009B699847002003B05DF804FB0DF10701C8
:101810000E20FFF775FF18B90122074B9A77F1E701
:101820009DF807100E2041F080018DF80710FFF79A
:10183000A7FF0028F0D0E5E758010020B2A8010872
:1018400084B073B506AC84E80F00334C06AE254671
:101850000FCE0FC596E80700002385E807006377E1
:10186000A3690BB92D4BA36163682BB1A3681BB1AE
:1018700023680BB1E3684BB99D212948F2F7B0F911
:10188000002002B0BDE8704004B0704723691BB966
:10189000A1212348F2F7A4F963691BB9A2212048CA
:1018A000F2F79EF9FFF786FF04210E208DF807104E
:1018B000FFF766FF38B9A3691A4898470123A37751
:1018C000FFF778FFDCE7FFF73BFF10B9A369164885
:1018D000F3E7002502A901F8015D0F20FFF710FFD3
:1018E00040B19DF90730AB4213DAA3690F4898471E
:1018F0000123237700210F20FFF742FF18B9C221EF
:101900000748F2F76DF90A48A36998470120607704
:10191000B7E72577EEE700BF580100208D7100087A
:1019200073A80108E0A80108B2A8010802A90108EB
:1019300033A90108024B0A465B680146302018476C
:10194000AC4F0020024B0A461B6801463020184766
:10195000AC4F00202F4B10B51B7823B940F201117A
:101960002D48F2F73DF92D4CA368984700211F2020
:10197000FFF7E8FF20B94FF482712748F2F730F9FA
:1019800090211E20FFF7DEFF20B94FF4837122481B
:10199000F2F726F900212020FFF7D4FF20B940F20A
:1019A00007111D48F2F71CF900212120FFF7CAFF9B
:1019B00020B94FF484711848F2F712F9002122205F
:1019C000FFF7C0FF20B940F209111348F2F708F9F8
:1019D00000212320FFF7B6FF20B94FF485710E4890
:1019E000F2F7FEF800212420FFF7ACFF20B940F207
:1019F0000B110948F2F7F4F800212520FFF7A2FFA8
:101A000020B94FF486710448F2F7EAF8E368BDE8BC
:101A100010401847C44F0020BFA90108AC4F002058
:101A200084B073B506AC84E80F002C4C06AE254696
:101A30000FCE0FC596E8030085E8030063690BB974
:101A4000274B6361636927489847636823B940F26D
:101A50007D112548F2F7C4F8236823B94FF4BF710C
:101A60002148F2F7BDF8A36823B940F27F111E4860
:101A7000F2F7B6F8E36823B94FF4C0711A48F2F7E9
:101A8000AFF8236923B940F281111748F2F7A8F89B
:101A9000A36898470DF107010F20FFF74BFFE3689C
:101AA000984763699DF80710104898479DF80730DC
:101AB000332B08D00E4863699847002002B0BDE878
:101AC000704004B0704701250A4B1D70FFF742FFBC
:101AD0000948636998472846F0E700BFAC4F0020EB
:101AE0008D71000851A90108BFA9010864A9010866
:101AF00089A90108C44F00209DA9010800BF7047B3
:101B0000174B37B51B781BB93C211648F2F768F81C
:101B10000021012000F0E1F9E0B9134C6420E368F2
:101B20009847322500F0EFF901280BD0002302A9D5
:101B300021F8023D0D4800F0EEF970B9BDF906003C
:101B400003B030BDE36819209847013DEAD147F65C
:101B5000FD70F5E747F6FF70F2E747F6FE70EFE736
:101B6000CD4F002027AA0108B8500020C54F002003
:101B7000F8B5144B05461B781BB957211248F2F7EC
:101B80002FF80021012000F0A8F933240F4E00F0B7
:101B9000BAF940B904466E1C05F581772B78A3424B
:101BA00008DC0120F8BDF36819209847013CEED10C
:101BB0002046F7E73946304600F0ADF901340836E3
:101BC0000237EBE7CD4F002027AA0108B8500020CC
:101BD000F0B5224B85B01B7805461BB99B212048E8
:101BE000F1F7FEFF1F4EFF24B369984700232A46F2
:101BF00047F6FF70CDE901338DF80C3005F5A17182
